S01800004343534D6F64756C65535733305765622E73726563A2
S315080080000000012075DA0008FDD0000805D1000837
S315080080100DD1000815D100081DD100080000000088
S3150800802000000000000000000000000025D1000844
S3150800803031D10008000000003DD1000849D10008F0
S31508008040BDDA0008BDDA0008BDDA0008BDDA0008A6
S31508008050BDDA0008BDDA0008BDDA0008BDDA000896
S31508008060BDDA0008BDDA0008BDDA0008BDDA000886
S31508008070BDDA0008BDDA0008BDDA0008BDDA000876
S31508008080BDDA0008BDDA0008BDDA0008BDDA000866
S3150800809055D10008BDDA0008BDDA0008BDDA0008C7
S315080080A0BDDA0008BDDA0008BDDA0008BDDA000846
S315080080B0BDDA000869D10008BDDA0008BDDA000893
S315080080C0BDDA0008BDDA0008BDDA0008BDDA000826
S315080080D0BDDA00087DD1000891D10008A5D10008B5
S315080080E0BDDA0008BDDA0008BDDA000800000000A5
S315080080F00000000000000000000000000000000072
S315080081000000000000000000BDDA0008BDDA000823
S31508008110BDDA0008B9D10008BDDA0008BDDA0008E2
S31508008120BDDA0008BDDA0008BDDA0008BDDA0008C5
S31508008130BDDA0008BDDA0008BDDA0008CDD10008AE
S31508008140BDDA0008E1D10008BDDA0008BDDA00088A
S315080081500000000000000000000000000000000011
S315080081600000000000000000000000000000000001
S3150800817000000000000000000000000000000000F1
S3150800818000000000000000000000000000000000E1
S3150800819000000000000000000000000000000000D1
S315080081A000000000000000000000000000000000C1
S315080081B000000000000000000000000000000000B1
S315080081C000000000000000000000000000000000A1
S315080081D00000000000000000000000000000000091
S309080081E05FF8E0F165
S315080081E810B5054C237833B9044B13B10448AFF3DB
S315080081F800800123237010BD400200200000000003
S31508008208B85C010808B5034B1BB103490348AFF32B
S31508008218008008BD0000000044020020B85C010880
S31508008228034613F8012B002AFBD1181A01387047A0
S3150800823881F0004102E000BF83F0004330B54FEA01
S3150800824841044FEA430594EA050F08BF90EA020F6E
S315080082581FBF54EA000C55EA020C7FEA645C7FEA01
S31508008268655C00F0E2804FEA5454D4EB5555B8BF24
S315080082786D420CDD2C4480EA020281EA030382EA95
S31508008288000083EA010180EA020281EA0303362D27
S3150800829888BF30BD11F0004F4FEA01314FF4801CFA
S315080082A84CEA113102D0404261EB410113F0004F0C
S315080082B84FEA03334CEA133302D0524263EB4303C3
S315080082C894EA050F00F0A780A4F10104D5F1200E61
S315080082D80DDB02FA0EFC22FA05F2801841F10001BC
S315080082E803FA0EF2801843FA05F359410EE0A5F190
S315080082F820050EF1200E012A03FA0EFC28BF4CF0C1
S31508008308020C43FA05F3C01851EBE37101F0004576
S3150800831807D54FF0000EDCF1000C7EEB00006EEB83
S315080083280101B1F5801F1BD3B1F5001F0CD349080D
S315080083385FEA30004FEA3C0C04F101044FEA445264
S3150800834812F5800F80F09A80BCF1004F08BF5FEAEB
S31508008358500C50F1000041EB045141EA050130BDCB
S315080083685FEA4C0C404141EB0101013C28BFB1F5DD
S31508008378801FE9D291F0000F04BF01460020B1FA28
S3150800838881F308BF2033A3F10B03B3F120020CDAFB
S315080083980C3208DD02F1140CC2F10C0201FA0CF0D9
S315080083A821FA02F10CE002F11402D8BFC2F1200C3E
S315080083B801FA02F120FA0CFCDCBF41EA0C019040F4
S315080083C8E41AA2BF01EB0451294330BD6FEA04043D
S315080083D81F3C1CDA0C340EDC04F11404C4F1200228
S315080083E820FA04F001FA02F340EA030021FA04F33A
S315080083F845EA030130BDC4F10C04C4F1200220FA91
S3150800840802F001FA04F340EA0300294630BD21FACE
S3150800841804F0294630BD94F0000F83F4801306BF94
S3150800842881F480110134013D4EE77FEA645C18BF88
S315080084387FEA655C29D094EA050F08BF90EA020F1F
S3150800844805D054EA000C04BF1946104630BD91EA17
S31508008458030F1EBF0021002030BD5FEA545C05D11A
S315080084684000494128BF41F0004130BD14F5800459
S315080084783CBF01F5801130BD01F0004545F0FE41CD
S3150800848841F470014FF0000030BD7FEA645C1ABF02
S31508008498194610467FEA655C1CBF0B46024650EA39
S315080084A8013406BF52EA033591EA030F41F4002165
S315080084B830BD00BF90F0000F04BF0021704730B5EB
S315080084C84FF4806404F132044FF000054FF00001C0
S315080084D850E700BF90F0000F04BF0021704730B581
S315080084E84FF4806404F1320410F0004548BF404256
S315080084F84FF000013EE700BF42004FEAE2014FEAAB
S3150800850831014FEA02701FBF12F07F4393F07F4F85
S3150800851881F06051704732F07F4208BF704793F088
S315080085287F4F04BF41F40021704730B54FF460749B
S3150800853801F0004521F000411CE700BF50EA01029E
S3150800854808BF704730B54FF000050AE050EA010247
S3150800855808BF704730B511F0004502D5404261EBB7
S3150800856841014FF4806404F132045FEA915C3FF4F8
S31508008578D8AE4FF003025FEADC0C18BF03325FEA95
S31508008588DC0C18BF033202EBDC02C2F1200300FA46
S3150800859803FC20FA02F001FA03FE40EA0E0021FA6B
S315080085A802F11444BDE600BF70B54FF0FF0C4CF459
S315080085B8E06C1CEA11541DBF1CEA135594EA0C0F0B
S315080085C895EA0C0F00F0DEF82C4481EA030621EA46
S315080085D84C5123EA4C5350EA013518BF52EA033581
S315080085E841F4801143F4801338D0A0FB02CE4FF033
S315080085F80005E1FB02E506F00042E0FB03E54FF063
S315080086080006E1FB03569CF0000F18BF4EF0010E5A
S31508008618A4F1FF04B6F5007F64F5407404D25FEA56
S315080086284E0E6D4146EB060642EAC62141EA555109
S315080086384FEAC52040EA5E504FEACE2EB4F1FD0C4B
S3150800864888BFBCF5E06F1ED8BEF1004F08BF5FEAC9
S31508008658500E50F1000041EB045170BD06F000467B
S3150800866846EA010140EA020081EA0301B4EB5C0428
S31508008678C2BFD4EB0C0541EA045170BD41F4801120
S315080086884FF0000E013C00F3AB8014F1360FDEBF45
S31508008698002001F0004170BDC4F10004203C35DA21
S315080086A80C341BDC04F11404C4F1200500FA05F3A4
S315080086B820FA04F001FA05F240EA020001F0004245
S315080086C821F0004110EBD37021FA04F642EB0601BB
S315080086D85EEA430E08BF20EAD37070BDC4F10C04E5
S315080086E8C4F1200500FA04F320FA05F001FA04F2A9
S315080086F840EA020001F0004110EBD37041F1000195
S315080087085EEA430E08BF20EAD37070BDC4F120059F
S3150800871800FA05F24EEA020E20FA04F301FA05F207
S3150800872843EA020321FA04F001F0004121FA04F2AF
S3150800873820EA020000EBD3705EEA430E08BF20EA7F
S31508008748D37070BD94F0000F0FD101F000464000B9
S3150800875841EB010111F4801F08BF013CF7D041EA3B
S31508008768060195F0000F18BF704703F0004652003F
S3150800877843EB030313F4801F08BF013DF7D043EA10
S315080087880603704794EA0C0F0CEA135518BF95EAC6
S315080087980C0F0CD050EA410618BF52EA4306D1D14D
S315080087A881EA030101F000414FF0000070BD50EA6C
S315080087B8410606BF1046194652EA430619D094EAF6
S315080087C80C0F02D150EA013613D195EA0C0F05D1E0
S315080087D852EA03361CBF104619460AD181EA030134
S315080087E801F0004141F0FE4141F470014FF00000EC
S315080087F870BD41F0FE4141F4780170BD70B54FF087
S31508008808FF0C4CF4E06C1CEA11541DBF1CEA135506
S3150800881894EA0C0F95EA0C0F00F0A7F8A4EB0504E8
S3150800882881EA030E52EA03354FEA013100F08880DF
S315080088384FEA03334FF0805545EA131343EA1263A8
S315080088484FEA022245EA111545EA10654FEA00265D
S315080088580EF000419D4208BF964244F1FD0404F516
S31508008868407402D25B084FEA3202B61A65EB030572
S315080088785B084FEA32024FF480104FF4002CB6EB2F
S31508008888020E75EB030E22BFB61A754640EA0C00AF
S315080088985B084FEA3202B6EB020E75EB030E22BFEF
S315080088A8B61A754640EA5C005B084FEA3202B6EB30
S315080088B8020E75EB030E22BFB61A754640EA9C00EF
S315080088C85B084FEA3202B6EB020E75EB030E22BFBF
S315080088D8B61A754640EADC0055EA060E18D04FEA7D
S315080088E8051545EA16754FEA06164FEAC30343EA1D
S315080088F852734FEAC2025FEA1C1CC0D111F4801FEA
S315080089080BD141EA00014FF000004FF0004CB6E7E2
S3150800891811F4801F04BF01430020B4F1FD0C88BF81
S31508008928BCF5E06F3FF6AFAEB5EB030C04BFB6EB8C
S31508008938020C5FEA500C50F1000041EB045170BD7F
S315080089480EF0004E4EEA113114EB5C04C2BFD4EBAC
S315080089580C0541EA045170BD41F480114FF0000E30
S31508008968013C90E645EA060E8DE60CEA135594EAAC
S315080089780C0F08BF95EA0C0F3FF43BAF94EA0C0FAF
S315080089880AD150EA01347FF434AF95EA0C0F7FF424
S3150800899825AF104619462CE795EA0C0F06D152EA78
S315080089A803353FF4FDAE1046194622E750EA41065C
S315080089B818BF52EA43067FF4C5AE50EA41047FF46D
S315080089C80DAF52EA43057FF4EBAE12E74FF0FF3CD2
S315080089D806E000BF4FF0010C02E000BF4FF0010CA3
S315080089E84DF804CD4FEA410C7FEA6C5C4FEA430C1C
S315080089F818BF7FEA6C5C1BD001B050EA410C0CBF6B
S31508008A0852EA430C91EA030F02BF90EA020F0020CC
S31508008A18704710F1000F91EA030F58BF994208BF33
S31508008A2890422CBFD8176FEAE37040F001007047F0
S31508008A384FEA410C7FEA6C5C02D150EA013C07D147
S31508008A484FEA430C7FEA6C5CD6D152EA033CD3D092
S31508008A585DF8040B704700BF8446104662468C468C
S31508008A681946634600E000BF01B5FFF7B7FF0028BF
S31508008A7848BF10F1000F01BD4DF808EDFFF7F4FFE8
S31508008A880CBF012000205DF808FB00BF4DF808ED73
S31508008A98FFF7EAFF34BF012000205DF808FB00BF96
S31508008AA84DF808EDFFF7E0FF94BF012000205DF8B8
S31508008AB808FB00BF4DF808EDFFF7CEFF94BF01206D
S31508008AC800205DF808FB00BF4DF808EDFFF7C4FF66
S31508008AD834BF012000205DF808FB00BF4FEA410CAF
S31508008AE87FEA6C5C02D150EA013C0AD14FEA430C92
S31508008AF87FEA6C5C02D152EA033C02D14FF00000CF
S31508008B0870474FF0010070474FEA410212F500120C
S31508008B1815D211D56FF47873B3EB625212D94FEAAE
S31508008B28C12343F0004343EA505311F0004F23FA98
S31508008B3802F018BF404270474FF00000704750EAED
S31508008B48013005D111F0004008BF6FF000407047AA
S31508008B584FF00000704700BF4FEA4102B2F1E04308
S31508008B6824BFB3F5001CDCF1FE5C0DD901F0004CFE
S31508008B784FEAC0024CEA5070B2F1004F40EB83004E
S31508008B8808BF20F00100704711F0804F21D113F17A
S31508008B983872BCBF01F00040704741F480114FEAB3
S31508008BA85252C2F11802C2F1200C10FA0CF320FA3C
S31508008BB802F018BF40F001004FEAC1234FEAD32359
S31508008BC803FA0CFC40EA0C0023FA02F34FEA4303C3
S31508008BD8CCE77FEA625307D150EA01331EBF4FF04C
S31508008BE8FE4040F44000704701F0004040F0FE4067
S31508008BF840F40000704700BF80F0004002E000BF64
S31508008C0881F0004142001FBF5FEA410392EA030F61
S31508008C187FEA226C7FEA236C6AD04FEA1262D2EBAB
S31508008C281363C1BFD218414048404140B8BF5B42B0
S31508008C38192B88BF704710F0004F40F4000020F049
S31508008C487F4018BF404211F0004F41F4000121F05F
S31508008C587F4118BF494292EA030F3FD0A2F10102A9
S31508008C6841FA03FC10EB0C00C3F1200301FA03F1E7
S31508008C7800F0004302D5494260EB4000B0F5000F0A
S31508008C8813D3B0F1807F06D340084FEA310102F1C9
S31508008C980102FE2A51D2B1F1004F40EBC25008BF7B
S31508008CA820F0010040EA03007047490040EB000045
S31508008CB8013A28BFB0F5000FEDD2B0FA80FCACF146
S31508008CC8080CB2EB0C0200FA0CF0AABF00EBC25073
S31508008CD852421843BCBFD0401843704792F0000F61
S31508008CE881F4000106BF80F400000132013BB5E7B4
S31508008CF84FEA41037FEA226C18BF7FEA236C21D02A
S31508008D0892EA030F04D092F0000F08BF084670478E
S31508008D1890EA010F1CBF0020704712F07F4F04D15C
S31508008D28400028BF40F00040704712F100723CBF6F
S31508008D3800F50000704700F0004343F0FE4040F499
S31508008D48000070477FEA226216BF08467FEA236357
S31508008D580146420206BF5FEA412390EA010F40F442
S31508008D68800070474FF0000304E000BF10F000438E
S31508008D7848BF40425FEA000C08BF704743F0964375
S31508008D8801464FF000001CE050EA010208BF704790
S31508008D984FF000030AE000BF50EA010208BF704717
S31508008DA811F0004302D5404261EB41015FEA010C2C
S31508008DB802BF84460146002043F0B64308BFA3F124
S31508008DC88053A3F50003BCFA8CF2083AA3EBC25306
S31508008DD810DB01FA02FC634400FA02FCC2F1200225
S31508008DE8BCF1004F20FA02F243EB020008BF20F05C
S31508008DF80100704702F1200201FA02FCC2F12002C2
S31508008E0850EA4C0021FA02F243EB020008BF20EAB6
S31508008E18DC7070474FF0FF0C1CEAD0521EBF1CEAE4
S31508008E28D15392EA0C0F93EA0C0F6FD01A4480EAD2
S31508008E38010C400218BF5FEA41211ED04FF00063BB
S31508008E4843EA501043EA5111A0FB01310CF00040E7
S31508008E58B1F5000F3EBF490041EAD3715B0040EA0D
S31508008E68010062F17F02FD2A1DD8B3F1004F40EBDD
S31508008E78C25008BF20F00100704790F0000F0CF0B0
S31508008E88004C08BF49024CEA502040EA51207F3A74
S31508008E98C2BFD2F1FF0340EAC250704740F400004F
S31508008EA84FF00003013A5DDC12F1190FDCBF00F040
S31508008EB800407047C2F10002410021FA02F1C2F1EE
S31508008EC8200200FA02FC5FEA310040F1000053EA8A
S31508008ED84C0308BF20EADC70704792F0000F00F0D8
S31508008EE8004C02BF400010F4000F013AF9D040EADE
S31508008EF80C0093F0000F01F0004C02BF490011F472
S31508008F08000F013BF9D041EA0C018FE70CEAD1536F
S31508008F1892EA0C0F18BF93EA0C0F0AD030F0004CEF
S31508008F2818BF31F0004CD8D180EA010000F00040A3
S31508008F38704790F0000F17BF90F0004F084691F061
S31508008F48000F91F0004F14D092EA0C0F01D142029B
S31508008F580FD193EA0C0F03D14B0218BF084608D164
S31508008F6880EA010000F0004040F0FE4040F40000AE
S31508008F78704740F0FE4040F4400070474FF0FF0C41
S31508008F881CEAD0521EBF1CEAD15392EA0C0F93EA88
S31508008F980C0F69D0A2EB030280EA010C49024FEADA
S31508008FA8402037D04FF0805343EA111143EA101393
S31508008FB80CF000408B4238BF5B0042F17D024FF44B
S31508008FC8000C8B4224BF5B1A40EA0C00B3EB510F26
S31508008FD824BFA3EB510340EA5C00B3EB910F24BF0F
S31508008FE8A3EB910340EA9C00B3EBD10F24BFA3EB94
S31508008FF8D10340EADC001B0118BF5FEA1C1CE0D15C
S31508009008FD2A3FF650AF8B4240EBC25008BF20F00E
S31508009018010070470CF0004C4CEA50207F32C2BF62
S31508009028D2F1FF0340EAC250704740F400004FF0FF
S315080090380003013A37E792F0000F00F0004C02BF30
S31508009048400010F4000F013AF9D040EA0C0093F0FA
S31508009058000F01F0004C02BF490011F4000F013B54
S31508009068F9D041EA0C0195E70CEAD15392EA0C0FBC
S3150800907808D142027FF47DAF93EA0C0F7FF470AFF4
S31508009088084676E793EA0C0F04D14B023FF44CAF37
S3150800909808466EE730F0004C18BF31F0004CCAD1CC
S315080090A830F000427FF45CAF31F000437FF43CAF08
S315080090B85FE700BF4FF0FF3C06E000BF4FF0010C2A
S315080090C802E000BF4FF0010C4DF804CD4FEA40020C
S315080090D84FEA41037FEA226C18BF7FEA236C11D056
S315080090E801B052EA530C18BF90EA010F58BFB2EB09
S315080090F8030088BFC81738BF6FEAE17018BF40F089
S31508009108010070477FEA226C02D15FEA402C05D13C
S315080091187FEA236CE4D15FEA412CE1D05DF8040BC1
S31508009128704700BF844608466146FFE70FB5FFF754
S31508009138C9FF002848BF10F1000F0FBD4DF808ED0C
S31508009148FFF7F4FF0CBF012000205DF808FB00BFFD
S315080091584DF808EDFFF7EAFF34BF012000205DF857
S3150800916808FB00BF4DF808EDFFF7E0FF94BF0120A4
S3150800917800205DF808FB00BF4DF808EDFFF7D2FFA1
S3150800918894BF012000205DF808FB00BF4DF808EDE4
S31508009198FFF7C8FF34BF012000205DF808FB00BFB1
S315080091A84FEA4002B2F1FE4F0FD34FF09E03B3EBDE
S315080091B812620DD94FEA002343F0004310F0004F1E
S315080091C823FA02F018BF404270474FF00000704774
S315080091D812F1610F01D1420205D110F0004008BF13
S315080091E86FF0004070474FF00000704753B94AB90E
S315080091F8002908BF00281CBF4FF0FF314FF0FF3089
S3150800920800F08CB9ADF1080C6DE904CE00F006F84B
S31508009218DDF804E0DDE9022304B070472DE9F047DC
S31508009228089D8E4604468846002B4AD18A42174628
S3150800923862D9B2FA82F64EB1C6F1200301FA06F8E7
S3150800924820FA03F3B74043EA0808B4404FEA174E32
S31508009258B8FBFEF11FFA87FC0EFB118801FB0CF21E
S31508009268230C43EA08439A4209D9FB1801F1FF304F
S3150800927880F0EB809A4240F2E88002393B449A1A19
S31508009288B2FBFEF00EFB102200FB0CFCA3B243EA6D
S3150800929802439C4509D9FB1800F1FF3280F0D780B4
S315080092A89C4540F2D4803B44023840EA01400021FC
S315080092B8A3EB0C031DB10022F340C5E90032BDE853
S315080092C8F0878B4205D90DB1C5E90001002108468A
S315080092D8F5E7B3FA83F1002946D1734502D38242EA
S315080092E800F20881841A6EEB030201209046002DCD
S315080092F8E5D0C5E90048E2E7002A00F09180B2FA0D
S3150800930882F6002E40F0A5808A1A0121030C4FEA3E
S31508009318174E80B2BCB2B2FBFEFC0EFB1C2243EA17
S31508009328024304FB0CF29A4207D9FB180CF1FF38E2
S3150800933802D29A4200F2E380C4469B1AB3FBFEF2B5
S315080093480EFB123302FB04F440EA03439C4207D996
S31508009358FB1802F1FF3002D29C4200F2CD80024689
S315080093681B1B42EA0C40A5E7C1F120068B4022FAEE
S3150800937806F71F432EFA06FA4FEA1749BAFBF9F811
S315080093880EFA01FE20FA06F309FB18AA1FFA87FC4B
S3150800939843EA0E0300FA01FE08FB0CF01C0C44EA2B
S315080093A80A44A04202FA01F20AD93C1908F1FF3A1E
S315080093B880F09E80A04240F29B80A8F102083C44B7
S315080093C8241A98B2B4FBF9F309FB134403FB0CFC03
S315080093D840EA0444A44509D93C1903F1FF3080F052
S315080093E88580A44540F28280023B3C4443EA084013
S315080093F8A4EB0C04A0FB028C64454346E14664D3FF
S3150800940861D05DB1BEEB030264EB090404FA06F603
S3150800941822FA01F31E43CC40C5E9006400214EE751
S31508009428B1FBF2FC010C41EA0E4180B240EA014266
S315080094383B46B1FBF7F138463C46B846BE462026B9
S31508009448A2EB080241EA0C4165E7014617E7104610
S315080094582BE7C6F120012EFA01FCB7400EFA06FEE4
S3150800946820FA01F141EA0E014FEA174EBCFBFEF855
S31508009478BCB20EFB18CC08FB04F90A0C42EA0C42EB
S31508009488B04091454FEA104380B23ED9BA1808F160
S31508009498FF3C01D291451FD8A2EB0902B2FBFEF99F
S315080094A809FB04F80EFB192A8AB242EA0A4242451F
S315080094B829D2BA1809F1FF31C2D24245C0D2A9F158
S315080094C802013A44BCE7C6459BD2B8EB02036CEBEB
S315080094D8070C0138E14694E7A7EB09094A44B2FBA9
S315080094E8FEF9A8F1020C09FB04F8DBE703467DE759
S315080094F8D04665E70846FAE63B44023A30E7ACF157
S31508009508020C3B4419E749469AE7A2EB0902B2FB63
S31508009518FEF9C44609FB04F8C4E700BF704700BF54
S3150800952880B584B000AF3B1D00221A605A609A6065
S31508009538184B194A1A60174B00229A60154B0022D5
S315080095481A73144B00221A75124B4FF46022DA610B
S31508009558104B00225A600F4B01221A610D4804F07D
S3150800956831FB0346002B01D001F014FB08237B606E
S315080095780123BB600023FB603B1D1946054804F020
S31508009588E5FD0346002B01D001F004FB00BF1037A8
S31508009598BD4680BD5C0200200024014080B58AB023
S315080095A800AF786007F1180300221A605A609A60BB
S315080095B8DA607B681B681F4A934237D11E4B9B6942
S315080095C81D4A43F4007393611B4B9B6903F40073AC
S315080095D87B617B69184B9B69174A43F004039361BF
S315080095E8154B9B6903F004033B613B69124B9B6966
S315080095F8114A43F0080393610F4B9B6903F008036C
S31508009608FB60FB681823BB610323FB6107F118039A
S3150800961819460A4806F01EF90323BB610323FB61B2
S3150800962807F118031946064806F014F900BF283743
S31508009638BD4680BD002401400010024000080140D4
S31508009648000C014080B582B000AF03460A46FB719C
S315080096581346BB71FB79072B50D801A252F823F0A1
S315080096688996000899960008A9960008B9960008E8
S31508009678C9960008D9960008E7960008F7960008DC
S31508009688BB791A464FF48071214806F07EFA36E00F
S31508009698BB791A464FF400711D4806F076FA2EE093
S315080096A8BB791A464FF48061194806F06EFA26E027
S315080096B8BB791A464FF40061154806F066FA1EE0AB
S315080096C8BB791A464FF48051114806F05EFA16E03F
S315080096D8BB791A4608210F4806F057FA0FE0BB79F6
S315080096E81A464FF400410C4806F04FFA07E0BB79D2
S315080096F81A460821094806F048FA00E000BFFB792F
S315080097080749BA79CA5400BF0837BD4680BD00BFA5
S3150800971800180140001001400008014000140140EB
S315080097288C02002080B483B000AF0346FB71FB7936
S31508009738034AD35C18460C37BD4680BC704700BF41
S315080097488C02002080B582B000AF0346FB71FB7916
S31508009758062B3BD801A252F823F000BF81970008D0
S315080097688D97000899970008A5970008B1970008EB
S31508009778BD970008C99700080221174806F0EEF9B0
S31508009788034624E00421144806F0E8F903461EE0D7
S315080097988021124806F0E2F9034618E080211048AD
S315080097A806F0DCF9034612E010210E4806F0D6F951
S315080097B803460CE008210B4806F0D0F9034606E0F4
S315080097C80221064806F0CAF9034600E000231846AF
S315080097D80837BD4680BD00BF000801400018014093
S315080097E800140140000C014080B500AF154804F08C
S315080097F841FE00210020FFF725FF00210120FFF781
S3150800980821FF00210220FFF71DFF00210320FFF793
S3150800981819FF00210420FFF715FF01210520FFF78E
S3150800982811FF01210620FFF70DFF00210720FFF78A
S3150800983809FF054803F0A0FB044803F09DFB00BF99
S3150800984880BD00BF5C02002098020020C0020020EC
S3150800985890B587B000AF78600C4B7B610C4B3B61C9
S3150800986879697868FFF7CCF903461C463969786937
S31508009878FFF7D0FA034619462046FFF77FFB03464B
S31508009888FB60FB6818461C37BD4690BD00007A4445
S315080098983211803B00000000B0B586B000AFF86012
S315080098A8B9607A603B60F868FEF714FE1CA3D3E932
S315080098B80023FEF7A3FF02460B4614461D46B86862
S315080098C8FEF71AFE02460B4620462946FEF76CFEA8
S315080098D802460B4610461946FFF73EF903467B61D2
S315080098E879687869FFF748FC0346002B01D00E4BC8
S315080098F810E079697868FFF783F9034619467869A5
S31508009908FFF73CFB034619463868FFF783FA034610
S315080099183B613B6918461837BD46B0BDAFF30080B2
S315080099280000000000FEAF40000080BF80B588B088
S3150800993800AF0346FB7100F09BF8FB79002B03D0B8
S31508009948082000F053F802E0092000F04FF82248F2
S3150800995804F010FA4FF0FF311F4804F0E5FA1E48E4
S3150800996804F0E8FBF8611C4804F0B2FAFB79002B0E
S3150800997801D0012200E0002213469B001344DB00B5
S31508009988164A1344FA691146184603F01AFBB861D1
S31508009998BB69B3F57A6F03D900F076F8142317E094
S315080099A80F4B7B610F4B3B610F4BFB60FB683A69BA
S315080099B87969B869FFF770FF03461846FFF748FF45
S315080099C8B86000F061F8B868FFF7EAFB03461BB20F
S315080099D818462037BD4680BD5C0200209802002044
S315080099E8333353400000A04000007A4480B586B05F
S315080099F800AF78607B68FB6001233B6103237B61CA
S31508009A0807F10C031946064804F0A0FB0346002B89
S31508009A1801D001F0BFF800BF1837BD4680BD00BFAA
S31508009A285C02002080B483B000AFEFF310833B607C
S31508009A383B687B6072B600BF0C4B1B78DBB2002B09
S31508009A4806D07B68002B01D162B600BF002308E068
S31508009A58064B01221A707B68002B01D162B600BF3B
S31508009A68012318460C37BD4680BC7047940200206F
S31508009A7880B500AF00BFFFF7D5FF0346002BFAD025
S31508009A8800BF00BF80BD000080B483B000AFEFF30D
S31508009A9810833B603B687B6072B600BF064B0022AA
S31508009AA81A707B68002B01D162B600BF00BF0C375D
S31508009AB8BD4680BC704700BF9402002080B500AF41
S31508009AC8174B184A1A60164B08225A60144B00227C
S31508009AD89A60134B0022DA60114B4FF460221A6120
S31508009AE80F4B4FF480125A610D4B00221A760C4B15
S31508009AF801225A760A4B01229A76094B0122DA760E
S31508009B08074B00221A77064B01225A77044804F0B5
S31508009B185FFD0346002B01D001F03CF800BF80BD6D
S31508009B28E80200200064004080B500AF174B184AC9
S31508009B381A60164B10225A60144B00229A60134B6F
S31508009B480022DA60114B4FF460221A610F4B4FF46A
S31508009B5880125A610D4B00221A760C4B01225A764E
S31508009B680A4B01229A76094B0122DA76074B00221C
S31508009B781A77064B01225A77044804F029FD03464A
S31508009B88002B01D001F006F800BF80BD10030020A5
S31508009B980068004080B58EB000AF786007F12003F2
S31508009BA800221A605A609A60DA607B681B68614A04
S31508009BB8934253D1604B1B6801335F4A13605E4B6F
S31508009BC81B68012B0BD15D4BDB695C4A43F00073BC
S31508009BD8D3615A4BDB6903F00073FB61FB69574B8A
S31508009BE89B69564A43F020039361544B9B6903F0DB
S31508009BF82003BB61BB6901233B6200237B62002308
S31508009C08BB6207F1200319464D4805F023FE0223D7
S31508009C183B6202237B620323FB6207F12003194692
S31508009C28474805F017FE474B5B683B633B6B23F4D5
S31508009C38C0433B633B6B43F0E0633B633B6B43F4D6
S31508009C48C0433B633F4A3B6B536000220021142004
S31508009C5805F06BFC142005F084FC67E07B681B683C
S31508009C68394A934262D1354BDB69344A43F08063FB
S31508009C78D361324BDB6903F080637B617B692E4BCA
S31508009C881B6801332C4A13602B4B1B68012B0BD11D
S31508009C982A4BDB69294A43F00073D361274BDB69F2
S31508009CA803F000733B613B69244B9B69234A43F0E5
S31508009CB808039361214B9B6903F00803FB60FB6863
S31508009CC820233B6200237B620023BB6207F1200343
S31508009CD819461E4805F0BEFD40233B6202237B62F7
S31508009CE80323FB6207F120031946184805F0B2FD5D
S31508009CF8144B5B687B637B6B43F0E0637B637B6B2E
S31508009D0843F480037B630F4A7B6B53600022002170
S31508009D183F2005F00AFC3F2005F023FC002200211D
S31508009D28412005F002FC412005F01BFC00BF38372E
S31508009D38BD4680BD0064004038030020001002407C
S31508009D48001401400000014000680040000C014072
S31508009D5880B400AF084B00221A70074B00225A70CD
S31508009D68054B002262F06902DA7300221A7400BFF2
S31508009D78BD4680BC704700BF3C03002080B500AFD5
S31508009D881A4B5A781A4B1B789A4206D0174B5A78A8
S31508009D98174B1A70154B00221A70164B1B7B002B93
S31508009DA803D0124B07225A770EE0124B5B7B002B27
S31508009DB803D00E4B0A225A7706E00C4B9B7F002BE2
S31508009DC802D10A4B00225A77084B5B7F00211846B6
S31508009DD800F078FD0346002B06D0044B5B7F1A4635
S31508009DE80021054809F036FE00BF80BD3C03002067
S31508009DF85C0300208C080020D05C010880B500AF01
S31508009E080F4B5B7F002B03D0022000F01FF816E0EB
S31508009E180C4B1B78002B07D10B4B1B78002B03D058
S31508009E28012000F013F80AE0064B1B78022B06D12E
S31508009E38034B5B7F002B02D1012000F007F880BD99
S31508009E483C0300205B0300202610002080B582B062
S31508009E5800AF0346FB71414B1B78FA799A4203D146
S31508009E683F4AFB79537075E03C4AFB7913703B4BC4
S31508009E781B78002B03D13B49072000F0CBFB374B57
S31508009E881B78012B03D13849072000F0C3FB334B55
S31508009E981B78022B03D13549072000F0BBFB2F4B53
S31508009EA81B78032B03D13249072000F0B3FB2B4B51
S31508009EB81B78042B03D12F49072000F0ABFB274B4F
S31508009EC81B78052B03D12C49072000F0A3FB234B4D
S31508009ED81B78062B03D12949072000F09BFB1F4B4B
S31508009EE81B78072B03D12649072000F093FB1B4B49
S31508009EF81B78082B03D12349072000F08BFB174B47
S31508009F081B78092B03D12049072000F083FB134B44
S31508009F181B780A2B03D11D49072000F07BFB0F4B42
S31508009F281B780B2B03D11A49072000F073FB0B4B40
S31508009F381B780C2B03D11749072000F06BFB074B3E
S31508009F481B780D2B03D11449072000F063FB044A3C
S31508009F58FB7953700837BD4680BD00BF5B030020F8
S31508009F683C030020E45C0108F85C0108105D010860
S31508009F78285D0108405D01085C5D01087C5D0108F3
S31508009F889C5D0108BC5D0108D45D0108EC5D01080B
S31508009F98045E0108205E0108385E010880B584B0B1
S31508009FA800AF78600023FB607868FFF71FFD094853
S31508009FB803F0E0FE0A21074803F0B6FF054804F057
S31508009FC8B9F8F860034803F083FFFB6818461037AA
S31508009FD8BD4680BD5C02002080B485B000AFF8603D
S31508009FE8B9607A60FA68BB689A4205DBFA687B68E2
S31508009FF89A4201DC012300E0002318461437BD46BF
S3150800A00880BC704780B483B000AF7860124B1B7869
S3150800A018002B08D1114A7B6813600F4B01221A706E
S3150800A0280E4B1B6812E00D4B1B687A68D31A26225A
S3150800A03802FB03F3002B00DAFF331B121A46074B01
S3150800A0481B681344054A1360044B1B6818460C37EB
S3150800A058BD4680BC704700BF680300206403002023
S3150800A06880B582B000AF78600B46FB70FB78052B8D
S3150800A0784AD801A252F823F099A00008A7A0000818
S3150800A088BFA00008D7A00008EFA0000805A100088F
S3150800A0987B6842F20F72934238DD00237EE042F66F
S3150800A0A8041241F64C517868FFF796FF0346002BD1
S3150800A0B82ED0012372E041F64C5241F29411786889
S3150800A0C8FFF78AFF0346002B24D0022366E041F2F5
S3150800A0D8941240F2DC517868FFF77EFF0346002B9E
S3150800A0E81AD003235AE040F6C4122E497868FFF7B7
S3150800A0F873FF0346002B11D004234FE07B682A4AD6
S3150800A10893420DDA052349E000BF0AE000BF08E0DC
S3150800A11800BF06E000BF04E000BF02E000BF00E0A1
S3150800A12800BF7B6842F6F722934201DD002335E03B
S3150800A13842F210724FF4FA517868FFF74DFF03465A
S3150800A148002B01D0012329E041F6583241F2883123
S3150800A1587868FFF741FF0346002B01D002231DE06C
S3150800A1684FF47A624FF4FA617868FFF735FF0346C9
S3150800A178002B01D0032311E04FF4FA620B497868E3
S3150800A188FFF72AFF0346002B01D0042306E07B6865
S3150800A198074A934201DA052300E0062318460837DA
S3150800A1A8BD4680BD24FAFFFFFDD6FFFF18FCFFFF5A
S3150800A1B815D3FFFF80B483B000AF0346FB71FB7964
S3150800A1C8052B07D1064B1B780A2B01D8642302E016
S3150800A1D83C2300E00A2318460C37BD4680BC704766
S3150800A1E86903002080B584B000AF0023FB60002314
S3150800A1F8BB6000237B600420FFF7D0FEF860FB688D
S3150800A20840F6E44203FB02F20D4BA3FB0213D21AF3
S3150800A21852081344DB0ABB60BB68A3F2BB634FF45E
S3150800A2287A7202FB03F3074A82FB03129211DB17C1
S3150800A238D31A7B607B6818461037BD4680BD00BFB9
S3150800A248010110007FE0077E80B500AF0E4B1B6842
S3150800A2589F229A620C4B1B6840F2C112DA620A4BBB
S3150800A2681B684FF4E1729A63074B1B6840F2C712E2
S3150800A2785A630421044806F0B3FF0021024806F091
S3150800A28861FE00BF80BD00BF2C10002080B485B0D9
S3150800A29800AF0346FB71FB794FF4E17202FB03F347
S3150800A2A80B4A82FB03125211DB17D31AFB60094AC1
S3150800A2B8FB791370084B1B68FA689A63064B1B6888
S3150800A2C801225A6300BF1437BD4680BC704700BFD9
S3150800A2D81F85EB51690300202C10002080B400AFBD
S3150800A2E8024B1B781846BD4680BC70476903002098
S3150800A2F890B585B000AF224B1B68FB6003F034FCB1
S3150800A308B860204B1B78062B02D01E4B1B7832E010
S3150800A3181D4B1B781946F868FFF7A2FE0346FB7122
S3150800A328194B1B78FA799A4207D1174B1A78174BA3
S3150800A3381A70174ABB6813601BE0144B1B78FA7926
S3150800A3489A4206D0114AFB791370114ABB68136002
S3150800A3580FE00F4B1B68BA68D41A0C4B1B781846C3
S3150800A368FFF728FF03469C4203D3084B1A78064B87
S3150800A3781A70054B1B7818461437BD4690BD00BFA2
S3150800A38864030020040000200500002006000020C1
S3150800A3986C03002080B582B000AF78607B681B68C4
S3150800A3A80E4A934216D17B681B7F012B12D1FFF701
S3150800A3B839FB0346002B0CD0FFF714FF0346084A5F
S3150800A3C81360074B1B681846FFF71CFEFFF75CFB74
S3150800A3D800E000BF0837BD4680BD00BF0004004046
S3150800A3E86003002080B500AF064B074A1A60054887
S3150800A3F805F0D1F80346002B01D000F0CBFB00BFCF
S3150800A40880BD00BF700300200030024080B485B0CC
S3150800A41800AF78607B681B68094A93420BD1094BE1
S3150800A4285B69084A43F040035361064B5B6903F0CE
S3150800A4384003FB60FB6800BF1437BD4680BC704705
S3150800A448003002400010024080B584B000AFF860C2
S3150800A458B9607A607B689BB21946B86800F006F856
S3150800A4687B6818461037BD4680BD000080B485B0A5
S3150800A47800AF78600B467B8072B600BF0023FB816D
S3150800A48845E0284BB3F804349BB2B3F5806F18D36C
S3150800A498244BB3F802349BB201335A42C3F3090377
S3150800A4A8C2F3090258BF53429AB21E4BA3F80224B4
S3150800A4B81C4BB3F804349BB2013B9AB2194BA3F868
S3150800A4C80424FB897A681344164AB2F8002492B21F
S3150800A4D81978144B9954134BB3F800349BB20133CB
S3150800A4E85A42C3F30903C2F3090258BF53429AB240
S3150800A4F80C4BA3F800240B4BB3F804349BB2013376
S3150800A5089AB2084BA3F80424FB890133FB81FA891C
S3150800A5187B889A42B5D362B600BF00BF1437BD46DA
S3150800A52880BC70477803002080B483B000AF72B649
S3150800A53800BF064BB3F80434FB8062B600BFFB883D
S3150800A54818460C37BD4680BC704700BF7803002004
S3150800A55880B582B000AF72B600BF2D4BB3F804348D
S3150800A5689BB2002B02D162B600BF4EE0284BB3F867
S3150800A5780434FB80FB88802B01D98023FB80244B7D
S3150800A588B3F802349BB2C3F58063BB80FA88BB88EC
S3150800A5989A4201D9BB88FB801D4BB3F804349BB299
S3150800A5A8FA889A420CD11A4BB3F802349BB21A4667
S3150800A5B8174B1344F9885022184602F0EFF90BE0B6
S3150800A5C8134BB3F802349BB21A46114B1344F98855
S3150800A5D85122184602F0E2F90D4BB3F802349AB242
S3150800A5E8FB8813449BB2C3F309039AB2084BA3F832
S3150800A5F80224074BB3F804349AB2FB88D31A9AB2E2
S3150800A608034BA3F8042462B600BF0837BD4680BDCD
S3150800A618780300200EB480B585B000AF0346FB71F9
S3150800A628154AFB79137007F12003BB60BB68FA6902
S3150800A6387E21124809F0E2F9F860FB68002B01DA76
S3150800A648FB6812E0FB687D2B01DD7E23FB60FB6857
S3150800A6580133094A0021D154FB689BB202339BB2E5
S3150800A66819460548FFF702FFFB6818461437BD4622
S3150800A678BDE8804003B070478007002081070020A6
S3150800A68880B58AB000AF07F1140300221A605A6031
S3150800A6989A60DA607D4B9B697C4A43F010039361A4
S3150800A6A87A4B9B6903F010033B613B69774B9B69BF
S3150800A6B8764A43F004039361744B9B6903F00403D9
S3150800A6C8FB60FB68714B9B69704A43F0080393610A
S3150800A6D86E4B9B6903F00803BB60BB686B4B9B69B1
S3150800A6E86A4A43F040039361684B9B6903F0400349
S3150800A6F87B607B68654B9B69644A43F020039361DA
S3150800A708624B9B6903F020033B603B6800223821B3
S3150800A7185F4805F03AFA00224FF4F8515D4805F00B
S3150800A72834FA00224FF400415B4805F02EFA00225D
S3150800A73818215A4805F029FA00228021584805F0B8
S3150800A74824FA38237B610123BB610023FB610223BA
S3150800A7583B6207F1140319464D4805F07BF80223B6
S3150800A7687B610023BB610023FB6107F114031946CB
S3150800A778494805F06FF804237B610023BB6102236F
S3150800A788FB6107F114031946434805F063F844F2D8
S3150800A79882037B610023BB610023FB6107F1140375
S3150800A7A819463C4805F056F84FF4F8537B610123DF
S3150800A7B8BB610023FB6102233B6207F114031946B8
S3150800A7C8344805F047F84FF400437B610123BB6121
S3150800A7D80023FB6102233B6207F1140319462E483E
S3150800A7E805F038F818237B610123BB610023FB6158
S3150800A7F802233B6207F114031946284805F02AF88C
S3150800A80880237B610023BB610023FB6107F11403E6
S3150800A8181946224805F01EF818237B610023BB61F8
S3150800A8280023FB6107F1140319461D4805F012F8C1
S3150800A83880237B610123BB610023FB6102233B6202
S3150800A84807F114031946164805F004F84FF440733F
S3150800A8587B611223BB6103233B6207F11403194684
S3150800A8680F4804F0F7FF0F4B5B687B627B6A43F07F
S3150800A878E0637B627B6A43F002037B62094A7B6A70
S3150800A888536000BF2837BD4680BD00BF0010024090
S3150800A898001001400018014000080140001401405A
S3150800A8A8000C01400000014080B400AF034B044A85
S3150800A8B89A6000BFBD4680BC704700BF00ED00E047
S3150800A8C80080000880B485B000AF03460A46FB71CD
S3150800A8D81346BB71BB791F2B01D900230EE0002351
S3150800A8E8FB73BB79084AD35CFA799A4201D00123EB
S3150800A8F8FB73BB790449FA79CA54FB7B18461437A3
S3150800A908BD4680BC704700BF0008002080B584B0EB
S3150800A91800AF786003F028F9B8607B68FB60FB68CD
S3150800A928B3F1FF3F0ED00E4B1B781A46FB6813444B
S3150800A938FB6007E001F036F9FFF760FA01F01EF848
S3150800A94801F0B2FE03F010F90246BB68D31AFA689A
S3150800A9589A42EFD800BF00BF1037BD4680BD00BF7A
S3150800A9687400002080B500AF0320FEF7EBFE03460F
S3150800A978002B02D1024B01221A7000BF80BD00BF0E
S3150800A9883C03002080B500AF0B4804F041F8FFF7F8
S3150800A99895F8094803F0F8FF0346002B01D000F0A4
S3150800A9A8F9F80221044804F0A0FA0346002B01D05E
S3150800A9B800F0F0F800BF80BDE802002080B582B03C
S3150800A9C802AFFFF771FF03F077F805F003F900F017
S3150800A9D871F8FFF755FEFEF7A3FDFFF76FF8FFF7C7
S3150800A9E8A3F801F069F802F023FD02F0A1FEFFF7CB
S3150800A9F8F9FC02F049FE02F071FE02F0C3FE02F00D
S3150800AA08A1FCFEF7F1FE00F099FF4FF4967003F0EB
S3150800AA18B5F801F0D9FA01F033FE21490720FFF706
S3150800AA28F9FD01F009FE1F4B1B889BB21A461E4901
S3150800AA380720FFF7EFFD1B4B9B781A461B49072093
S3150800AA48FFF7E8FD174B9B889BB21A46154BDB8820
S3150800AA589BB21946134B1B899BB200930B461449A4
S3150800AA680720FFF7D7FDFFF78DFF00F07DFAFFF700
S3150800AA786FF900F087FB00F033FC0A20FFF746FF62
S3150800AA8800F08EF8FFF77AF900F01EFE0A20FFF7A5
S3150800AA983DFFFFF767FF3220FFF738FF00BFE8E7FB
S3150800AAA8845E01081C100020985E0108AC5E010847
S3150800AAB8C05E010880B59CB000AF07F1380338229C
S3150800AAC80021184608F0D8FF07F1240300221A6067
S3150800AAD85A609A60DA601A613B1D202200211846DE
S3150800AAE808F0CAFF0523BB634FF480333B6404238D
S3150800AAF87B640123BB640123FB644FF48033FB6347
S3150800AB080223BB654FF48033FB654FF4E0133B66BD
S3150800AB1802237B664FF4C063BB664023FB6607F1D6
S3150800AB283803184605F026F90346002B01D000F02D
S3150800AB3831F80F237B620223BB620023FB624FF4C2
S3150800AB4880633B6300237B6307F1240302211846CD
S3150800AB5805F026FC0346002B01D000F01BF803235A
S3150800AB687B604FF48073BB604FF40043FB603B1D6A
S3150800AB78184605F00BFE0346002B01D000F00AF82C
S3150800AB88034B01221A6000BF7037BD4680BD00BF5F
S3150800AB987000424280B400AF72B600BF00BFFDE73E
S3150800ABA82DE9B04384B000AF2E4B00221A712E4B04
S3150800ABB85B78082B04D12B4B012283F8242003E069
S3150800ABC8284B002283F8242002F0CEFFF860254B94
S3150800ABD89B68FA68D31ABB60224AFB689360224BC3
S3150800ABE8D3F80330BA6802FB03F3204AA2FB03230F
S3150800ABF89B097B601B4BD3E90423796800200C4624
S3150800AC08054612EB040843EB0509164BC3E9048904
S3150800AC18144BD3E90423164BA3FB0223DB0A114A78
S3150800AC289361104B93F82430002B08D00D4B9A6982
S3150800AC380C4BDB69D31A0C4AC2F807300CE00A4BEE
S3150800AC480022DA7100221A7200225A7200229A72B7
S3150800AC58044B9B69034AD36100BF1037BD46BDE85C
S3150800AC68B08300BF200800203C030020D34D6210A3
S3150800AC78C5B3A29180B582B000AF0346FB71064AF8
S3150800AC88FB79D37102F070FF0346034A136100BFCC
S3150800AC980837BD4680BD00BF8C08002080B500AFC8
S3150800ACA802F062FF0246024B1B69D31A184680BD9A
S3150800ACB88C08002080B584B000AF7860884B894A34
S3150800ACC80121786803F0F0FF0346002B40F0048161
S3150800ACD8844B5B68BB603B7A002B40F0FC8002F033
S3150800ACE843FF0346804A1360BB7A03F03F03DBB28F
S3150800ACF8022B05D17D4B7A4A92E8030083E80300C4
S3150800AD08BB7A03F03F03DBB2042B19D1784B744A9C
S3150800AD1892E8030083E80300754B1B791A46754BBE
S3150800AD28DA61734B1A7A734B83F82020704BDA79F9
S3150800AD38704B83F821206E4B9A796E4B83F8222044
S3150800AD48BB7A03F03F03DBB2062B23D16A4B644A6E
S3150800AD5892E8030083E80300674B5B781A46664B5C
S3150800AD681B781B0213441A46634B9A60624BDB78BE
S3150800AD781A46614B9B781B0213441A465E4BDA60E7
S3150800AD885D4B5B791A465C4B1B791B0213441A46C2
S3150800AD98594B1A61BB7A03F03F03DBB2082B05D17E
S3150800ADA8564B4F4A92E8030083E80300BB7A03F040
S3150800ADB83F03DBB2092B40F08F80514B484A92E893
S3150800ADC8030083E803004E4BDB791A464C4BDA60DE
S3150800ADD84B4BDA684A4B9B791B021343484AD360A4
S3150800ADE8474BDA68464B5B791B041343444AD360DE
S3150800ADF8434BDA68424B1B791B061343404AD36018
S3150800AE083F4BDB781A463E4B9A603D4B9A683C4B5B
S3150800AE189B781B0213433A4A9360394B9A68384B16
S3150800AE285B781B041343364A9360354B9A68344B50
S3150800AE381B781B061343324A9360314B9B68314A89
S3150800AE48A2FB03239B09FB812D4BDB682E4AA2FB39
S3150800AE5803235B09BB81274AFB895380254ABB899B
S3150800AE689380FB89132B8CBF01230023DBB21A4678
S3150800AE78204B9A721F4B01221A721D4B1A791D4BC9
S3150800AE889A711C4BDB79012B26D91A4B5A881F4B0A
S3150800AE98A3F81320174BB3F904309AB21B4BA3F83F
S3150800AEA815201A4BB3F815309BB21A46174BB3F848
S3150800AEB813309BB202FB03F3154A82FB0312921066
S3150800AEC8DB17D31A1A46114BC3F80320094B9A7A8B
S3150800AED80E4B1A7600E000BF1037BD4680BD00BF8E
S3150800AEE8D0080020B4080020B00800204808002030
S3150800AEF8540800208C0800206008002074080020E8
S3150800AF087C080020D34D62101F85EB513C030020B6
S3150800AF186766666680B58AB000AF0E237B61002334
S3150800AF28BB610123FB6100233B6000237B60002390
S3150800AF38BB600023FB6000233B6101233B620123BE
S3150800AF483B610E237B623B461946064803F03CFCE8
S3150800AF580346002B01D0FFF71DFE00BF2837BD4664
S3150800AF6880BD00BF1003002080B500AF134803F06A
S3150800AF784FFDFEF7D9FDFFF7CDFF104803F004FD96
S3150800AF8810210E4803F0B1FF242200210C4808F0CE
S3150800AF9873FD0B4B0022DA7102F0E6FD0346084AF8
S3150800AFA81361074B47F230525A61054B00221A764D
S3150800AFB80021002000F006F800BF80BD100300201D
S3150800AFC88C08002080B584B000AF03460A46FB719A
S3150800AFD81346BB7107F1080308220021184608F032
S3150800AFE84BFDFB79002B15D10D4B1B7A002B13D083
S3150800AFF8BB79002B0CBF01230023DBB23B72F9791E
S3150800B00807F108031A22F02000F066F81420FFF763
S3150800B0187DFC02E000BF00E000BF1037BD4680BDDA
S3150800B0288C08002080B586B000AF0346FB710B4636
S3150800B038BB8013467B8007F10803082200211846BF
S3150800B04808F01AFDFB79002B40D1BB88952B01D84F
S3150800B0589623BB801F4B1B7E002B06D1BB88B3F5F6
S3150800B068FA7F02D340F2F313BB807B88642202FB83
S3150800B07803F37B61BB884FF47A7202FB03F33B61E7
S3150800B0887B691B0EDBB23B737B691B0CDBB27B73DC
S3150800B0987B691B0ADBB2BB737B69DBB2FB733B6953
S3150800B0A81B0EDBB23B723B691B0CDBB27B723B693E
S3150800B0B81B0ADBB2BB723B69DBB2FB72F97907F193
S3150800B0C808031C22F02000F007F800E000BF183734
S3150800B0D8BD4680BD8C08002080B58CB000AF3B60AB
S3150800B0E80346FB710B46BB7113467B71FB7987F8E0
S3150800B0F82830BB7987F829307B7903F03F03DAB221
S3150800B10897F82A3062F3050387F82A307B8D0A22D6
S3150800B11862F389137B850A2387F82F30BB6A7B611C
S3150800B1280023FB610423BB6108233B621EE0144825
S3150800B13803F086FD0346002B0ED007F10C0307F132
S3150800B14810013A680E4803F0ACFC034687F82E301F
S3150800B15897F82E30002B0ED00120FFF7D7FB97F96A
S3150800B1682F30DBB2013BDBB287F82F3097F92F3047
S3150800B178002BDCDC00E000BF3037BD4680BD00BFD1
S3150800B1881003002080B582B000AF3B4600221A6043
S3150800B1985A603B4604220021F020FFF79DFF142041
S3150800B1A8FFF7B4FB3B4606220021F020FFF794FF81
S3150800B1B81420FFF7ABFB3B4609220021F020FFF7D6
S3150800B1C88BFF1420FFF7A2FB414BB3F81B309BB249
S3150800B1D8404AA2FB0323DB089BB21A463C4BB3F84A
S3150800B1E813309BB202FB03F31A463B4B5B699A4240
S3150800B1F811D9394B5A6913469B0013445B001A4602
S3150800B208334BB3F813309BB2B2FBF3F39AB2304B15
S3150800B218A3F8112006E02E4BB3F81B309AB22C4B34
S3150800B228A3F811202A4BB3F811309BB240F23252D8
S3150800B238934208D9264B002242F032025A74002259
S3150800B24842F005029A74224BB3F811309BB21A469B
S3150800B2581F4BB3F80F309BB202FB03F31F4A82FB5E
S3150800B26803129210DB17D31A1A46194BC3F80B2088
S3150800B278194B5B7A002B26D0154BB3F80F309BB2C7
S3150800B288B3F5FA7F06D10A224FF496710020FFF724
S3150800B298C9FE0BE00E4BB3F80F309BB20C4AB2F856
S3150800B2A8112092B219460020FFF7BCFE1420FFF7BA
S3150800B2B82DFB074BB3F813309BB2B3F5F57F02D9CC
S3150800B2C8054B01221A7600BF0837BD4680BD00BF68
S3150800B2D83C030020CDCCCCCC8C080020676666667B
S3150800B2E898B500AF02F040FC0246B44B1B68D31A67
S3150800B2F8B3F5FA7F20D9B24B00221A72B04B002256
S3150800B3089A72B04B00221A71AE4B00221A72AD4BD4
S3150800B3180022DA71AB4B00229A71AB4B00229A6075
S3150800B328A94B0022DA60A84B00221A61A74B002213
S3150800B338DA60A64B00229A60A14B1B7A002B03D031
S3150800B3489F4B1B78002B0CD1A14B0022DA740022E4
S3150800B3581A759F4B00225A7500229A759C4B002233
S3150800B3681A769B4B9B7F002B0CD001210420FEF7F5
S3150800B37869F902F0F9FB0346964A1360904B0122D5
S3150800B3881A7010E002F0F0FB0246924B1B68D31ABB
S3150800B3984EF66022934206D900210420FEF752F998
S3150800B3A8874B00221A700520FEF7CCF903461A4681
S3150800B3B8834BDA72824B1B7A002B07D0804B1B7B98
S3150800B3C8002B03D17E4B1B78002B02D17C4B002225
S3150800B3D85A727B4BDB79092B00F2558101A252F888
S3150800B3E823F000BF15B4000849B4000865B400087E
S3150800B3F89DB40008EBB400082DB5000897B50008F9
S3150800B40841B60008F1B500087BB600086C4B002267
S3150800B4185A7000210320FEF715F9694B1B7A002B91
S3150800B42800F03581664B1B78002B00F03081644BA1
S3150800B4381B7B002B40F02B810120FFF71BFC26E124
S3150800B448FFF72CFC0346B3F57A6F40F222815C4B72
S3150800B45801225A720220FFF70DFC1AE1584B002206
S3150800B4681A7600210320FEF7EDF8554B5B7A002B78
S3150800B47803D10020FFF7FEFB1CE1554BDB7D002BB3
S3150800B48800F0098101210020FFF79CFD0320FFF742
S3150800B498F1FB00E14A4B9B7A002B0CD0484B5B7AB0
S3150800B4A8002B08D002F060FB03464B4A13600420C1
S3150800B4B8FFF7E0FBF1E0FFF7F1FB034642F21072F3
S3150800B4C8934240F2EA803E4B01225A73404B0A22C5
S3150800B4D85A770020FFF7CEFB40490420FFF79AF871
S3150800B4E8DBE001210320FEF7ADF8354BDB7A002BAC
S3150800B4F803D00520FFF7BEFBD1E0FFF7CFFB0346D5
S3150800B508B3F57A7F40F2CB802D4B01221A73304B64
S3150800B51807225A770620FFF7ADFB31490420FFF7C3
S3150800B52879F8BCE02A4BDB7D002B03D0244B5B7AE9
S3150800B538002B03D10620FFF79DFBBBE00520FEF78D
S3150800B54801F903461C460320FEF7ECF803469C421D
S3150800B55817D002F009FB0246224B1B68D31AB3F52B
S3150800B5687A7F40F29E801A4B07225A77144B01229B
S3150800B5781A730620FFF77EFB19490420FFF74AF8D5
S3150800B5888FE002F0F1FA0346164A136089E0104B79
S3150800B59800225A7400229A740D4BB3F815309BB2E0
S3150800B5A81D2B06D9FFF77AFB034641F288329342E8
S3150800B5B879D90820FFF75EFB75E000BFB0080020C0
S3150800B5C88C08002054080020600800207C08002009
S3150800B5D83C030020D8080020DC080020D85E0108B3
S3150800B5E8E85E0108E008002000210320FEF72AF893
S3150800B5F8314BDB7A002B07D100210020FFF7E2FC4C
S3150800B6080720FFF737FB50E0FFF748FB0346B3F57B
S3150800B6187A7F4AD9284B01221A73284B07225A7768
S3150800B62800210020FFF7CEFC0720FFF723FB24495B
S3150800B6380420FEF7EFFF38E01F4B9B7A002B03D157
S3150800B6480920FFF717FB32E0FFF728FB034642F20B
S3150800B658107293422BD9184B01225A73174B0A2298
S3150800B6685A770020FFF706FB16490420FEF7D2FF93
S3150800B6781DE0FFF713FB0346B3F57A6F19D90220C5
S3150800B688FFF7F8FA15E00020FFF7F4FA12E000BF12
S3150800B69810E000BF0EE000BF0CE000BF0AE000BFE4
S3150800B6A808E000BF06E000BF04E000BF02E000BFF4
S3150800B6B800E000BF00BF98BD8C0800203C030020AE
S3150800B6C8E85E0108085F010880B500AF344B5B7F68
S3150800B6D8002B03D0334800F01FF95FE0304B5B7846
S3150800B6E80D2B57D801A252F823F000BF2DB7000832
S3150800B6F835B700083DB7000845B700084DB7000834
S3150800B70855B700085DB7000865B700086DB70008A3
S3150800B71875B700087DB7000885B700088DB7000813
S3150800B72895B70008204800F0F7F837E01F4800F0FA
S3150800B738F3F833E01B4800F0EFF82FE01C4800F058
S3150800B748EBF82BE01A4800F0E7F827E0194800F06C
S3150800B758E3F823E0174800F0DFF81FE0154800F083
S3150800B768DBF81BE0134800F0D7F817E0124800F09A
S3150800B778D3F813E0104800F0CFF80FE00E4800F0B1
S3150800B788CBF80BE00C4800F0C7F807E0084800F0CB
S3150800B798C3F803E0044800F0BFF800BF80BD00BF47
S3150800B7A83C03002044000020080000201400002064
S3150800B7B8200000202C0000203800002080B487B024
S3150800B7C800AFF860B96011461A460B46FB80134667
S3150800B7D8BB80FA88BB889A4201D9BB88FB80BB889C
S3150800B7E8002B01D10123BB80FA8813461B029A1A3B
S3150800B7F8BB8892FBF3F3FB82FB681B781A46FB8A25
S3150800B808C3F1FF0303FB02F2BB681B781946FB8AE0
S3150800B81801FB03F31344204A82FB03121A44D2118C
S3150800B828DB17D31ADAB23B6A1A70FB685B781A46D2
S3150800B838FB8AC3F1FF0303FB02F2BB685B78194670
S3150800B848FB8A01FB03F31344134A82FB03121A44C7
S3150800B858D211DB17D31ADAB23B6A5A70FB689B789F
S3150800B8681A46FB8AC3F1FF0303FB02F2BB689B78FF
S3150800B8781946FB8A01FB03F31344074A82FB0312A2
S3150800B8881A44D211DB17D31ADAB23B6A9A7000BF88
S3150800B8981C37BD4680BC70478180808080B483B0E1
S3150800B8A800AF78607B681B781A46642302FB03F3AB
S3150800B8B8174A82FB03121A44D211DB17D21A154B00
S3150800B8C81B689A637B685B781A46642302FB03F352
S3150800B8D80F4A82FB03121A44D211DB17D21A0D4BF0
S3150800B8E81B68DA637B689B781A46642302FB03F3B2
S3150800B8F8074A82FB03121A44D211DB17D21A054BE0
S3150800B9081B681A6400BF0C37BD4680BC704700BF69
S3150800B918818080807410002080B483B000AF78607E
S3150800B928054B7A681068516803C312891A8000BFE4
S3150800B9380C37BD4680BC7047EC08002080B582B03D
S3150800B94800AF00233B7100237B710023BB710421E0
S3150800B958094805F045FC0821074805F041FC0C2173
S3150800B968054805F03DFC3B1D1846FFF797FF00BF45
S3150800B9780837BD4680BD00BF7410002080B582B068
S3150800B98802AF02F0F1F80246464B1B68D31A142B8D
S3150800B99840F2858002F0E8F80346424A1360424BB3
S3150800B9A85B8801339AB2404B5A803F4B1B78032B6E
S3150800B9B867D801A252F823F0D1B9000803BA0008DB
S3150800B9C82FBA000861BA0008374B5A88374BDB7814
S3150800B9D81946374B00930B4634493648FFF7EEFEAF
S3150800B9E8314B5B88314AD27893424ED92E4B012285
S3150800B9F81A702D4B00225A8047E02B4B2B4A0433EA
S3150800BA081268114619800233120C1A70264B5B8885
S3150800BA18264A127993423AD9234B02221A70224BA4
S3150800BA2800225A8033E0204B5A88204B5B79194606
S3150800BA381F4B00930B461F491C48FFF7BFFE1A4BBE
S3150800BA485B881A4A5279934223D9174B03221A70EC
S3150800BA58154B00225A801CE0134B144A043307324C
S3150800BA681188927819809A700F4B5B880F4A9279D9
S3150800BA78934210D90C4B00221A700B4B00225A809D
S3150800BA8809E0094B00221A7006E000BF04E000BF6F
S3150800BA9802E000BF00E000BF0548FFF7FFFE00BF51
S3150800BAA8BD4680BDF8080020E4080020EC08002000
S3150800BAB8E8080020F308002080B500AF0A4B0B4AB7
S3150800BAC81A60094B4FF0FF325A60074B4FF48072E1
S3150800BAD89A60054805F0DEF80346002B01D0FFF703
S3150800BAE859F800BF80BD00BFFC08002000280040A8
S3150800BAF880B584B000AF78607B681B680B4A9342B0
S3150800BB0810D104F05BF80A4BDB69094A43F0006375
S3150800BB18D361074BDB6903F00063FB60FB68054BE1
S3150800BB2801221A6000BF1037BD4680BD00280040B4
S3150800BB38001002403C04424280B400AFBFF34F8F66
S3150800BB4800BF064BDB6803F4E0620449044B134361
S3150800BB58CB60BFF34F8F00BF00BFFDE700ED00E0E5
S3150800BB680400FA0580B582B000AF78600B467B8082
S3150800BB787B680A4A93420CD17B88002B0AD07B88BB
S3150800BB88B3F5807F06D87B881946054800F0E4FC9B
S3150800BB9800E000BF0837BD4680BD00BF94110020ED
S3150800BBA83409002080B500AFA74806F0C2FE034650
S3150800BBB8202B05D14FF48072A449A34806F09AFAB7
S3150800BBC8FEF796FB03461A46A14B1A70A14B1B783B
S3150800BBD8002B03D09F4B1A789F4B1A7001F0C4FFAD
S3150800BBE802469E4B1B68D31A0A2B53D901F0BCFF91
S3150800BBF802469B4B1B68D31AC72B06D900F01AFBBB
S3150800BC0801F0B2FF0346964A1360964B1B78002B41
S3150800BC1808D095490420FEF7FDFC00F0ACFA914BD4
S3150800BC2800221A708B4B1B78012B03D0894B5B7F3C
S3150800BC38002B13D001F098FF02468C4B1B68D31AC9
S3150800BC48B3F57A7F0AD901F08FFF0346874A13604E
S3150800BC5887490520FEF7DEFC00F08DFA854B1B7830
S3150800BC680C2B03D0834B1B780B2B13D101F07CFFCD
S3150800BC7802467E4B1B68D31AB3F57A7F0AD901F0B8
S3150800BC8873FF0346794A13607B490520FEF7C2FC11
S3150800BC9800F071FA794B1B78002B07D10121052092
S3150800BCA8FDF7D0FC0020FEF7D1F8FCE0744B1B78B2
S3150800BCB8042B00F2F88001A252F823F0D9BC000838
S3150800BCC8F9BC00083DBD000879BD0008C9BD0008D3
S3150800BCD800210520FDF7B6FC0220FEF7B7F85D4BF4
S3150800BCE85B7F002B40F0A780654B01221A70A2E003
S3150800BCF801210520FDF7A6FC0120FEF7A7F8544BFD
S3150800BD081B78012B03D0524B1B78022B02D15C4BB4
S3150800BD1802221A704F4B5B7F002B00F08E804D4B2A
S3150800BD285B7F1A4657490420FEF774FC544B0022D9
S3150800BD381A7082E001210520FDF784FC0420FEF72D
S3150800BD4885F8444B1B78022B06D14F490720FEF786
S3150800BD5861FC4B4B03221A703D4B1B78002B6ED1A6
S3150800BD684A490720FEF756FC454B01221A7066E039
S3150800BD7801210520FDF766FC3E4B1B78022B03D8EC
S3150800BD880320FEF763F804E03A4B1B781846FEF7DB
S3150800BD985DF82F4B1B78002B06D13C490720FEF788
S3150800BDA839FC374B01221A70394B1B78002B48D0BF
S3150800BDB838490720FEF72EFC314B04221A7040E05A
S3150800BDC800210520FDF73EFC0D20FEF73FF801F09F
S3150800BDD8CBFE0246304B1B68D31AB3F57A7F1AD9BD
S3150800BDE801F0C2FE03462C4A1360294B1B78002B28
S3150800BDF80AD0274B1B78FF2B0DD0254B1B78013B08
S3150800BE08DAB2234B1A7006E024490720FEF702FC2B
S3150800BE181B4B01221A701E4B1B78002B42D10C4B68
S3150800BE281B78012B3ED11E490720FEF7F3FB144B5E
S3150800BE3802221A7036E000BF35E000BF33E000BFC3
S3150800BE4831E000BF2FE000BF94110020340900201C
S3150800BE584F0000203C030020300900202809002054
S3150800BE68940B0020340B00201C5F01082C090020C5
S3150800BE78305F0108900B0020485F01082610002053
S3150800BE8850000020645F01088C5F0108B05F010854
S3150800BE98350B0020C05F0108980B0020D05F010809
S3150800BEA8F85F010800BF3F4B1B78002B1FD03E4B9D
S3150800BEB81B68002B08D001F057FE02463A4B1B6850
S3150800BEC8D31AB3F5FA6F08D338490420FEF7A2FB4C
S3150800BED801F04AFE0346344A1360354B0022DA75E8
S3150800BEE8344B00221A706420FEF7D0F944E0324B2E
S3150800BEF81B68002B23D001F037FE02462E4B1B6821
S3150800BF08D31AB3F5FA6F1AD928490420FEF782FB23
S3150800BF18244B01221A7001F027FE0346264A1360AD
S3150800BF2801F022FE0346204A1360214B0022DA75E7
S3150800BF38204B00221A706420FEF7A8F91CE01F4B54
S3150800BF481B78012B03D11A4B0022DA7514E01C4B17
S3150800BF581B78002B14BF01230023DBB21A46144BA7
S3150800BF68DA75134BDB7D002B06D1114B5B78032B57
S3150800BF7802D10F4B0022DA75124B1B78012B07D01A
S3150800BF88104B1B78022B03D00E4B1B78032B03D1BF
S3150800BF98074B01229A7703E0054B00229A7700BFE0
S3150800BFA800BF80BD3C0B0020400B00203460010810
S3150800BFB83C030020900B0020380B00203009002095
S3150800BFC8310900204F00002080B500AFFEF73CF984
S3150800BFD86420FEF75BF90D4B4FF47A721A800B4B07
S3150800BFE896225A80094B40F232529A80074B0A2207
S3150800BFF8DA80064B47F230529A6000F0B3F80449E3
S3150800C0080720FEF707FB00BF80BD00BF1009002008
S3150800C0184860010880B485B000AF78600B467B801D
S3150800C0284FF6FF73FB810023BB8122E0BB897A6840
S3150800C03813441B781A46FB895340FB810023FB727D
S3150800C04811E0FB8903F00103002B06D0FB895B0886
S3150800C0589AB20D4B5340FB8102E0FB895B08FB81D2
S3150800C068FB7A0133FB72FB7A072BEAD9BB890133C2
S3150800C078BB81BA897B889A42D8D3FB891846143774
S3150800C088BD4680BC704700BF01A0FFFF80B586B0DB
S3150800C09800AFB9607B600346FB731346BB81BB8957
S3150800C0A80333FB82FA8A3B8C9A4201D9002329E09A
S3150800C0B87B68FA7B1A70BB89002B09D0BB68002BF2
S3150800C0C806D07B680133BA89B968184607F01CFD9B
S3150800C0D8BB8901339BB219467868FFF79BFF03466D
S3150800C0E8BB82BB8901337A681344BA8AD2B21A70FA
S3150800C0F8BB8A1B0A99B2BB8902337A681344CAB247
S3150800C1081A70FB8A18461837BD4680BD80B586B0B2
S3150800C11802AF03463960FB711346BB80BA88F879C3
S3150800C1284FF4807300930C4B3968FFF7AFFF03464B
S3150800C138FB81FB89002B06D0FA894FF47A730649E6
S3150800C148064805F017FF01F00FFD0346044A136079
S3150800C15800BF1037BD4680BD340A00209411002060
S3150800C1682809002080B500AF002200215220FFF7D9
S3150800C178CDFF00BF80BD80B500AF00220021532047
S3150800C188FFF7C4FF00BF80BD80B582B000AF01F0DD
S3150800C198EBFC78601E4B1B687A68D31A3B601C4A0E
S3150800C1A87B6813601B4BB3F813309BB21A46194BBE
S3150800C1B8B3F815309BB202FB03F3174A82FB031246
S3150800C1C89210DB17D31A1A46144B1A60134B1B68BE
S3150800C1D83A6802FB03F3124AA2FB03239A09114B96
S3150800C1E81B6813440F4A13600F4B1B78012B02D1A7
S3150800C1F80C4B00221A600B4B1B680C4AA2FB032344
S3150800C208DB0A0B4A136000BF0837BD4680BD00BF6E
S3150800C2189C0B00203C030020676666661C09002004
S3150800C228D34D621020090020900B0020C5B3A291B7
S3150800C2382409002080B500AFFFF7A6FFFEF74EF8E1
S3150800C24803461A46304B1A70304BDA7A2E4B5A7018
S3150800C2582F4BB3F813309AB22B4B5A802C4BB3F8A2
S3150800C2680F309BB2B3F5FA7F03D1274B4FF4FA7216
S3150800C2785A80274BB3F815309AB2234B9A80254B28
S3150800C2881B68214AC2F80630234B1B681E4AC2F8A7
S3150800C2980A30224B1B78032B04D1214B1A781A4BE8
S3150800C2A8DA7402E0184B0022DA741E4B1A88164B09
S3150800C2B89A821C4B5A88144BDA821A4B9A88124B64
S3150800C2C81A83184BDA88104B5A83164B9B680E4A02
S3150800C2D8D361154B1A780C4B9A740B4A002343F012
S3150800C2E87F4343F47F0343F43B4343F0A003D381DE
S3150800C2F8002343F00D031382202203495020FFF739
S3150800C30805FF00BF80BD00BF440B00208C08002035
S3150800C3183C0300201C0900202409002050000020A6
S3150800C3284F00002010090020370B002080B483B086
S3150800C33800AF0346FB71FB79403B092B2AD801A2BB
S3150800C34852F823F075C3000879C300087DC30008AE
S3150800C35881C3000885C3000889C300088DC300087F
S3150800C36891C3000895C3000899C30008012313E080
S3150800C378012311E001230FE001230DE001230BE05F
S3150800C388042309E0012307E02C2305E0012303E041
S3150800C398002301E04FF6FF7318460C37BD4680BCEC
S3150800C3A8704700BFF0B58BB000AF03463960FB7124
S3150800C3B81346BB8001F0D8FB03465B4A13605B4B08
S3150800C3C800221A705A4B00221A60FB79403B092B47
S3150800C3D800F2A38001A252F823F000BF0DC400089A
S3150800C3E83BC4000855C4000877C400080BC50008F4
S3150800C3F891C40008AFC40008BDC4000801C50008F8
S3150800C40817C500083B68FB60FB681B7887F8273068
S3150800C41897F82730642B02D9642387F82730454ACA
S3150800C42897F82730137097F827301846FDF72EFF28
S3150800C43876E03B683B613B691B78002B14BF0123F8
S3150800C4480023DBB21A463C4B1A7069E03B687B61ED
S3150800C4587B691B78002B62D038490520FEF7DAF885
S3150800C468FFF780FE0A2001F089FBFFF765FB3B68AA
S3150800C478BB61BB691B78002B14BF01230023DBB201
S3150800C4881A462F4B1A704BE03B68FB61FB691B8801
S3150800C4989AB22C4BA3F80F20FB695B889AB2294BF2
S3150800C4A8A3F81B203CE03B683B623B6A1A78264B9C
S3150800C4B81A7035E0254A3B681C46164604F1200CD6
S3150800C4C835462346186859689A68DB680FC51034D4
S3150800C4D810366445F4D13346224610685168926886
S3150800C4E807C31A4B5B881A4AA2FB0323DB089BB2CD
S3150800C4F8DAB2144B9A7013E03B681A78154B1A701F
S3150800C5080EE00C4B1B781846FDF7C0FE08E001F054
S3150800C5182BFB0346044A136002E000BF00E000BF95
S3150800C52800BF2C37BD46F0BD380B00203C0B002059
S3150800C538400B00204E0000203109002054600108F5
S3150800C548360B00203C030020370B0020640B002024
S3150800C558CDCCCCCC900B002080B586B000AF7860E7
S3150800C5680B467B807B88022B01D800235AE07B6820
S3150800C5781B78FB757B88033BBB827B88023B7A6802
S3150800C58813441B781AB27B88013B79680B441B78DD
S3150800C5981BB21B021BB213431BB27B82BB8A013335
S3150800C5A89BB219467868FFF735FD03463B827A8AB7
S3150800C5B83B8A9A4205D01D490420FEF72BF800232A
S3150800C5C830E0FB7D1846FFF7B1FE0346FB81FB8981
S3150800C5D84FF6FF72934207D1FB7D1A461449052088
S3150800C5E8FEF718F800231DE0FA89BB8A9A4207D095
S3150800C5F8FB7D1A460F490420FEF70CF8002311E0C4
S3150800C608BB8A002B07D07B68591CBA8AFB7D18465B
S3150800C618FFF7C8FE05E0FB7D002200211846FFF754
S3150800C628C1FE012318461837BD4680BD6C6001084F
S3150800C638806001089460010880B400AF0E4B1B683F
S3150800C6481B689AB20D4B1A800B4B1B685A790B4B11
S3150800C6589A70094B1B681A79084BDA70074B01223E
S3150800C6689A80064B0022DA80044B0A221A8100BFF8
S3150800C678BD4680BC704700BF000000201C10002083
S3150800C68880B500AF4FF404720021054807F0F4F9A5
S3150800C6984FF404720021034807F0EEF900BF80BD85
S3150800C6A8A00B0020B00D002080B500AF2A4B93F8E8
S3150800C6B84230DBB2202B0AD1284B93F80832DBB27A
S3150800C6C8002B04D1FF222649234805F013FD254BE4
S3150800C6D893F84230DBB2202B04D1FF2222492148A5
S3150800C6E805F008FD1C4B93F84130DBB2212B19D114
S3150800C6F81A4BD3F80C32002B14D001F035FA02463F
S3150800C708164BD3F80C32D31A642B0BD9124805F0FA
S3150800C7184FFD00221021154803F037FA0F4B002267
S3150800C728C3F80C220D4B93F80832DBB2002B11D054
S3150800C738094B93F84130DBB2212B0BD00C4800F09B
S3150800C748EDF9FF220649044805F0D4FC034B0022FC
S3150800C75883F8082200BF80BD4C110020A00B0020DA
S3150800C768A00C0020BC100020B00E002000140140C8
S3150800C778A00D002080B582B000AF78600B467B809C
S3150800C7887B681A68224B1B689A4216D17B881A4618
S3150800C7982049214800F08EF90346002B04D11422BB
S3150800C7A80021002000F0FAF81C4B00221A70FF221C
S3150800C7B81849174805F09EFC25E07B681A68184B47
S3150800C7C81B689A4214D17B881A461649164800F0FF
S3150800C7D871F90346002B05D0104B01221A7013482D
S3150800C7E800F09CF9FF220F490D4805F083FC0AE082
S3150800C7F87B681A680E4B1B689A4204D17B881946CF
S3150800C8087868FFF7AFF900BF0837BD4680BD00BF97
S3150800C8184C110020A00C0020A00B0020C00F0020FF
S3150800C828BC100020B00E0020B00D0020B00F00206C
S3150800C8389411002080B582B000AF78607B681A68CA
S3150800C848084B1B689A4208D100221021064803F0B3
S3150800C8589CF9064B0022C3F80C2200BF0837BD46D0
S3150800C86880BD00BF4C11002000140140A00B002019
S3150800C87880B485B000AF78600B467B804FF0FF33F5
S3150800C888FB6000237B8121E07B897A6813441B7847
S3150800C8981A46FB685340FB6000237B7210E0FB686E
S3150800C8A803F00103002B05D0FB685A080D4B5340CB
S3150800C8B8FB6002E0FB685B08FB607B7A01337B72EE
S3150800C8C87B7A072BEBD97B8901337B817A897B882D
S3150800C8D89A42D9D3FB68DB4318461437BD4680BC51
S3150800C8E8704700BF2083B8ED80B588B000AFF86000
S3150800C8F87A601A460B467B8113467B720023FB83B4
S3150800C908FB8B5A1CFA831A467B6813447A7A1A7080
S3150800C918FB68002B19D00023BB8312E0BB8BFA688F
S3150800C9281A44FB8B591CF98319467B680B44127801
S3150800C9381A70FB8BFA2B01D900232AE0BB8B01332B
S3150800C948BB83BA8B7B899A42E8D3FB8B19467868EE
S3150800C958FFF78EFF03463B6107F110037B6100234F
S3150800C968BB6112E0BB697A691A44FB8B591CF983C7
S3150800C97819467B680B4412781A70FB8BFE2B01D973
S3150800C988002306E0BB690133BB61BB69032BE9DDFC
S3150800C998FB8B18462037BD4680BD000080B584B09D
S3150800C9A800AF78600B467B8013467B707B78798866
S3150800C9B8154A7868FFF798FF0346FB81FB89002B21
S3150800C9C81ED0124B93F84130DBB2212B07D10F4802
S3150800C9D805F0EEFB002210210D4803F0D6F80122D7
S3150800C9E810210B4803F0D1F8FB891A46064907486F
S3150800C9F805F04BFB01F0B8F80346034AC2F80C32B7
S3150800CA0800BF1037BD4680BDA00B00204C11002082
S3150800CA180014014080B588B000AFF8600B467A600C
S3150800CA287B817B89042B01D800233FE07B89B3F5FA
S3150800CA38807F01D9002339E07B89043BFB83FB8B84
S3150800CA48FA6813441B781946FB8B0133FA681344B2
S3150800CA581B781B0241EA0302FB8B0233F9680B4475
S3150800CA681B781B041A43FB8B0333F9680B441B78A2
S3150800CA781B061343BB61FB8B1946F868FFF7F8FEDC
S3150800CA887861BA697B699A4201D000230EE0FB688F
S3150800CA985A1C7B685A60FB681A787B681A70FB8B85
S3150800CAA8DBB2013BDAB27B685A7001231846203795
S3150800CAB8BD4680BD80B584B000AFF860B96013463E
S3150800CAC8FB80FB6803F50072FB881946B868FFF710
S3150800CAD8A1FF0346002B01D1002304E0FB680122CD
S3150800CAE883F80822012318461037BD4680BD000082
S3150800CAF880B400AFBFF34F8F00BF064BDB6803F463
S3150800CB08E0620449044B1343CB60BFF34F8F00BF61
S3150800CB1800BFFDE700ED00E00400FA0580B584B023
S3150800CB2800AF78601323FB737B681B78C22B00F36E
S3150800CB38CC80B02B0FDA602B42D0602B00F3C5806F
S3150800CB48502B43D0502B00F3C080012B00F0A68051
S3150800CB58402B2DD0B9E0B03B122B00F2B68001A2CB
S3150800CB6852F823F0DBCB0008D3CC0008D3CC000856
S3150800CB78D3CC0008D3CC000883CC0008D3CC000853
S3150800CB88D3CC0008D3CC0008D3CC0008D3CC0008F3
S3150800CB98D3CC0008D3CC0008D3CC0008D3CC0008E3
S3150800CBA8D3CC000819CC00087DCC000851CC000865
S3150800CBB800F0B2F8402258214B48FFF7EFFE8FE005
S3150800CBC860220A214948FFF7E9FE89E0FDF7C0FC1B
S3150800CBD886E07B685B780B2B17D17B685A68444BD1
S3150800CBE81068516803C31189927A19809A70414B63
S3150800CBF801221A703E4BD3F803303D4A3E490720B6
S3150800CC08FDF708FD1223FB7362E01323FB735FE04D
S3150800CC187B685B78012B14D17B685B681B781A469E
S3150800CC284FF47A7302FB03F31A46344B5A61334BB3
S3150800CC385B691A4632490720FDF7ECFC1223FB7399
S3150800CC4846E01323FB7343E07B685B78012B0ED120
S3150800CC587B685B681A782B4B1A702A4B1B781A461E
S3150800CC6829490720FDF7D6FC1223FB7330E0132366
S3150800CC78FB732DE01323FB732AE012220021002000
S3150800CC88FFF78CFE00BF214B93F84130DBB2212B0E
S3150800CC98F9D00A2000F072FFFFF72AFF7B685B7855
S3150800CCA8092B0FD17B685A68194B1068516803C35A
S3150800CCB8127A1A70174B1B78DBB2012B0FD0122386
S3150800CCC8FB7305E01323FB7302E01323FB7300BF12
S3150800CCD8FB7B1A4600210020FFF760FE00E000BF34
S3150800CCE81037BD4680BD00BFC40F00201C100020A9
S3150800CCF86000002026100020B46001088C08002077
S3150800CD08C86001083C030020DC6001084C110020BB
S3150800CD1854000020C00F002080B500AF8F4B9A78CA
S3150800CD288F4B9A708D4BD3F807308D4AC2F803306B
S3150800CD388A4BB3F80F309AB2894BA3F80720874B6A
S3150800CD48B3F81B309AB2864BA3F80920834BB3F87D
S3150800CD5813309AB2824BA3F80B20804BB3F81530E0
S3150800CD689AB27F4BA3F80D207C4B1A7E7C4BDA735C
S3150800CD787A4B5A7F7A4B5A70784B5A78784B1A708E
S3150800CD88774B00221A7400225A74754B00229A743B
S3150800CD98734B0022DA7400221A750420FCF7C2FCC9
S3150800CDA8034603F00103D9B26D4A537D61F30003C4
S3150800CDB853750320FCF7B6FC034603F00103D9B202
S3150800CDC8674A537D61F3410353750020FCF7AAFCB3
S3150800CDD8034603F00103D9B2614A537D61F382031E
S3150800CDE853755F4A537D23F0080353750320FCF7F0
S3150800CDF8A9FC0346002B0CBF01230023D9B2584AC5
S3150800CE08537D61F304135375FDF78EFB0346002B18
S3150800CE1814BF01230023D9B2514A537D61F3451340
S3150800CE2853754F4A537D23F0400353754D4B1B7A70
S3150800CE3803F00103D9B24A4A537D61F3C713537500
S3150800CE480020FCF773FD03465AB2454B5A76012073
S3150800CE58FCF76CFD03465AB2414B9A76414BDB699F
S3150800CE685AB23F4BDA763E4B00221A773C4B0022E1
S3150800CE785A773B4B00229A770022DA77384B0022FA
S3150800CE8883F82020384B9B689AB2354BA3F82120A3
S3150800CE98354BDB689AB2324BA3F82320324B1B6911
S3150800CEA89AB22F4BA3F82520112200212F4806F005
S3150800CEB8E3FD2B4B002283F83820294B002283F800
S3150800CEC83920002283F83A20254B002283F83B2094
S3150800CED8002283F83C2004220021254806F0CCFDD0
S3150800CEE81F4B002283F84120002283F842200022A3
S3150800CEF883F84320002283F84420194B002283F83C
S3150800CF084720174B002283F84620154B002283F842
S3150800CF184520134B002283F84820002283F849202D
S3150800CF280F4B002283F84A2008220021114806F0F0
S3150800CF38A3FD0B4B002283F85320094B002283F8E4
S3150800CF485420002283F85520054B002283F85620E2
S3150800CF58002283F8572000BF80BD00BF3C0300208D
S3150800CF68C40F00208C08002060080020EB0F002062
S3150800CF78011000200F10002080B485B000AF78603B
S3150800CF887B68002B18D07B6800221A607B68002211
S3150800CF989A807B680022DA800023FB8108E0FA89F8
S3150800CFA87B680232002143F82210FB890133FB8192
S3150800CFB8FB89072BF3D900E000BF1437BD4680BCB0
S3150800CFC8704780B485B000AF786039607B68002BFD
S3150800CFD801D13B6856E07B68DB88072B27D87B6836
S3150800CFE89B881A467B680232396843F822107B68A0
S3150800CFF81A683B681A447B681A607B689B88013301
S3150800D0089AB27B689A807B689B88072B02D97B68CB
S3150800D01800229A807B68DB8801339AB27B68DA80BB
S3150800D0287B681B687A68D28893FBF2F32AE07B68E8
S3150800D0389B881A467B68023253F82230FB607B6865
S3150800D0489B881A467B680232396843F822107B683F
S3150800D0581A683968FB68CB1A1A447B681A607B68B1
S3150800D0689B8801339AB27B689A807B689B88072BD2
S3150800D07802D97B6800229A807B681B68002B00DA35
S3150800D0880733DB1018461437BD4680BC70470000C6
S3150800D09880B485B000AF154B9B69144A43F0010369
S3150800D0A89361124B9B6903F00103BB60BB680F4B86
S3150800D0B8DB690E4A43F08053D3610C4BDB6903F0F6
S3150800D0C880537B607B680A4B5B68FB60FB6823F0D0
S3150800D0D8E063FB60FB6843F00073FB60044AFB6887
S3150800D0E8536000BF1437BD4680BC70470010024025
S3150800D0F80000014080B400AF00BFFDE780B400AF70
S3150800D10800BFFDE780B400AF00BFFDE780B400AFFD
S3150800D11800BFFDE780B400AF00BFFDE780B400AFED
S3150800D12800BFBD4680BC704780B400AF00BFBD468F
S3150800D13880BC704780B400AF00BFBD4680BC70474E
S3150800D14880B500AF00F0FEFC00BF80BD80B500AF1B
S3150800D158024801F0EFFE00BF80BD00BFE8020020CC
S3150800D16880B500AF024804F0E5F800BF80BD00BFEF
S3150800D1782C10002080B500AF024805F02DF900BF35
S3150800D18880BD00BF0411002080B500AF024805F035
S3150800D19823F900BF80BD00BF4C11002080B500AF41
S3150800D1A8024805F019F900BF80BD00BF9411002098
S3150800D1B880B500AF024805F00FF900BF80BD00BF73
S3150800D1C8BC10002080B500AF024801F0B3FE00BFCE
S3150800D1D880BD00BF1003002080B500AF024801F0EB
S3150800D1E8A9FE00BF80BD00BF1003002080B400AFB1
S3150800D1F801231846BD4680BC704780B582B000AF8B
S3150800D2087860396006F040FC034616221A604FF02B
S3150800D218FF3318460837BD4680BD80B582B000AFD3
S3150800D22878604FF0FF317868FFF7E7FF00BFFDE742
S3150800D23880B586B000AFF860B9607A6000237B6174
S3150800D2480AE0AFF300800146BB685A1CBA60CAB246
S3150800D2581A707B6901337B617A697B689A42F0DBCD
S3150800D2687B6818461837BD4680BD80B483B000AFC2
S3150800D27878604FF0FF3318460C37BD4680BC7047B8
S3150800D28880B483B000AF786039603B684FF40052C9
S3150800D2985A60002318460C37BD4680BC704780B4D0
S3150800D2A883B000AF7860012318460C37BD4680BCAA
S3150800D2B8704780B485B000AFF860B9607A6000231B
S3150800D2C818461437BD4680BC7047000080B586B03E
S3150800D2D800AF7860144A154BD31A7B617B693B61AA
S3150800D2E8134B1B68002B02D1114B124A1A60104BBC
S3150800D2F81A687B6813443A699A4207D206F0C4FB4F
S3150800D30803460C221A604FF0FF3309E0084B1B68E6
S3150800D318FB60074B1A687B681344054A1360FB6869
S3150800D32818461837BD4680BD0000012000040000D5
S3150800D338281000203013002080B400AF00BFBD4677
S3150800D34880BC704780B58EB000AF07F1280300226D
S3150800D3581A605A609A60DA6007F1200300221A6098
S3150800D3685A603B1D00221A605A609A60DA601A6190
S3150800D3785A619A612C4B2D4A1A602B4B00225A6027
S3150800D388294B00229A60284B4FF6FF72DA60264B23
S3150800D39800221A61244B00229A61234803F083FD70
S3150800D3A80346002B01D0FDF7F5FB4FF48053BB620B
S3150800D3B807F1280319461C4804F06EF90346002BA2
S3150800D3C801D0FDF7E7FB184803F0B2FE0346002B29
S3150800D3D801D0FDF7DFFB00233B6200237B6207F1E0
S3150800D3E820031946104804F0FDFC0346002B01D01B
S3150800D3F8FDF7D0FB60237B600023BB600023FB603E
S3150800D40800237B613B1D04221946074804F082F86D
S3150800D4180346002B01D0FDF7BDFB034800F0CEF804
S3150800D42800BF3837BD4680BD2C10002000040040D8
S3150800D43880B58EB000AF07F1280300221A605A603B
S3150800D4489A60DA6007F1200300221A605A603B1DC9
S3150800D45800221A605A609A60DA601A615A619A61FB
S3150800D468374B384A1A60364B4FF434725A60344B85
S3150800D47800229A60324B6422DA60314B00221A6124
S3150800D4882F4B00229A612E4803F00DFD0346002B08
S3150800D49801D0FDF77FFB4FF48053BB6207F12803E1
S3150800D4A81946274804F0F8F80346002B01D0FDF77B
S3150800D4B871FB234803F03CFE0346002B01D0FDF719
S3150800D4C869FB00233B6200237B6207F120031946A8
S3150800D4D81B4804F087FC0346002B01D0FDF75AFBCE
S3150800D4E860237B600023BB600023FB6000237B610D
S3150800D4F83B1D04221946124804F00CF80346002B73
S3150800D50801D0FDF747FB3B1D082219460C4804F0D5
S3150800D51801F80346002B01D0FDF73CFB3B1D0C2206
S3150800D5281946074803F0F6FF0346002B01D0FDF716
S3150800D53831FB034800F042F800BF3837BD4680BDC6
S3150800D548741000200008004080B584B000AF7860E9
S3150800D5587B681B68164A934214D1164BDB69154A31
S3150800D56843F00203D361134BDB6903F00203FB6044
S3150800D578FB68002200211D2001F0D7FF1D2001F0BD
S3150800D588F0FF10E07B681B680B4A93420BD1094BE6
S3150800D598DB69084A43F00403D361064BDB6903F0E9
S3150800D5A80403BB60BB6800BF1037BD4680BD00BF1B
S3150800D5B800040040001002400008004080B58AB008
S3150800D5C800AF786007F1140300221A605A609A605F
S3150800D5D8DA607B681B68264A934218D1254B9B69F3
S3150800D5E8244A43F004039361224B9B6903F004031E
S3150800D5F83B613B6980237B610223BB6102233B6253
S3150800D60807F1140319461C4802F024F92BE07B6835
S3150800D6181B681A4A934226D1164B9B69154A43F04A
S3150800D62820039361134B9B6903F02003FB60FB6897
S3150800D6384FF460437B610223BB6102233B6207F117
S3150800D648140319460E4802F005F90E4B5B687B620F
S3150800D6587B6A43F0E0637B627B6A43F480537B62B0
S3150800D668084A7B6A536000BF2837BD4680BD00BF9D
S3150800D678000400400010024000080140000800406D
S3150800D688001401400000014080B500AF114B124A52
S3150800D6981A60104B4FF416525A600E4B00229A60C5
S3150800D6A80C4B0022DA600B4B00221A61094B0C223C
S3150800D6B85A61084B00229A61064B0022DA6105482E
S3150800D6C804F008FC0346002B01D0FDF763FA00BFF7
S3150800D6D880BD00BFBC1000200050004080B500AFD8
S3150800D6E8114B124A1A60104B4FF4E1325A600E4B2E
S3150800D6F800229A600C4B0022DA600B4B00221A6152
S3150800D708094B0C225A61084B00229A61064B0022E3
S3150800D718DA61054804F0DEFB0346002B01D0FDF765
S3150800D72839FA00BF80BD00BF041100200038014047
S3150800D73880B500AF114B124A1A60104B4FF4E1320C
S3150800D7485A600E4B00229A600C4B0022DA600B4B8B
S3150800D75800221A61094B0C225A61084B00229A6169
S3150800D768064B0022DA61054804F0B4FB0346002B91
S3150800D77801D0FDF70FFA00BF80BD00BF4C1100208D
S3150800D7880044004080B500AF114B124A1A60104B8E
S3150800D7984FF4E1325A600E4B00229A600C4B002275
S3150800D7A8DA600B4B00221A61094B0C225A61084BA6
S3150800D7B800229A61064B0022DA61054804F08AFBC2
S3150800D7C80346002B01D0FDF7E5F900BF80BD00BF71
S3150800D7D8941100200048004080B592B000AF7860E8
S3150800D7E807F1300300221A605A609A60DA607B688B
S3150800D7F81B68954A934245D1944BDB69934A43F48F
S3150800D8088013D361914BDB6903F48013FB62FB6ACF
S3150800D8188E4B9B698D4A43F0100393618B4B9B692A
S3150800D82803F01003BB62BB6A884B9B69874A43F0BF
S3150800D83820039361854B9B6903F020037B627B6A0F
S3150800D8484FF480533B6302237B630323FB6307F18F
S3150800D858300319467E4801F0FDFF04233B63002385
S3150800D8687B630023BB6307F130031946794801F047
S3150800D878F1FF00220021352001F057FE352001F07E
S3150800D88870FEDCE07B681B68734A93423AD16F4B9B
S3150800D8989B696E4A43F4804393616C4B9B6903F416
S3150800D8A880433B623B6A694B9B69684A43F00403B9
S3150800D8B89361664B9B6903F00403FB61FB694FF4AC
S3150800D8C800733B6302237B630323FB6307F130037F
S3150800D8D81946624801F0BEFF4FF480633B63002394
S3150800D8E87B630023BB6307F1300319465B4801F0E5
S3150800D8F8B1FF00220021252001F017FE252001F09E
S3150800D90830FE9CE07B681B68554A934246D14F4BCC
S3150800D918DB694E4A43F40033D3614C4BDB6903F4A5
S3150800D9280033BB61BB69494B9B69484A43F02003EE
S3150800D9389361464B9B6903F020037B617B6920232F
S3150800D9483B6302237B630323FB6307F13003194612
S3150800D958404801F07FFF40233B6300237B63002395
S3150800D968BB6307F1300319463A4801F073FF3D4B8C
S3150800D9785B683B643B6C43F0E0633B643B6C43F099
S3150800D98808033B64374A3B6C536000220021262073
S3150800D99801F0CBFD262001F0E4FD50E07B681B680A
S3150800D9A8314A93424BD1294BDB69284A43F48023F1
S3150800D9B8D361264BDB6903F480233B613B69234B20
S3150800D9C89B69224A43F010039361204B9B6903F035
S3150800D9D81003FB60FB684FF480633B6302237B6399
S3150800D9E80323FB6307F130031946194801F032FF90
S3150800D9F84FF400633B6300237B630023BB6307F193
S3150800DA0830031946124801F025FF164B5B687B64FC
S3150800DA187B6C23F030037B647B6C43F0E0637B64A8
S3150800DA287B6C43F010037B640E4A7B6C53600022C0
S3150800DA380021272001F079FD272001F092FD00BF7B
S3150800DA484837BD4680BD00BF005000400010024060
S3150800DA580010014000140140003801400008014048
S3150800DA68004400400000014000480040FFF764FCFD
S3150800DA780B480C490C4A002302E0D458C450043316
S3150800DA88C4188C42F9D3094A094C002301E01360EB
S3150800DA980432A242FBD305F0FDFFFCF78FFF70475F
S3150800DAA80000002040020020CC6401084002002043
S3150800DAB82C130020FEE7000080B500AF084B1B6852
S3150800DAC8074A43F010031360032001F023FD0F20D3
S3150800DAD800F008F8FFF7DCFA0023184680BD00BFF7
S3150800DAE80020024080B582B000AF7860124B1A68F1
S3150800DAF8124B1B7819464FF47A73B3FBF1F3B2FB52
S3150800DB08F3F3184601F03BFD0346002B01D0012329
S3150800DB180EE07B680F2B0AD8002279684FF0FF3091
S3150800DB2801F003FD064A7B681360002300E0012321
S3150800DB3818460837BD4680BD6C00002074000020D2
S3150800DB487000002080B400AF054B1B781A46054BB9
S3150800DB581B681344034A136000BFBD4680BC704760
S3150800DB6874000020DC11002080B400AF024B1B684B
S3150800DB781846BD4680BC7047DC11002080B584B0C5
S3150800DB8800AF7860FFF7F0FFB8607B68FB60FB685A
S3150800DB98B3F1FF3F05D00A4B1B781A46FB681344B6
S3150800DBA8FB6000BFFFF7E0FF0246BB68D31AFA68B6
S3150800DBB89A42F7D800BF00BF1037BD4680BD00BFE0
S3150800DBC87400002080B586B000AF78600023FB7526
S3150800DBD800233B610023BB600023FB607B68002BA6
S3150800DBE801D10123BEE07B689B68002B7B689B6A92
S3150800DBF8002B09D17B680022DA627B68002283F849
S3150800DC0824207868FBF7CAFC786800F0F1FB03461D
S3150800DC18FB757B689B6A03F01003002B40F099801C
S3150800DC28FB7D002B40F095807B689B6A23F488531C
S3150800DC3823F0020343F002027B689A627B685A68FB
S3150800DC487B68DB691A437B681B7B5B001343BA68EE
S3150800DC581343BB607B689B68B3F5807F03D07B68FA
S3150800DC689B68012B02D14FF4807300E000233A69C0
S3150800DC7813433B617B681B7D012B19D17B681B7B92
S3150800DC88002B09D17B689B69013B5A033B691343FF
S3150800DC9843F400633B610BE07B689B6A43F0200210
S3150800DCA87B689A627B68DB6A43F001027B68DA6202
S3150800DCB87B681B685B6823F469417B681B683A695B
S3150800DCC80A435A607B681B689A68284B13407A6827
S3150800DCD81268B9680B4393607B689B68B3F5807FC5
S3150800DCE803D07B689B68012B04D17B681B69013BC1
S3150800DCF81B05FB607B681B68DB6A23F470017B687D
S3150800DD081B68FA680A43DA627B681B689A68184BC4
S3150800DD181340BA689A420BD17B680022DA627B689C
S3150800DD289B6A23F0030343F001027B689A6218E0B2
S3150800DD387B689B6A23F0120343F010027B689A6299
S3150800DD487B68DB6A43F001027B68DA620123FB75AC
S3150800DD5807E07B689B6A43F010027B689A62012396
S3150800DD68FB75FB7D18461837BD4680BDFDF7E1FFF4
S3150800DD78FE0E1FFF80B584B000AF78600023FB73E2
S3150800DD887B6893F82430012B01D1022398E07B683D
S3150800DD98012283F82420786800F0D0FA0346FB733A
S3150800DDA8FB7B002B40F087807B689B6A23F44073D3
S3150800DDB823F0010343F480727B689A627B681B68C8
S3150800DDC8414A934205D1414B5B6803F47023002B03
S3150800DDD815D17B689B6A23F480127B689A627B68F4
S3150800DDE81B685B6803F48063002B26D07B689B6AF4
S3150800DDF823F4405343F480527B689A621DE07B689B
S3150800DE089B6A43F480127B689A627B681B682F4A70
S3150800DE18934204D07B681B682B4A93420DD12B4B3F
S3150800DE285B6803F48063002B07D07B689B6A23F43E
S3150800DE38405343F480527B689A627B689B6A03F472
S3150800DE488053002B06D07B68DB6A23F006027B68C2
S3150800DE58DA6202E07B680022DA627B68002283F8CD
S3150800DE6824207B681B686FF002021A607B681B68AF
S3150800DE789B6803F46023B3F5602F13D17B681B688E
S3150800DE88114A934205D1114B5B6803F47023002BA2
S3150800DE9808D17B681B689A687B681B6842F4A002ED
S3150800DEA89A600CE07B681B689A687B681B6842F472
S3150800DEB880129A6003E07B68002283F82420FB7BA3
S3150800DEC818461037BD4680BD002801400024014089
S3150800DED880B584B000AF78600023FB737B6893F83D
S3150800DEE82430012B01D102231AE07B68012283F82A
S3150800DEF82420786800F07CFA0346FB73FB7B002B2A
S3150800DF0809D17B689B6A23F4885323F0010343F0FD
S3150800DF1801027B689A627B68002283F82420FB7BCF
S3150800DF2818461037BD4680BD90B587B000AF7860F3
S3150800DF38396000237B610023FB6000233B61FFF700
S3150800DF4813FE78617B681B689B6803F48073002B53
S3150800DF580BD07B689B6A43F020027B689A627B68D1
S3150800DF68002283F824200123D3E07B681B685B68BA
S3150800DF7803F48073002B31D17B681B68DB6A03F4D2
S3150800DF887003002B2AD121E03B68B3F1FF3F1DD06F
S3150800DF983B68002B07D0FFF7E7FD02467B69D31AD3
S3150800DFA83A689A4212D27B681B681B6803F0020318
S3150800DFB8002B0BD17B689B6A43F004027B689A6244
S3150800DFC87B68002283F824200323A2E07B681B6869
S3150800DFD81B6803F00203002BD6D070E04F4B1C6871
S3150800DFE8022002F005FD0346B4FBF3F27B681B68C2
S3150800DFF819694B4B0B40002B18D17B681B68D968ED
S3150800E008484B0B40002B11D17B681B681969464B96
S3150800E0180B40002B08D17B681B68D968434B0B401B
S3150800E028002B01D1142320E029231EE07B681B68F6
S3150800E03819693D4B0B40002B06D17B681B68D968CC
S3150800E0483A4B0B40002B0DD07B681B681969384B77
S3150800E0580B40002B08D17B681B68D968344B0B40EA
S3150800E068002B01D1542300E0FC2302FB03F33B6198
S3150800E07821E03B68B3F1FF3F1AD03B68002B07D075
S3150800E088FFF772FD02467B69D31A3A689A420FD29D
S3150800E098FB683A699A420BD97B689B6A43F0040283
S3150800E0A87B689A627B68002283F82420032330E081
S3150800E0B8FB680133FB60FB683A699A42D9D87B68E2
S3150800E0C81B686FF012021A607B689B6A43F4007239
S3150800E0D87B689A627B681B689B6803F46023B3F5C0
S3150800E0E8602F15D17B681B7B002B11D17B689B6A37
S3150800E0F823F480727B689A627B689B6A03F4805370
S3150800E108002B05D17B689B6A43F001027B689A62FB
S3150800E118002318461C37BD4690BD00BF6C0000207A
S3150800E12824499224244992009224491292244900A7
S3150800E1384992240080B483B000AF78607B681B6876
S3150800E148DB6C18460C37BD4680BC704780B485B072
S3150800E15800AF786039600023FB730023BB607B68D7
S3150800E16893F82430012B01D10223DCE07B680122D5
S3150800E17883F824203B685B68062B1CD87B681B68D9
S3150800E188596B3B685A6813469B001344053B1F2284
S3150800E19802FA03F3DB4319403B6818683B685A6878
S3150800E1A813469B001344053B00FA03F27B681B6879
S3150800E1B80A435A633CE03B685B680C2B1CD87B68AF
S3150800E1C81B68196B3B685A6813469B001344233B24
S3150800E1D81F2202FA03F3DB4319403B6818683B68B9
S3150800E1E85A6813469B001344233B00FA03F27B68DC
S3150800E1F81B680A431A631BE07B681B68D96A3B6875
S3150800E2085A6813469B001344413B1F2202FA03F33C
S3150800E218DB4319403B6818683B685A6813469B00F5
S3150800E2281344413B00FA03F27B681B680A43DA6227
S3150800E2383B681B68092B1CD97B681B68D9683B682F
S3150800E2481A6813465B0013441E3B072202FA03F3B7
S3150800E258DB4319403B6898683B681A6813465B00B5
S3150800E26813441E3B00FA03F27B681B680A43DA600C
S3150800E27819E07B681B6819693B681A6813465B00CE
S3150800E2881344072202FA03F3DB4319403B689868EC
S3150800E2983B681A6813465B00134400FA03F27B6866
S3150800E2A81B680A431A613B681B68102B03D03B6836
S3150800E2B81B68112B32D17B681B681D4A934225D1EE
S3150800E2C87B681B689B6803F40003002B26D17B68D0
S3150800E2D81B689A687B681B6842F400029A603B6868
S3150800E2E81B68102B1AD1134B1B68134AA2FB03236E
S3150800E2F89A0C13469B0013445B00BB6002E0BB689C
S3150800E308013BBB60BB68002BF9D107E07B689B6AB9
S3150800E31843F020027B689A620123FB737B6800221C
S3150800E32883F82420FB7B18461437BD4680BC704703
S3150800E338002401406C00002083DE1B4380B584B0AE
S3150800E34800AF78600023FB600023BB607B681B680E
S3150800E3589B6803F00103012B40D07B681B689A6809
S3150800E3687B681B6842F001029A601F4B1B681F4AAC
S3150800E378A2FB03239B0CBB6002E0BB68013BBB60A6
S3150800E388BB68002BF9D1FFF7EFFBF8601FE0FFF732
S3150800E398EBFB0246FB68D31A022B18D97B681B6865
S3150800E3A89B6803F00103012B11D07B689B6A43F035
S3150800E3B810027B689A627B68DB6A43F001027B6815
S3150800E3C8DA627B68002283F82420012307E07B6849
S3150800E3D81B689B6803F00103012BD8D10023184654
S3150800E3E81037BD4680BD00BF6C00002083DE1B4386
S3150800E3F880B584B000AF78600023FB607B681B6833
S3150800E4089B6803F00103012B2ED17B681B689A6869
S3150800E4187B681B6822F001029A60FFF7A5FBF86083
S3150800E4281BE0FFF7A1FB0246FB68D31A022B14D997
S3150800E4387B681B689B6803F00103012B0DD17B6879
S3150800E4489B6A43F010027B689A627B68DB6A43F032
S3150800E45801027B68DA62012307E07B681B689B6810
S3150800E46803F00103012BDCD0002318461037BD46FC
S3150800E47880BD000090B587B000AF78600023FB75B3
S3150800E4880023FB607B6893F82430012B01D1022313
S3150800E49897E07B68012283F824207868FFF7A8FFAD
S3150800E4A80346FB757868FFF749FF0346FB75FB7D4E
S3150800E4B8002B40F081807B689B6A23F4885323F0FD
S3150800E4C8020343F002027B689A62404B1C680220EA
S3150800E4D802F08EFA0346B4FBF3F35B00FB6002E036
S3150800E4E8FB68013BFB60FB68002BF9D17B681B685E
S3150800E4F89A687B681B6842F008029A60FFF734FB43
S3150800E50838611BE0FFF730FB02463B69D31A0A2B32
S3150800E51814D97B681B689B6803F00803002B0DD089
S3150800E5287B689B6A23F0120343F010027B689A62A1
S3150800E5387B68002283F82420012342E07B681B6855
S3150800E5489B6803F00803002BDCD17B681B689A6874
S3150800E5587B681B6842F004029A60FFF705FB38617E
S3150800E5681BE0FFF701FB02463B69D31A0A2B14D9AD
S3150800E5787B681B689B6803F00403002B0DD07B6837
S3150800E5889B6A23F0120343F010027B689A627B6841
S3150800E598002283F82420012313E07B681B689B6804
S3150800E5A803F00403002BDCD17B689B6A23F0030382
S3150800E5B843F001027B689A627B68002283F824206C
S3150800E5C8FB7D18461C37BD4690BD00BF6C00002071
S3150800E5D880B584B000AF78607B68002B01D1012331
S3150800E5E8EDE07B6893F82030DBB2002B02D178681F
S3150800E5F8FBF7D0FA7B681B681A687B681B6842F0C9
S3150800E60801021A60FFF7B0FAF86012E0FFF7ACFAF1
S3150800E6180246FB68D31A0A2B0BD97B685B6A43F454
S3150800E62800327B685A627B68052283F8202001231A
S3150800E638C5E07B681B685B6803F00103002BE5D01F
S3150800E6487B681B681A687B681B6822F002021A60D6
S3150800E658FFF78AFAF86012E0FFF786FA0246FB68BF
S3150800E668D31A0A2B0BD97B685B6A43F400327B689A
S3150800E6785A627B68052283F8202001239FE07B687D
S3150800E6881B685B6803F00203002BE5D17B681B7ED9
S3150800E698012B08D17B681B681A687B681B6842F0DF
S3150800E6A880021A6007E07B681B681A687B681B6823
S3150800E6B822F080021A607B685B7E012B08D17B6892
S3150800E6C81B681A687B681B6842F040021A6007E0F4
S3150800E6D87B681B681A687B681B6822F040021A6008
S3150800E6E87B689B7E012B08D17B681B681A687B6848
S3150800E6F81B6842F020021A6007E07B681B681A68E4
S3150800E7087B681B6822F020021A607B68DB7E012B77
S3150800E71808D17B681B681A687B681B6822F0100298
S3150800E7281A6007E07B681B681A687B681B6842F0F2
S3150800E73810021A607B681B7F012B08D17B681B684F
S3150800E7481A687B681B6842F008021A6007E07B684B
S3150800E7581B681A687B681B6822F008021A607B68BF
S3150800E7685B7F012B08D17B681B681A687B681B6866
S3150800E77842F004021A6007E07B681B681A687B681F
S3150800E7881B6822F004021A607B689A687B68DB6853
S3150800E7981A437B681B691A437B685B6942EA03016B
S3150800E7A87B685B685A1E7B681B680A43DA617B6864
S3150800E7B800225A627B68012283F820200023184623
S3150800E7C81037BD4680BD000080B487B000AF7860BA
S3150800E7D839607B681B687B617B6893F82030FB741B
S3150800E7E8FB7C012B03D0FB7C022B40F0BE80654BDB
S3150800E7F87B617B69D3F8003243F001027B69C3F871
S3150800E80800227B69D3F8003223F47C527B69C3F86B
S3150800E81800227B69D3F800223B685B6A1B021A430D
S3150800E8287B69C3F800223B685B6903F01F03012272
S3150800E83802FA03F3FB607B69D3F81C22FB68DB4307
S3150800E8481A407B69C3F81C223B68DB69002B23D175
S3150800E8587B69D3F80C22FB68DB431A407B69C3F84B
S3150800E8680C223B68DB6819043B685B689BB23A680C
S3150800E878526919437B69483243F832103B689B68EA
S3150800E88819043B681B689AB23B685B690A4379694D
S3150800E8984833DB000B445A603B68DB69012B22D1FD
S3150800E8A87B69D3F80C22FB681A437B69C3F80C22E8
S3150800E8B83B681B6819043B685B689BB23A685269EF
S3150800E8C819437B69483243F832103B689B68190438
S3150800E8D83B68DB689AB23B685B690A4379694833DF
S3150800E8E8DB000B445A603B689B69002B09D17B699E
S3150800E8F8D3F80422FB68DB431A407B69C3F8042271
S3150800E90807E07B69D3F80422FB681A437B69C3F8D6
S3150800E91804223B681B69002B09D17B69D3F81422AA
S3150800E928FB68DB431A407B69C3F8142207E07B6956
S3150800E938D3F81422FB681A437B69C3F814223B6888
S3150800E9481B6A012B07D17B69D3F81C22FB681A437B
S3150800E9587B69C3F81C227B69D3F8003223F00102CD
S3150800E9687B69C3F80022002306E07B685B6A43F4E8
S3150800E97880227B685A62012318461C37BD4680BC2C
S3150800E988704700BF0064004080B584B000AF786067
S3150800E9987B6893F82030DBB2012B2ED17B680222E4
S3150800E9A883F820207B681B681A687B681B6822F036
S3150800E9B801021A60FFF7D8F8F86012E0FFF7D4F8F2
S3150800E9C80246FB68D31A0A2B0BD97B685B6A43F4A1
S3150800E9D800327B685A627B68052283F82020012367
S3150800E9E812E07B681B685B6803F00103002BE5D11E
S3150800E9F87B6800225A62002306E07B685B6A43F458
S3150800EA0800227B685A62012318461037BD4680BD26
S3150800EA1880B584B000AF78607B6893F82030DBB2A5
S3150800EA28022B33D17B681B681A687B681B6842F01F
S3150800EA3801021A60FFF798F8F86012E0FFF794F8F1
S3150800EA480246FB68D31A0A2B0BD97B685B6A43F420
S3150800EA5800327B685A627B68052283F820200123E6
S3150800EA681BE07B681B685B6803F00103002BE5D095
S3150800EA787B681B681A687B681B6822F002021A60A2
S3150800EA887B68012283F82020002306E07B685B6AFE
S3150800EA9843F480127B685A62012318461037BD462C
S3150800EAA880BD80B489B000AFF860B9607A603B6011
S3150800EAB8FB6893F82030FB77FB681B689B68BB618B
S3150800EAC8FB7F012B03D0FB7F022B40F0AD80BB698F
S3150800EAD803F08063002B0AD1BB6903F00063002B9F
S3150800EAE805D1BB6903F08053002B00F09580BB69FC
S3150800EAF81B0E03F003037B6101227B699A403B687E
S3150800EB081A60BB689B68002B0DD1BB681B685A0541
S3150800EB18BB68DB68F96809681A437B6918331B01FF
S3150800EB280B441A600FE0BB685B68DA00BB689B6831
S3150800EB381A43BB68DB68F96809681A437B6918339E
S3150800EB481B010B441A60FB681968BB681A697B695C
S3150800EB5818331B010B4404331A60BB681B7D012B51
S3150800EB6811D1FB681A687B6918331B0113440433EF
S3150800EB781B68FA68116843F480727B6918331B01AD
S3150800EB880B4404331A607B6807331B781A067B68BC
S3150800EB9806331B781B041A437B6805331B781B024C
S3150800EBA813437A68043212781046FA68116843EAF9
S3150800EBB800027B691B010B4403F5C6731A607B6860
S3150800EBC803331B781A067B6802331B781B041A431F
S3150800EBD87B6801331B781B0213437A681278104640
S3150800EBE8FA68116843EA00027B691B010B4403F5BE
S3150800EBF8C4731A60FB681A687B6918331B011344C7
S3150800EC081B68FA68116843F001027B6918331B010F
S3150800EC180B441A6000230EE0FB685B6A43F4001293
S3150800EC28FB685A62012306E0FB685B6A43F48022A4
S3150800EC38FB685A62012318462437BD4680BC7047CC
S3150800EC4880B485B000AF78600023FB607B6893F8D2
S3150800EC582030FB72FB7A012B02D0FB7A022B1DD1DE
S3150800EC687B681B689B6803F08063002B02D0FB68EF
S3150800EC780133FB607B681B689B6803F00063002B05
S3150800EC8802D0FB680133FB607B681B689B6803F04E
S3150800EC988053002B02D0FB680133FB60FB681846DB
S3150800ECA81437BD4680BC704780B487B000AFF8609B
S3150800ECB8B9607A603B60FB6893F82030FB75FB7D8A
S3150800ECC8012B03D0FB7D022B40F00381BB68002B88
S3150800ECD80ED1FB681B68DB6803F00303002B16D10B
S3150800ECE8FB685B6A43F40012FB685A620123F7E083
S3150800ECF8FB681B681B6903F00303002B07D1FB6835
S3150800ED085B6A43F40012FB685A620123E8E0FB6871
S3150800ED181A68BB681B331B0113441B6803F00402FB
S3150800ED287B689A607B689B68002B0CD1FB681A681D
S3150800ED38BB681B331B0113441B685B0DC3F30A022C
S3150800ED487B681A600BE0FB681A68BB681B331B01F3
S3150800ED5813441B68DB0823F060427B685A60FB682B
S3150800ED681A68BB681B331B0113441B6803F00202AD
S3150800ED787B68DA60FB681A68BB681B331B01134497
S3150800ED8804331B6803F00803002B03D07B680822AA
S3150800ED981A610BE0FB681A68BB681B331B0113442E
S3150800EDA804331B6803F00F027B681A61FB681A684C
S3150800EDB8BB681B331B01134404331B681B0ADAB2EE
S3150800EDC87B689A61FB681A68BB681B331B01134486
S3150800EDD804331B681B0C9AB27B685A61FB681A686D
S3150800EDE8BB681B01134403F5DC731B68DAB23B687E
S3150800EDF81A70FB681A68BB681B01134403F5DC73B1
S3150800EE081B681A0A3B680133D2B21A70FB681A687B
S3150800EE18BB681B01134403F5DC731B681A0C3B68B3
S3150800EE280233D2B21A70FB681A68BB681B0113440E
S3150800EE3803F5DC731B681A0E3B680333D2B21A70E3
S3150800EE48FB681A68BB681B01134403F5DE731A6866
S3150800EE583B680433D2B21A70FB681A68BB681B0190
S3150800EE68134403F5DE731B681A0A3B680533D2B2E6
S3150800EE781A70FB681A68BB681B01134403F5DE732E
S3150800EE881B681A0C3B680633D2B21A70FB681A68F4
S3150800EE98BB681B01134403F5DE731B681A0E3B682F
S3150800EEA80733D2B21A70BB68002B08D1FB681B68F7
S3150800EEB8DA68FB681B6842F02002DA6007E0FB683C
S3150800EEC81B681A69FB681B6842F020021A6100234E
S3150800EED806E0FB685B6A43F48022FB685A620123F2
S3150800EEE818461C37BD4680BC704780B485B000AF4D
S3150800EEF8786039607B6893F82030FB73FB7B012BBD
S3150800EF0802D0FB7B022B09D17B681B6859697B6891
S3150800EF181B683A680A435A61002306E07B685B6AFD
S3150800EF2843F480227B685A62012318461437BD4683
S3150800EF3880BC704780B58AB000AF786000237B62D2
S3150800EF487B681B685B693B627B681B685B68FB615F
S3150800EF587B681B689B68BB617B681B68DB687B6191
S3150800EF687B681B681B693B617B681B689B69FB6040
S3150800EF783B6A03F00103002B7CD0BB6903F001034D
S3150800EF88002B23D07B681B6801229A60BB6903F0B3
S3150800EF980203002B03D0786800F083F916E0BB69F2
S3150800EFA803F00403002B04D07B6A43F400637B62F6
S3150800EFB80CE0BB6903F00803002B04D07B6A43F412
S3150800EFC880537B6202E0786800F086F9BB6903F42F
S3150800EFD88073002B24D07B681B684FF480729A6074
S3150800EFE8BB6903F40073002B03D0786800F062F954
S3150800EFF816E0BB6903F48063002B04D07B6A43F4EC
S3150800F00800537B620CE0BB6903F40063002B04D051
S3150800F0187B6A43F480437B6202E0786800F065F90E
S3150800F028BB6903F48033002B24D07B681B684FF434
S3150800F03880329A60BB6903F40033002B03D07868E2
S3150800F04800F041F916E0BB6903F48023002B04D0CD
S3150800F0587B6A43F400437B620CE0BB6903F4002334
S3150800F068002B04D07B6A43F480337B6202E078681D
S3150800F07800F044F93B6A03F00803002B0CD07B69BF
S3150800F08803F01003002B07D07B6A43F400737B62F6
S3150800F0987B681B681022DA603B6A03F00403002BBE
S3150800F0A80BD07B6903F00803002B06D07B681B6826
S3150800F0B80822DA60786800F033F93B6A03F002033D
S3150800F0C8002B09D07B681B68DB6803F00303002B59
S3150800F0D802D0786800F01BF93B6A03F04003002B5E
S3150800F0E80CD03B6903F01003002B07D07B6A43F466
S3150800F0F880637B627B681B6810221A613B6A03F08F
S3150800F1082003002B0BD03B6903F00803002B06D01D
S3150800F1187B681B6808221A61786800F00AF93B6A56
S3150800F12803F01003002B09D07B681B681B6903F0E2
S3150800F1380303002B02D07868FBF7BCFD3B6A03F48F
S3150800F1480033002B0BD0FB6903F01003002B06D005
S3150800F1587B681B6810225A60786800F0F3F83B6AE7
S3150800F16803F48033002B0BD0FB6903F00803002B4C
S3150800F17806D07B681B6808225A60786800F0EBF8A6
S3150800F1883B6A03F40043002B7BD0FB6903F00403B6
S3150800F198002B72D03B6A03F48073002B08D0FB68F7
S3150800F1A803F00103002B03D07B6A43F001037B625B
S3150800F1B83B6A03F40073002B08D0FB6803F00203CC
S3150800F1C8002B03D07B6A43F002037B623B6A03F495
S3150800F1D88063002B08D0FB6803F00403002B03D0D8
S3150800F1E87B6A43F004037B623B6A03F40063002BE3
S3150800F1F843D0FB6803F07003002B3ED0FB6803F08E
S3150800F2087003602B2BD0602B2ED8502B22D0502B76
S3150800F2182AD8402B19D0402B26D8302B10D0302B83
S3150800F22822D8102B02D0202B05D01DE07B6A43F08C
S3150800F23808037B6219E07B6A43F010037B6214E0DB
S3150800F2487B6A43F020037B620FE07B6A43F0400346
S3150800F2587B620AE07B6A43F080037B6205E07B6A8F
S3150800F26843F480737B6200E000BF7B681B689A6979
S3150800F2787B681B6822F070029A617B681B68042207
S3150800F2885A607B6A002B08D07B685A6A7B6A1A43DD
S3150800F2987B685A62786800F067F800BF2837BD4669
S3150800F2A880BD80B483B000AF786000BF0C37BD4618
S3150800F2B880BC704780B483B000AF786000BF0C3755
S3150800F2C8BD4680BC704780B483B000AF786000BF85
S3150800F2D80C37BD4680BC704780B483B000AF7860F1
S3150800F2E800BF0C37BD4680BC704780B483B000AFFA
S3150800F2F8786000BF0C37BD4680BC704780B483B0C1
S3150800F30800AF786000BF0C37BD4680BC704780B434
S3150800F31883B000AF786000BF0C37BD4680BC704725
S3150800F32880B483B000AF786000BF0C37BD4680BC98
S3150800F338704780B483B000AF786000BF0C37BD460D
S3150800F34880BC704780B483B000AF786000BF0C37C4
S3150800F358BD4680BC704780B483B000AF786000BFF4
S3150800F3680C37BD4680BC704780B483B000AF786060
S3150800F37800BF0C37BD4680BC7047000080B485B016
S3150800F38800AF78607B6803F00703FB600C4BDB680B
S3150800F398BB60BA684FF6FF031340BB60FB681A02E6
S3150800F3A8BB68134343F0BF6343F40033BB60044AA6
S3150800F3B8BB68D36000BF1437BD4680BC704700BF22
S3150800F3C800ED00E080B400AF044BDB681B0A03F0CD
S3150800F3D807031846BD4680BC704700BF00ED00E02D
S3150800F3E880B483B000AF0346FB7197F90730002B4A
S3150800F3F80BDBFB7903F01F02064997F907305B090F
S3150800F408012000FA02F241F8232000BF0C37BD4656
S3150800F41880BC704700E100E080B483B000AF0346C3
S3150800F4283960FB7197F90730002B0ADB3B68DAB2BB
S3150800F4380C4997F907301201D2B20B4483F8002316
S3150800F4480AE03B68DAB20849FB7903F00F03043B84
S3150800F4581201D2B20B441A7600BF0C37BD4680BCDF
S3150800F468704700BF00E100E000ED00E080B489B015
S3150800F47800AFF860B9607A60FB6803F00703FB61C0
S3150800F488FB69C3F10703042B28BF0423BB61FB6987
S3150800F4980433062B02D9FB69033B00E000237B6192
S3150800F4A84FF0FF32BB6902FA03F3DA43BB681A4026
S3150800F4B87B699A404FF0FF317B6901FA03F3D94318
S3150800F4C87B680B40134318462437BD4680BC7047F3
S3150800F4D880B582B000AF78607B68013BB3F1807F66
S3150800F4E801D301230FE00A4A7B68013B53600F21C9
S3150800F4F84FF0FF30FFF790FF054B00229A60044B48
S3150800F50807221A60002318460837BD4680BD00BF83
S3150800F51810E000E080B582B000AF78607868FFF741
S3150800F5282DFF00BF0837BD4680BD80B586B000AF41
S3150800F5380346B9607A60FB7300237B61FFF742FFD5
S3150800F54878617A68B9687869FFF790FF024697F98B
S3150800F5580F3011461846FFF75FFF00BF1837BD463C
S3150800F56880BD80B582B000AF0346FB7197F90730B6
S3150800F5781846FFF735FF00BF0837BD4680BD80B57A
S3150800F58882B000AF78607868FFF7A2FF034618468E
S3150800F5980837BD4680BD80B582B000AF78607B6805
S3150800F5A8002B01D101230EE07B685B79DBB2002BC7
S3150800F5B805D17B6800221A717868FAF727FF7B68F5
S3150800F5C801225A71002318460837BD4680BD80B403
S3150800F5D885B000AF78600023FB737B6893F8213009
S3150800F5E8DBB2022B08D07B6804229A637B68002268
S3150800F5F883F82020012320E07B681B681A687B684B
S3150800F6081B6822F00E021A607B681B681A687B68FA
S3150800F6181B6822F001021A607B681A6C7B68DB6B30
S3150800F628012101FA02F25A607B68012283F8212037
S3150800F6387B68002283F82020FB7B18461437BD46D2
S3150800F64880BC704780B584B000AF78600023FB7330
S3150800F6587B6893F82130DBB2022B05D07B6804223D
S3150800F6689A630123FB73D6E07B681B681A687B6874
S3150800F6781B6822F00E021A607B681B681A687B688A
S3150800F6881B6822F001021A607B681B681A46644BDD
S3150800F6989A4258D97B681B68624A93424FD07B685E
S3150800F6A81B68614A934248D07B681B685F4A934245
S3150800F6B840D07B681B685E4A934238D07B681B68D3
S3150800F6C85C4A934230D07B681B685B4A934228D0D1
S3150800F6D87B681B68524A934220D07B681B68574A46
S3150800F6E8934219D07B681B68554A934212D07B68A7
S3150800F6F81B68544A93420AD07B681B68524A93424D
S3150800F70802D14FF480531BE04FF4803318E04FF4CE
S3150800F718807315E0102313E0012311E04FF080737E
S3150800F7280EE04FF480130BE04FF4803308E04FF4F3
S3150800F738805305E04FF4807302E0102300E00123AC
S3150800F748424A536057E07B681B68364A93424FD053
S3150800F7587B681B68344A934248D07B681B68334ADF
S3150800F768934240D07B681B68314A934238D07B68FD
S3150800F7781B68304A934230D07B681B682E4A9342EE
S3150800F78828D07B681B68264A934220D07B681B686A
S3150800F7982A4A934219D07B681B68294A934212D091
S3150800F7A87B681B68274A93420AD07B681B68264AE7
S3150800F7B8934202D14FF480531BE04FF4803318E08C
S3150800F7C84FF4807315E0102313E0012311E04FF07E
S3150800F7D880730EE04FF480130BE04FF4803308E093
S3150800F7E84FF4805305E04FF4807302E0102300E0DD
S3150800F7F80123174A53607B68012283F821207B6816
S3150800F808002283F820207B685B6B002B03D07B687B
S3150800F8185B6B78689847FB7B18461037BD4680BDF2
S3150800F82880000240080002401C00024030000240E6
S3150800F83844000240580002406C0002400804024096
S3150800F8481C040240300402404404024000040240FA
S3150800F8580000024080B48BB000AF7860396000239E
S3150800F8687B6200233B6269E101227B6A02FA03F3A1
S3150800F878FB613B681B68FA691340BB61BA69FB6997
S3150800F8889A4240F058813B685B689A4A93425ED030
S3150800F898984A934275D8984A934258D0964A9342BA
S3150800F8A86FD8964A934252D0944A934269D8944A52
S3150800F8B893424CD0924A934263D8924A934246D08E
S3150800F8C8904A93425DD8122B2AD8122B59D801A2EE
S3150800F8D852F823F057F9000831F9000843F90008E7
S3150800F8E885F900088BF900088BF900088BF90008D8
S3150800F8F88BF900088BF900088BF900088BF90008C2
S3150800F9088BF900088BF900088BF900088BF90008B1
S3150800F9188BF900088BF9000839F900084DF9000831
S3150800F928794A934213D02CE03B68DB683B6229E0AE
S3150800F9383B68DB6804333B6224E03B68DB680833D2
S3150800F9483B621FE03B68DB680C333B621AE03B68A6
S3150800F9589B68002B02D104233B6213E03B689B6833
S3150800F968012B05D108233B627B68FA691A6109E00D
S3150800F97808233B627B68FA695A6103E000233B6205
S3150800F98800E000BFBB69FF2B01D87B6801E07B68F4
S3150800F99804337B61BB69FF2B02D87B6A9B0002E0B4
S3150800F9A87B6A083B9B003B617B691A680F213B69A8
S3150800F9B801FA03F3DB431A40396A3B6901FA03F390
S3150800F9C81A437B691A603B685B6803F08053002B0F
S3150800F9D800F0B1804D4B9B694C4A43F00103936193
S3150800F9E84A4B9B6903F00103BB60BB68484A7B6ABC
S3150800F9F89B08023352F82330FB607B6A03F0030343
S3150800FA089B000F2202FA03F3DB43FA681340FB60F4
S3150800FA187B68404A934213D07B683F4A93420DD08D
S3150800FA287B683E4A934207D07B683D4A934201D198
S3150800FA38032306E0042304E0022302E0012300E08E
S3150800FA4800237A6A02F0030292009340FA68134385
S3150800FA58FB602F497B6A9B080233FA6841F8232022
S3150800FA683B685B6803F48013002B06D02D4B9A6815
S3150800FA782C49BB6913438B6006E02A4B9A68BB6915
S3150800FA88DB43284913408B603B685B6803F4001323
S3150800FA98002B06D0234BDA682249BB691343CB608F
S3150800FAA806E0204BDA68BB69DB431E491340CB6086
S3150800FAB83B685B6803F40033002B06D0194B5A6879
S3150800FAC81849BB6913434B6006E0164B5A68BB696D
S3150800FAD8DB43144913404B603B685B6803F4803387
S3150800FAE8002B21D00F4B1A680E49BB6913430B60CC
S3150800FAF821E000BF0000321000003110000022107B
S3150800FB080000211000001210000011100010024019
S3150800FB180000014000080140000C014000100140A7
S3150800FB2800140140000401400B4B1A68BB69DB430B
S3150800FB38094913400B607B6A01337B623B681A6884
S3150800FB487B6A22FA03F3002B7FF48EAE00BF00BF50
S3150800FB582C37BD4680BC70470004014080B485B088
S3150800FB6800AF78600B467B807B689A687B88134071
S3150800FB78002B02D00123FB7301E00023FB73FB7BF8
S3150800FB8818461437BD4680BC704780B483B000AFAA
S3150800FB9878600B467B8013467B707B78002B03D0F6
S3150800FBA87A887B681A6103E07B881A047B681A617D
S3150800FBB800BF0C37BD4680BC7047000080B400AF54
S3150800FBC8034B01221A6000BFBD4680BC704700BFC0
S3150800FBD820000E4280B582B000AFFDF7C5FF7860F9
S3150800FBE8604B1B685F4A43F00103136008E0FDF7A2
S3150800FBF8BBFF02467B68D31A022B01D90323ACE064
S3150800FC08584B1B6803F00203002BF0D0554B1B68B2
S3150800FC1823F0F803534A43F080031360FDF7A4FF63
S3150800FC287860504B00225A600AE0FDF79DFF0246AD
S3150800FC387B68D31A41F28832934201D903238CE0B0
S3150800FC48484B5B6803F00C03002BEED1464B474A3A
S3150800FC581A60474B1B681846FDF744FF0346002BF6
S3150800FC6801D0012379E0FDF77FFF78603D4B1B68DB
S3150800FC783C4A23F08073136008E0FDF775FF0246D7
S3150800FC887B68D31A022B01D9032366E0354B1B6818
S3150800FC9803F00073002BF0D1324B00225A60FDF7AF
S3150800FCA863FF78602F4B1B682E4A23F410231360D2
S3150800FCB808E0FDF759FF02467B68D31A642B01D979
S3150800FCC803234AE0274B1B6803F40033002BF0D1C3
S3150800FCD8244B1B68234A23F480231360FDF744FF4B
S3150800FCE87860204B1B681F4A23F08063136008E07E
S3150800FCF8FDF73AFF02467B68D31A642B01D903231A
S3150800FD082BE0184B1B6803F00063002BF0D1FDF7B6
S3150800FD182BFF7860134B1B68124A23F08053136035
S3150800FD2808E0FDF721FF02467B68D31A642B01D940
S3150800FD38032312E00B4B1B6803F00053002BF0D18A
S3150800FD48084B0022DA62074B5B6A064A43F080735F
S3150800FD585362044B00229A60002318460837BD46AA
S3150800FD6880BD00BF001002406C00002000127A0017
S3150800FD787000002080B586B000AF78607B68002BDD
S3150800FD8801D1012304E37B681B6803F00103002BF8
S3150800FD9800F08780924B5B6803F00C03042B0CD0A9
S3150800FDA88F4B5B6803F00C03082B12D18C4B5B68EE
S3150800FDB803F48033B3F5803F0BD1894B1B6803F4F2
S3150800FDC80033002B6CD07B689B68002B68D1012315
S3150800FDD8DEE27B689B68B3F5803F06D1804B1B68DB
S3150800FDE87F4A43F4803313602EE07B689B68002BB8
S3150800FDF80CD17B4B1B687A4A23F480331360784B03
S3150800FE081B68774A23F4802313601DE07B689B6888
S3150800FE18B3F5A02F0CD1724B1B68714A43F48023A3
S3150800FE2813606F4B1B686E4A43F4803313600BE00C
S3150800FE386B4B1B686A4A23F480331360684B1B684C
S3150800FE48674A23F4802313607B689B68002B13D0CA
S3150800FE58FDF78AFE386108E0FDF786FE02463B692B
S3150800FE68D31A642B01D9032392E25D4B1B6803F46A
S3150800FE780033002BF0D014E0FDF776FE386108E071
S3150800FE88FDF772FE02463B69D31A642B01D9032390
S3150800FE987EE2534B1B6803F40033002BF0D100E0D5
S3150800FEA800BF7B681B6803F00203002B63D04C4B2A
S3150800FEB85B6803F00C03002B0BD0494B5B6803F017
S3150800FEC80C03082B1CD1464B5B6803F48033002BC4
S3150800FED816D1434B1B6803F00203002B05D07B6839
S3150800FEE85B69012B01D0012352E23D4B1B6823F0C5
S3150800FEF8F8027B689B69DB00394913430B603AE0D3
S3150800FF087B685B69002B20D0364B01221A60FDF707
S3150800FF182BFE386108E0FDF727FE02463B69D31A2F
S3150800FF28022B01D9032333E22D4B1B6803F0020386
S3150800FF38002BF0D02A4B1B6823F0F8027B689B69D4
S3150800FF48DB00274913430B6015E0264B00221A608D
S3150800FF58FDF70AFE386108E0FDF706FE02463B692A
S3150800FF68D31A022B01D9032312E21D4B1B6803F08F
S3150800FF780203002BF0D17B681B6803F00803002BEB
S3150800FF883AD07B68DB69002B19D0174B01221A6017
S3150800FF98FDF7EAFD386108E0FDF7E6FD02463B692C
S3150800FFA8D31A022B01D90323F2E10D4B5B6A03F03E
S3150800FFB80203002BF0D0012000F0CAFB1CE00A4B14
S3150800FFC800221A60FDF7D0FD38610FE0FDF7CCFD79
S3150800FFD802463B69D31A022B08D90323D8E100BF86
S3150800FFE80010024000004242800442429B4B5B6A72
S3150800FFF803F00203002BE9D17B681B6803F00403AE
S31508010008002B00F0A6800023FB75944BDB6903F0EF
S315080100188053002B0DD1914BDB69904A43F08053ED
S31508010028D3618E4BDB6903F08053BB60BB68012340
S31508010038FB758B4B1B6803F48073002B18D1884B0F
S315080100481B68874A43F480731360FDF78DFD386191
S3150801005808E0FDF789FD02463B69D31A642B01D9E5
S31508010068032395E17E4B1B6803F48073002BF0D0BC
S315080100787B681B69012B06D1784B1B6A774A43F0C3
S31508010088010313622DE07B681B69002B0CD1734BA6
S315080100981B6A724A23F001031362704B1B6A6F4A83
S315080100A823F0040313621CE07B681B69052B0CD13A
S315080100B86A4B1B6A694A43F004031362674B1B6A56
S315080100C8664A43F0010313620BE0644B1B6A634AF1
S315080100D823F001031362614B1B6A604A23F0040388
S315080100E813627B681B69002B15D0FDF73DFD386146
S315080100F80AE0FDF739FD02463B69D31A41F288320F
S31508010108934201D9032343E1544B1B6A03F00203C3
S31508010118002BEED014E0FDF727FD38610AE0FDF75C
S3150801012823FD02463B69D31A41F28832934201D923
S3150801013803232DE1494B1B6A03F00203002BEED179
S31508010148FB7D012B05D1454BDB69444A23F08053D6
S31508010158D3617B68DB6A002B00F08C803F4B5B68B8
S3150801016803F48033B3F5803F0ED13C4B5B6803F04B
S315080101780C03082B08D1394BDB6A03F48033B3F532
S31508010188803F01D1012303E17B68DB6A022B4ED14B
S31508010198324B1B6803F08053002B09D02F4BDB6ABF
S315080101A803F0F0027B685B6B9A4201D00123EFE00A
S315080101B82C4B00221A60FDF7D7FC386108E0FDF7D9
S315080101C8D3FC02463B69D31A642B01D90323DFE022
S315080101D8224B1B6803F00063002BF0D11F4BDB6A27
S315080101E823F0F0027B685B6B1C491343CB621B4BFC
S315080101F8DB6A23F470627B681B6B18491343CB626D
S31508010208184B01221A60FDF7AFFC386108E0FDF7C3
S31508010218ABFC02463B69D31A642B01D90323B7E021
S315080102280E4B1B6803F00063002BF0D022E00B4B42
S31508010238DB6A0A4A23F48033D3620A4B00221A601E
S31508010248FDF792FC38610FE0FDF78EFC02463B6923
S31508010258D31A642B08D903239AE000BF0010024079
S3150801026800700040680042424B4B1B6803F000636C
S31508010278002BE9D17B681B6A002B00F08880464B66
S315080102885B6803F00C03082B68D07B681B6A022B92
S315080102984DD1424B00221A60FDF766FC386108E029
S315080102A8FDF762FC02463B69D31A022B01D90323DF
S315080102B86EE0394B1B6803F00073002BF0D17B689D
S315080102C85B6AB3F5803F0FD1334BDA6A7B685B68A3
S315080102D831491343CB62304BDB6A23F00F027B6843
S315080102E8DB682D491343CB622B4B5B6823F47412E5
S315080102F87B68596A7B689B6A0B43274913434B609A
S31508010308264B01221A60FDF72FFC386108E0FDF734
S315080103182BFC02463B69D31A022B01D9032337E082
S315080103281D4B1B6803F00073002BF0D02FE01B4B05
S3150801033800221A60FDF718FC386108E0FDF714FC7D
S3150801034802463B69D31A022B01D9032320E0124B33
S315080103581B6803F00073002BF0D118E07B681B6A51
S31508010368012B01D1012313E00B4B5B68FB60FB688A
S3150801037803F480327B685B6A9A4206D1FB6803F408
S3150801038870127B689B6A9A4201D0012300E0002318
S3150801039818461837BD4680BD001002406000424223
S315080103A880B584B000AF786039607B68002B01D1CD
S315080103B80123D0E06A4B1B6803F007033A689A429F
S315080103C810D9674B1B6823F0070265493B68134335
S315080103D80B60634B1B6803F007033A689A4201D01E
S315080103E80123B8E07B681B6803F00203002B20D0C1
S315080103F87B681B6803F00403002B05D0594B5B681F
S31508010408584A43F4E06353607B681B6803F00803A2
S31508010418002B05D0534B5B68524A43F4605353602B
S31508010428504B5B6823F0F0027B689B684D49134380
S315080104384B607B681B6803F00103002B40D07B687F
S315080104485B68012B07D1474B1B6803F40033002B64
S3150801045815D101237FE07B685B68022B07D1414BE5
S315080104681B6803F00073002B09D1012373E03D4B88
S315080104781B6803F00203002B01D101236BE0394BFA
S315080104885B6823F003027B685B68364913434B6054
S31508010498FDF76AFBF8600AE0FDF766FB0246FB68AA
S315080104A8D31A41F28832934201D9032353E02D4BDB
S315080104B85B6803F00C027B685B689B009A42EBD188
S315080104C8274B1B6803F007033A689A4210D2244B54
S315080104D81B6823F0070222493B6813430B60204B2C
S315080104E81B6803F007033A689A4201D0012332E0F0
S315080104F87B681B6803F00403002B08D0194B5B685B
S3150801050823F4E0627B68DB68164913434B607B6812
S315080105181B6803F00803002B09D0124B5B6823F408
S3150801052860527B681B69DB000E4913434B6000F078
S3150801053821F802460B4B5B681B0903F00F030A49AE
S31508010548CB5C22FA03F3094A1360094B1B68184660
S31508010558FDF7C8FA002318461037BD4680BD00BF07
S315080105680020024000100240F06001086C000020DB
S31508010578700000202DE9B04F8EB000AF0023FB6252
S315080105880023BB6200237B6300237B6200233B6352
S3150801059800233B620023FB614E4B5B68FB62FB6AE7
S315080105A803F00C03042B02D0082B03D089E04A4B2D
S315080105B83B6389E0FB6A9B0C03F00F02474B9B5C84
S315080105C87B62FB6A03F48033002B72D0414BDB6AEA
S315080105D803F00F02424B9B5CBB623E4BDB6A03F49A
S315080105E88033002B53D03B4BDB6A1B0903F00F03FF
S315080105F801333B62374BDB6A1B0A03F00F030233ED
S31508010608FB61FB6900229A4693467B6A00223B6195
S315080106187A613B6903FB0BF27B690AFB03F3134413
S315080106283A69AAFB02010B4419462B4B03FB01F253
S31508010638002300FB03F31344274AA0FB02452B4476
S315080106481D463B6A0022BB60FA60BB6A00223B6012
S315080106587A60D7E902010B46D7E900AB524602FB95
S3150801066803F25B4684460CFB03F3134402465146E0
S31508010678A2FB01894B44994642464B4620462946E0
S31508010688F8F7B4FD02460B4613467B6307E07B6A17
S31508010698114A03FB02F2BB6AB2FBF3F37B630F4B06
S315080106A85B7B1A467B6A934208D17B6B5B087B6343
S315080106B804E07B6A0B4A02FB03F37B637B6B3B63B0
S315080106C802E0094B3B6300BF3B6B18463837BD460A
S315080106D8BDE8B08F0010024040787D010861010825
S315080106E81861010800093D0000127A0080B400AFBC
S315080106F8024B1B681846BD4680BC70476C00002033
S3150801070880B500AFFFF7F2FF0246054B5B681B0A87
S3150801071803F007030349CB5C22FA03F3184680BDA5
S31508010728001002400061010880B500AFFFF7DEFF3F
S315080107380246054B5B68DB0A03F007030349CB5CF2
S3150801074822FA03F3184680BD001002400061010829
S3150801075880B485B000AF78600A4B1B680A4AA2FBC9
S3150801076803235B0A7A6802FB03F3FB6000BFFB6895
S315080107785A1EFA60002BF9D100BF00BF1437BD46CF
S3150801078880BC70476C000020D34D621080B588B0D4
S3150801079800AF786000237B6100233B610023FB617E
S315080107A87B681B6803F00103002B7DD00023FB76C9
S315080107B88B4BDB6903F08053002B0DD1884BDB6922
S315080107C8874A43F08053D361854BDB6903F080532D
S315080107D8FB60FB680123FB76824B1B6803F4807375
S315080107E8002B18D17F4B1B687E4A43F4807313602C
S315080107F8FDF7BAF9786108E0FDF7B6F902467B69AB
S31508010808D31A642B01D90323E5E0764B1B6803F455
S315080108188073002BF0D0724B1B6A03F440733B615B
S315080108283B69002B2ED07B685B6803F440733A69F1
S315080108389A4227D06A4B1B6A23F440733B616A4B79
S3150801084801221A60684B00221A60654A3B691362DD
S315080108583B6903F00103002B14D0FDF785F978618C
S315080108680AE0FDF781F902467B69D31A41F2883213
S31508010878934201D90323AEE0594B1B6A03F00203DD
S31508010888002BEED0564B1B6A23F440727B685B68D3
S31508010898534913430B62FB7E012B05D1504BDB6988
S315080108A84F4A23F08053D3617B681B6803F0020320
S315080108B8002B08D04A4B5B6823F440427B689B6847
S315080108C8474913434B607B681B6803F00403002BF5
S315080108D808D0434BDB6A23F400327B68DB6840495E
S315080108E81343CB627B681B6803F00803002B08D007
S315080108F83B4BDB6A23F480227B681B69384913431F
S31508010908CB62374BDB6A03F40033002B05D1344B32
S31508010918DB6A03F48023002B01D00123FB61FB6901
S31508010928012B48D12E4B1B6803F08053002B38D175
S315080109382B4B1B6803F08063002B09D0284BDB6A15
S3150801094803F0F0027B689B699A4201D0012342E0D1
S31508010958234BDB6A23F0F0027B689B692049134322
S31508010968CB621F4BDB6A23F470427B685B691C49BF
S315080109781343CB621D4B01221A60FDF7F5F878611E
S3150801098808E0FDF7F1F802467B69D31A642B01D909
S31508010998032320E0124B1B6803F00053002BF0D009
S315080109A809E00F4BDB6A03F470427B685B699A427C
S315080109B801D001230FE07B681B6803F01003002BA5
S315080109C808D0074B5B6823F480027B68DB69044916
S315080109D813434B60002318462037BD4680BD00BF28
S315080109E80010024000700040400442427000424232
S315080109F880B58AB000AF78600023FB6100237B626B
S31508010A080023BB6100237B6100233B610023FB6054
S31508010A180023BB6000233B627B68013B0F2B00F276
S31508010A281D8101A252F823F0E50B0108490C0108BA
S31508010A38650C0108430B0108650C0108650C0108DA
S31508010A48650C0108950B0108650C0108650C010878
S31508010A58650C0108650C0108650C0108650C010897
S31508010A68650C0108710A0108834B5B68BB60824BF8
S31508010A781B6803F08073002B00F0F280BB689B0C9F
S31508010A8803F00F037D4AD35CBB61BB6803F480336B
S31508010A98002B3BD0784BDB6A03F00F03784AD35C0B
S31508010AA8FB61754BDB6A03F48033002B1CD0724B50
S31508010AB8DB6A1B0903F00F030133FB606E4BDB6A24
S31508010AC81B0A03F00F0302337B616E4AFB68B2FB0C
S31508010AD8F3F37A6903FB02F2FB69B2FBF3F2BB692A
S31508010AE802FB03F37B6207E0664AFB69B2FBF3F292
S31508010AF8BB6902FB03F37B62604B5B7B1A46BB69E6
S31508010B08934208D17B6A5B087B6204E0BB695E4A4B
S31508010B1802FB03F37B62584B5B6803F48003B3F566
S31508010B28800F02D17B6A3B629AE07B6A5B00574A6F
S31508010B38A2FB03235B083B6292E04F4BDB6A03F493
S31508010B480033002B03D1FFF715FD38628AE04A4BBB
S31508010B581B6803F08053002B00F08480464BDB6A40
S31508010B681B0903F00F030133FB60434BDB6A1B0BBD
S31508010B7803F00F0302333B61424AFB68B2FBF3F306
S31508010B883A6902FB03F35B003B626BE03A4BDB6AAB
S31508010B9803F48023002B03D1FFF7ECFC386263E0EA
S31508010BA8354B1B6803F08053002B5DD0324BDB6A4B
S31508010BB81B0903F00F030133FB602F4BDB6A1B0B81
S31508010BC803F00F0302333B612E4AFB68B2FBF3F3CA
S31508010BD83A6902FB03F35B003B6245E0264B1B6A55
S31508010BE8BB60BB6803F44073B3F5807F08D1BB6863
S31508010BF803F00203002B03D04FF400433B621EE0C7
S31508010C08BB6803F44073B3F5007F09D11A4B5B6AD5
S31508010C1803F00203002B03D049F640433B620EE07A
S31508010C28BB6803F44073B3F5407F1FD1124B1B68A9
S31508010C3803F40033002B19D0154B3B6216E015E077
S31508010C48FFF772FD02460C4B5B689B0B03F0030327
S31508010C5801335B00B2FBF3F33B6208E000BF06E031
S31508010C6800BF04E000BF02E000BF00E000BF3B6A26
S31508010C7818462837BD4680BD00100240286101087C
S31508010C883861010840787D0100093D00ABAAAAAA86
S31508010C98F0FA020080B584B000AF78600023FB60E3
S31508010CA87B68002B01D101237AE07B685B7CDBB288
S31508010CB8002B05D17B6800221A747868FAF718FFA1
S31508010CC87B6802225A74786800F070F80346002B8C
S31508010CD804D07B6804225A74012361E0786800F01D
S31508010CE892F80346002B04D07B6804225A74012320
S31508010CF856E07B681B685A687B681B6822F00702FE
S31508010D085A607B689B68002B05D0274B1B6B264AC4
S31508010D1823F001031363244BDB6A23F460727B68AF
S31508010D289B6821491343CB627B685B68B3F1FF3F34
S31508010D3803D07B685B68FB600EE00120FFF758FE6D
S31508010D48F860FB68002B04D17B6804225A740123D6
S31508010D5826E0FB68013BFB60FB681A0C7B681B688D
S31508010D6802F00F029A607B681B68FA6892B2DA6029
S31508010D78786800F070F80346002B04D07B680422D3
S31508010D885A7401230CE07B680022DA737B68012216
S31508010D985A737B6801229A737B6801225A74002365
S31508010DA818461037BD4680BD006C004080B584B032
S31508010DB800AF78600023FB607B68002B01D1012313
S31508010DC81DE07B681B685A687B681B6822F0080265
S31508010DD85A60FCF7C9FEF86009E0FCF7C5FE024649
S31508010DE8FB68D31AB3F57A7F01D9032307E07B6831
S31508010DF81B685B6803F00803002BEED0002318462E
S31508010E081037BD4680BD80B584B000AF7860002331
S31508010E18FB60FCF7A9FEF86009E0FCF7A5FE0246A7
S31508010E28FB68D31AB3F57A7F01D903230FE07B68E8
S31508010E381B685B6803F02003002BEED07B681B68F0
S31508010E485A687B681B6842F010025A6000231846E4
S31508010E581037BD4680BD80B584B000AF78600023E1
S31508010E68FB607B681B685A687B681B6822F010025E
S31508010E785A60FCF779FEF86009E0FCF775FE024648
S31508010E88FB68D31AB3F57A7F01D9032307E07B6890
S31508010E981B685B6803F02003002BEED00023184675
S31508010EA81037BD4680BD80B582B000AF78607B68D3
S31508010EB8002B01D1012341E07B6893F83D30DBB271
S31508010EC8002B06D17B68002283F83C207868FCF75A
S31508010ED83BFB7B68022283F83D207B681A687B689E
S31508010EE804331946104600F0C3FC7B68012283F8CF
S31508010EF846207B68012283F83E207B68012283F815
S31508010F083F207B68012283F840207B68012283F809
S31508010F1841207B68012283F842207B68012283F8F5
S31508010F2843207B68012283F844207B68012283F8E1
S31508010F3845207B68012283F83D2000231846083797
S31508010F48BD4680BD80B584B000AF7860396000239E
S31508010F58FB733B68002B09D17B6893F83E30DBB2FB
S31508010F68012B14BF01230023DBB222E03B68042BC3
S31508010F7809D17B6893F83F30DBB2012B14BF0123F3
S31508010F880023DBB215E03B68082B09D17B6893F887
S31508010F984030DBB2012B14BF01230023DBB208E082
S31508010FA87B6893F84130DBB2012B14BF0123002378
S31508010FB8DBB2002B01D00123AEE03B68002B04D13C
S31508010FC87B68022283F83E2013E03B68042B04D190
S31508010FD87B68022283F83F200BE03B68082B04D183
S31508010FE87B68022283F8402003E07B68022283F8A3
S31508010FF841203B680C2B41D801A252F823F000BFC7
S315080110083D10010885100108851001088510010899
S315080110184F10010885100108851001088510010877
S315080110286110010885100108851001088510010855
S31508011038731001087B681B68DA687B681B6842F0CD
S315080110480202DA601DE07B681B68DA687B681B6840
S3150801105842F00402DA6014E07B681B68DA687B6888
S315080110681B6842F00802DA600BE07B681B68DA68DD
S315080110787B681B6842F01002DA6002E00123FB7301
S3150801108800BFFB7B002B46D17B681B6801223968A8
S31508011098184600F083FE7B681B68214A934207D1EC
S315080110A87B681B685A6C7B681B6842F400425A6461
S315080110B87B681B681A4A934213D07B681B68B3F18D
S315080110C8804F0ED07B681B68164A934209D07B6805
S315080110D81B68154A934204D07B681B68134A9342D6
S315080110E811D17B681B689B6803F00703BB60BB6863
S315080110F8062B10D07B681B681A687B681B6842F048
S3150801110801021A6007E07B681B681A687B681B6816
S3150801111842F001021A60FB7B18461037BD4680BDAE
S31508011128002C01400004004000080040000C004063
S3150801113880B582B000AF78607B68002B01D10123A6
S3150801114841E07B6893F83D30DBB2002B06D17B681A
S31508011158002283F83C20786800F039F87B68022277
S3150801116883F83D207B681A687B680433194610465C
S3150801117800F07EFB7B68012283F846207B68012202
S3150801118883F83E207B68012283F83F207B68012289
S3150801119883F840207B68012283F841207B68012275
S315080111A883F842207B68012283F843207B68012261
S315080111B883F844207B68012283F845207B6801224D
S315080111C883F83D20002318460837BD4680BD80B4FC
S315080111D883B000AF786000BF0C37BD4680BC704746
S315080111E880B584B000AF786039603B68002B09D1B7
S315080111F87B6893F83E30DBB2012B14BF0123002329
S31508011208DBB222E03B68042B09D17B6893F83F30AF
S31508011218DBB2012B14BF01230023DBB215E03B68BF
S31508011228082B09D17B6893F84030DBB2012B14BF30
S3150801123801230023DBB208E07B6893F84130DBB26F
S31508011248012B14BF01230023DBB2002B01D0012394
S3150801125863E03B68002B04D17B68022283F83E20B1
S3150801126813E03B68042B04D17B68022283F83F20EC
S315080112780BE03B68082B04D17B68022283F84020DF
S3150801128803E07B68022283F841207B681B680122F8
S315080112983968184600F082FD7B681B68214A934223
S315080112A807D17B681B685A6C7B681B6842F4004245
S315080112B85A647B681B681B4A934213D07B681B6870
S315080112C8B3F1804F0ED07B681B68174A934209D041
S315080112D87B681B68154A934204D07B681B68144AC5
S315080112E8934211D17B681B689B6803F00703FB606F
S315080112F8FB68062B10D07B681B681A687B681B6815
S3150801130842F001021A6007E07B681B681A687B6865
S315080113181B6842F001021A60002318461037BD46B9
S3150801132880BD00BF002C01400004004000080040B1
S31508011338000C004080B584B000AF78607B681B68F4
S31508011348DB68FB607B681B681B69BB60BB6803F0CD
S315080113580203002B20D0FB6803F00203002B1BD0E5
S315080113687B681B686FF002021A617B6801221A778B
S315080113787B681B689B6903F00303002B03D0786815
S3150801138800F05AFA05E07868F9F704F8786800F081
S315080113985CFA7B6800221A77BB6803F00403002B02
S315080113A820D0FB6803F00403002B1BD07B681B685D
S315080113B86FF004021A617B6802221A777B681B6838
S315080113C89B6903F44073002B03D0786800F034FA5C
S315080113D805E07868F8F7DEFF786800F036FA7B6882
S315080113E800221A77BB6803F00803002B20D0FB6894
S315080113F803F00803002B1BD07B681B686FF00802F3
S315080114081A617B6804221A777B681B68DB6903F013
S315080114180303002B03D0786800F00EFA05E0786814
S31508011428F8F7B8FF786800F010FA7B6800221A778F
S31508011438BB6803F01003002B20D0FB6803F01003E8
S31508011448002B1BD07B681B686FF010021A617B683A
S3150801145808221A777B681B68DB6903F44073002B3B
S3150801146803D0786800F0E8F905E07868F8F792FF9C
S31508011478786800F0EAF97B6800221A77BB6803F0F6
S315080114880103002B0CD0FB6803F00103002B07D0DE
S315080114987B681B686FF001021A61786800F0C3F966
S315080114A8BB6803F08003002B0CD0FB6803F08003AC
S315080114B8002B07D07B681B686FF080021A61786871
S315080114C800F0FFFCBB6803F04003002B0CD0FB6857
S315080114D803F04003002B07D07B681B686FF04002B6
S315080114E81A61786800F0BAF9BB6803F02003002B83
S315080114F80CD0FB6803F02003002B07D07B681B6818
S315080115086FF020021A61786800F0D2FC00BF103724
S31508011518BD4680BD80B586B000AFF860B9607A600F
S315080115280023FB75FB6893F83C30012B01D1022394
S31508011538AEE0FB68012283F83C207B680C2B00F29D
S315080115489F8001A252F823F085150108891601081A
S315080115588916010889160108C51501088916010899
S315080115688916010889160108071601088916010846
S31508011578891601088916010847160108FB681B68B8
S31508011588B968184600F0ECF9FB681B689A69FB68A4
S315080115981B6842F008029A61FB681B689A69FB682E
S315080115A81B6822F004029A61FB681B689969BB6883
S315080115B81A69FB681B680A439A6164E0FB681B6839
S315080115C8B968184600F032FAFB681B689A69FB681D
S315080115D81B6842F400629A61FB681B689A69FB6892
S315080115E81B6822F480629A61FB681B689969BB6863
S315080115F81B691A02FB681B680A439A6143E0FB6880
S315080116081B68B968184600F07BFAFB681B68DA6933
S31508011618FB681B6842F00802DA61FB681B68DA692D
S31508011628FB681B6822F00402DA61FB681B68D96942
S31508011638BB681A69FB681B680A43DA6123E0FB6819
S315080116481B68B968184600F0C5FAFB681B68DA69A9
S31508011658FB681B6842F40062DA61FB681B68DA6991
S31508011668FB681B6822F48062DA61FB681B68D96922
S31508011678BB681B691A02FB681B680A43DA6102E040
S315080116880123FB7500BFFB68002283F83C20FB7D1C
S3150801169818461837BD4680BD80B584B000AF786056
S315080116A839600023FB737B6893F83C30012B01D121
S315080116B80223B4E07B68012283F83C207B68022276
S315080116C883F83D207B681B689B68BB60BB6823F071
S315080116D87703BB60BB6823F47F43BB607B681B68E1
S315080116E8BA689A603B681B68B3F5005F3ED0B3F5E4
S315080116F8005F00F28780B3F5805F00F08680B3F556
S31508011708805F7FD8702B1AD0702B7BD8602B50D06E
S31508011718602B77D8502B3CD0502B73D8402B58D0F8
S31508011728402B6FD8302B64D0302B6BD8202B60D048
S31508011738202B67D8002B5CD0102B5AD062E07B6827
S3150801174818683B6899683B685A683B68DB6800F023
S3150801175806FB7B681B689B68BB60BB6843F077031D
S31508011768BB607B681B68BA689A604FE07B68186833
S315080117783B6899683B685A683B68DB6800F0EFFA8A
S315080117887B681B689A687B681B6842F480429A6082
S315080117983CE07B6818683B6859683B68DB681A4609
S315080117A800F066FA7B681B685021184600F0BDFAF6
S315080117B82CE07B6818683B6859683B68DB681A46F9
S315080117C800F084FA7B681B686021184600F0ADFAB8
S315080117D81CE07B6818683B6859683B68DB681A46E9
S315080117E800F046FA7B681B684021184600F09DFA06
S315080117F80CE07B681A683B681B681946104600F0B6
S3150801180894FA03E00123FB7300E000BF7B68012219
S3150801181883F83D207B68002283F83C20FB7B184629
S315080118281037BD4680BD80B483B000AF786000BF6D
S315080118380C37BD4680BC704780B483B000AF78606A
S3150801184800BF0C37BD4680BC704780B483B000AF73
S31508011858786000BF0C37BD4680BC704780B483B03A
S3150801186800AF786000BF0C37BD4680BC70470000E2
S3150801187880B485B000AF786039607B681B68FB6007
S315080118887B68334A93420FD07B68B3F1804F0BD0FC
S315080118987B68304A934207D07B682F4A934203D024
S315080118A87B682E4A934208D1FB6823F07003FB60D4
S315080118B83B685B68FA681343FB607B68244A934272
S315080118C80FD07B68B3F1804F0BD07B68214A9342CE
S315080118D807D07B68204A934203D07B681F4A934204
S315080118E808D1FB6823F44073FB603B68DB68FA6838
S315080118F81343FB60FB6823F080023B685B6913436B
S31508011908FB607B68FA681A603B689A687B68DA62E2
S315080119183B681A687B689A627B680D4A934203D1C9
S315080119283B681A697B681A637B6801225A617B6876
S315080119381B6903F00103002B05D07B681B6923F09B
S3150801194801027B681A6100BF1437BD4680BC70471F
S31508011958002C01400004004000080040000C00402B
S3150801196880B487B000AF786039607B681B6A7B6191
S315080119787B681B6A23F001027B681A627B685B68CD
S315080119883B617B689B69FB60FB6823F07003FB601E
S31508011998FB6823F00303FB603B681B68FA6813437B
S315080119A8FB607B6923F002037B613B689B687A6964
S315080119B813437B617B681C4A93420CD17B6923F0EC
S315080119C808037B613B68DB687A6913437B617B693A
S315080119D823F004037B617B68134A934211D13B695F
S315080119E823F480733B613B6923F400733B613B68CD
S315080119F85B693A6913433B613B689B693A691343D7
S31508011A083B617B683A695A607B68FA689A613B6800
S31508011A185A687B685A637B687A691A6200BF1C37F9
S31508011A28BD4680BC704700BF002C014080B487B012
S31508011A3800AF786039607B681B6A7B617B681B6AC3
S31508011A4823F010027B681A627B685B683B617B68D6
S31508011A589B69FB60FB6823F4E043FB60FB6823F49E
S31508011A684073FB603B681B681B02FA681343FB60FB
S31508011A787B6923F020037B613B689B681B017A69B4
S31508011A8813437B617B681D4A93420DD17B6923F019
S31508011A9880037B613B68DB681B017A6913437B61B9
S31508011AA87B6923F040037B617B68144A934213D10F
S31508011AB83B6923F480633B613B6923F400633B611B
S31508011AC83B685B699B003A6913433B613B689B69C1
S31508011AD89B003A6913433B617B683A695A607B689C
S31508011AE8FA689A613B685A687B689A637B687A6977
S31508011AF81A6200BF1C37BD4680BC7047002C0140DE
S31508011B0880B487B000AF786039607B681B6A7B61EF
S31508011B187B681B6A23F480727B681A627B685B6838
S31508011B283B617B68DB69FB60FB6823F07003FB603C
S31508011B38FB6823F00303FB603B681B68FA681343D9
S31508011B48FB607B6923F400737B613B689B681B0216
S31508011B587A6913437B617B681D4A93420DD17B6978
S31508011B6823F400637B613B68DB681B027A691343CC
S31508011B787B617B6923F480637B617B68144A9342A2
S31508011B8813D13B6923F480533B613B6923F4005322
S31508011B983B613B685B691B013A6913433B613B68D7
S31508011BA89B691B013A6913433B617B683A695A6029
S31508011BB87B68FA68DA613B685A687B68DA637B6826
S31508011BC87A691A6200BF1C37BD4680BC704700BFD8
S31508011BD8002C014080B487B000AF786039607B6813
S31508011BE81B6A3B617B681B6A23F480527B681A620D
S31508011BF87B685B687B617B68DB69FB60FB6823F450
S31508011C08E043FB60FB6823F44073FB603B681B6891
S31508011C181B02FA681343FB603B6923F400533B61D3
S31508011C283B689B681B033A6913433B617B680F4A08
S31508011C38934209D17B6923F480437B613B685B69DD
S31508011C489B017A6913437B617B687A695A607B6869
S31508011C58FA68DA613B685A687B681A647B683A6984
S31508011C681A6200BF1C37BD4680BC7047002C01406C
S31508011C7880B487B000AFF860B9607A60FB681B6A00
S31508011C887B61FB681B6A23F00102FB681A62FB6821
S31508011C989B693B613B6923F0F0033B617B681B0148
S31508011CA83A6913433B617B6923F00A037B617A69C5
S31508011CB8BB6813437B61FB683A699A61FB687A6971
S31508011CC81A6200BF1C37BD4680BC704780B487B00E
S31508011CD800AFF860B9607A60FB681B6A7B61FB68CC
S31508011CE81B6A23F01002FB681A62FB689B693B6151
S31508011CF83B6923F470433B617B681B033A691343C9
S31508011D083B617B6923F0A0037B61BB681B017A6988
S31508011D1813437B61FB683A699A61FB687A691A62B7
S31508011D2800BF1C37BD4680BC704780B485B000AF7C
S31508011D38786039607B689B68FB60FB6823F07003F1
S31508011D48FB603A68FB68134343F00703FB607B684B
S31508011D58FA689A6000BF1437BD4680BC704780B4DC
S31508011D6887B000AFF860B9607A603B60FB689B682A
S31508011D787B617B6923F47F437B613B681A027B6835
S31508011D881A43BB6813437A6913437B61FB687A690B
S31508011D989A6000BF1C37BD4680BC704780B487B0BF
S31508011DA800AFF860B9607A60BB6803F01F030122C7
S31508011DB802FA03F37B61FB681A6A7B69DB431A40FB
S31508011DC8FB681A62FB681A6ABB6803F01F0379681D
S31508011DD801FA03F31A43FB681A6200BF1C37BD46AA
S31508011DE880BC704780B485B000AF786039607B687D
S31508011DF893F83C30012B01D102234BE07B68012281
S31508011E0883F83C207B68022283F83D207B681B689F
S31508011E185B68FB607B681B689B68BB60FB6823F093
S31508011E287003FB603B681B68FA681343FB607B68B1
S31508011E381B68FA685A607B681B68194A934213D06B
S31508011E487B681B68B3F1804F0ED07B681B68154AFF
S31508011E58934209D07B681B68134A934204D07B686E
S31508011E681B68124A93420CD1BB6823F08003BB60F6
S31508011E783B685B68BA681343BB607B681B68BA68CA
S31508011E889A607B68012283F83D207B68002283F8E3
S31508011E983C20002318461437BD4680BC704700BF4E
S31508011EA8002C01400004004000080040000C0040D6
S31508011EB880B483B000AF786000BF0C37BD4680BCDC
S31508011EC8704780B483B000AF786000BF0C37BD4651
S31508011ED880BC704780B582B000AF78607B68002BFC
S31508011EE801D1012342E07B6893F84130DBB2002B2C
S31508011EF806D17B68002283F840207868FBF76CFCDA
S31508011F087B68242283F841207B681B68DA687B682A
S31508011F181B6822F40052DA60786800F0B5FF7B681E
S31508011F281B681A697B681B6822F490421A617B68E8
S31508011F381B685A697B681B6822F02A025A617B6802
S31508011F481B68DA687B681B6842F40052DA607B68AA
S31508011F5800225A647B68202283F841207B68202264
S31508011F6883F842207B6800225A63002318460837FB
S31508011F78BD4680BD80B58AB002AFF860B9603B60DE
S31508011F881346FB8000237B61FB6893F84130DBB27B
S31508011F98202B75D1BB68002B02D0FB88002B01D1F9
S31508011FA801236EE0FB6800225A64FB68212283F844
S31508011FB84120FBF7D9FD7861FB68FA889A84FB68A2
S31508011FC8FA88DA84FB689B68B3F5805F08D1FB68F1
S31508011FD81B69002B04D10023FB61BB68BB6103E0C5
S31508011FE8BB68FB610023BB612EE03B6800937B69F4
S31508011FF800228021F86800F0B9FC0346002B05D0B9
S31508012008FB68202283F8412003233AE0FB69002B69
S315080120180BD1BB691B881A46FB681B68C2F3080201
S315080120285A60BB690233BB6107E0FB691A78FB682A
S315080120381B685A60FB690133FB61FB68DB8C9BB241
S31508012048013B9AB2FB68DA84FB68DB8C9BB2002BEE
S31508012058CBD13B6800937B6900224021F86800F0E0
S3150801206885FC0346002B05D0FB68202283F841200E
S31508012078032306E0FB68202283F84120002300E0B9
S31508012088022318462037BD4680BD80B485B000AF07
S31508012098F860B9601346FB80FB6893F84130DBB2F8
S315080120A8202B21D1BB68002B02D0FB88002B01D13C
S315080120B801231AE0FB68BA681A62FB68FA889A84E7
S315080120C8FB68FA88DA84FB6800225A64FB682122CD
S315080120D883F84120FB681B68DA68FB681B6842F0CD
S315080120E88002DA60002300E0022318461437BD4649
S315080120F880BC704780B58CB000AFF860B9601346EC
S31508012108FB80FB6893F84230DBB2202B4AD1BB68C7
S31508012118002B02D0FB88002B01D1012343E0FB6881
S3150801212801221A63FB6800225A63FB881A46B968B2
S31508012138F86800F074FC034687F82F3097F82F30B3
S31508012148002B2CD1FB681B6B012B25D100233B6186
S31508012158FB681B681B683B61FB681B685B683B611E
S315080121683B69FB681B680C33BB61BB6953E8003FD5
S315080121787B617B6943F01003BB62FB681B680C3300
S31508012188BA6A7A623B62396A7A6A41E80023FB616C
S31508012198FB69002BE5D102E0012387F82F3097F870
S315080121A82F3000E0022318463037BD4680BD0000AF
S315080121B880B5A2B000AF78600123C7F884307B6880
S315080121C81B680C333B663B6E53E8003FFB65FB6DAA
S315080121D823F4F073C7F880307B681B680C33D7F88B
S315080121E88020FA66BB66B96EFA6E41E800237B66FB
S315080121F87B6E002BE3D17B681B681433FB64FB6C8D
S3150801220853E8003FBB64BB6C23F00103FB677B689B
S315080122181B681433FA6FBA657B65796DBA6D41E83F
S3150801222800233B653B6D002BE5D17B681B6B012BB6
S3150801223819D17B681B680C33BB63BB6B53E8003F3A
S315080122487B637B6B23F01003BB677B681B680C33C6
S31508012258BA6F7A643B64396C7A6C41E80023FB638C
S31508012268FB6B002BE5D17B689B6B002B0FD07B683A
S315080122781B685B6903F08003002B04D07B689B6BA2
S31508012288534A5A6303E07B689B6B00225A637B684F
S31508012298DB6B002B0FD07B681B685B6903F0400377
S315080122A8002B04D07B68DB6B4A4A5A6303E07B68D8
S315080122B8DB6B00225A637B681B685B6903F0800342
S315080122C8002B2DD07B681B6814337B627B6A53E825
S315080122D8003F3B623B6A23F080037B677B681B6888
S315080122E814337A6F3A63FB62F96A3A6B41E8002359
S315080122F8BB62BB6A002BE5D17B689B6B002B0FD0B1
S315080123087B689B6B1846FDF79DF90346002B04D09D
S315080123187B689B6B00225A6302E00023C7F8843066
S315080123287B681B685B6903F04003002B30D07B6828
S315080123381B6814333B613B6953E8003FFB60FB6844
S3150801234823F040033B677B681B6814333A6FFA61CD
S31508012358BB61B969FA6941E800237B617B69002B8E
S31508012368E5D17B68DB6B002B12D07B68DB6B1846E3
S31508012378FDF768F90346002B07D07B68DB6B00225B
S315080123885A630123C7F8843002E00023C7F884306A
S31508012398D7F88430012B16D17B680022DA847B684A
S315080123A80022DA857B6800225A647B68202283F832
S315080123B841207B68202283F842207B6800221A6321
S315080123C8786800F0ADFA002318468837BD4680BDFF
S315080123D8852B0108E52B010880B5BAB000AF7860EE
S315080123E87B681B681B68C7F8E4307B681B68DB6871
S315080123F8C7F8E0307B681B685B69C7F8DC300023DF
S31508012408C7F8D8300023C7F8D430D7F8E43003F032
S315080124180F03C7F8D830D7F8D830002B0FD1D7F81B
S31508012428E43003F02003002B09D0D7F8E03003F095
S315080124382003002B03D0786800F067FC5BE2D7F825
S31508012448D830002B00F0DE80D7F8DC3003F0010322
S31508012458002B06D1D7F8E03003F49073002B00F06F
S31508012468D180D7F8E43003F00103002B0BD0D7F855
S31508012478E03003F48073002B05D07B685B6C43F06E
S3150801248801027B685A64D7F8E43003F00403002B89
S315080124980BD0D7F8DC3003F00103002B05D07B6895
S315080124A85B6C43F002027B685A64D7F8E43003F0A0
S315080124B80203002B0BD0D7F8DC3003F00103002BFD
S315080124C805D07B685B6C43F004027B685A64D7F8CD
S315080124D8E43003F00803002B11D0D7F8E03003F0F5
S315080124E82003002B05D1D7F8DC3003F00103002BB4
S315080124F805D07B685B6C43F008027B685A647B6885
S315080125085B6C002B00F0F281D7F8E43003F0200366
S31508012518002B08D0D7F8E03003F02003002B02D0AF
S31508012528786800F0F2FB7B681B685B6903F0400377
S31508012538002B14BF01230023DBB2C7F8D4307B680C
S315080125485B6C03F00803002B03D1D7F8D430002BB2
S315080125584FD0786800F09CFA7B681B685B6903F0C2
S315080125684003002B41D07B681B681433C7F89C309D
S31508012578D7F89C3053E8003FC7F89830D7F8983011
S3150801258823F04003C7F8D0307B681B681433D7F8A3
S31508012598D020C7F8A820C7F8A430D7F8A410D7F8C8
S315080125A8A82041E80023C7F8A030D7F8A030002BA7
S315080125B8D9D17B68DB6B002B13D07B68DB6B7E4A32
S315080125C85A637B68DB6B1846FDF73CF80346002B14
S315080125D816D07B68DB6B5B6B7A68D26B10469847BB
S315080125E80EE0786800F093F90AE0786800F08FF948
S315080125F806E0786800F08BF97B6800225A6475E171
S3150801260800BF73E17B681B6B012B40F04F81D7F83C
S31508012618E43003F01003002B00F04881D7F8E030C6
S3150801262803F01003002B00F041810023BB607B688F
S315080126381B681B68BB607B681B685B68BB60BB68FB
S315080126487B681B685B6903F04003002B00F0B680C2
S315080126587B68DB6B1B685B68A7F8BE30B7F8BE30CA
S31508012668002B00F045817B689B8DB7F8BE209A42FE
S3150801267880F03E817B68B7F8BE20DA857B68DB6B1C
S315080126889B69202B00F088807B681B680C33C7F888
S315080126988830D7F8883053E8003FC7F88430D7F828
S315080126A8843023F48073C7F8B8307B681B680C3309
S315080126B8D7F8B820C7F89420C7F89030D7F89010FB
S315080126C8D7F8942041E80023C7F88C30D7F88C301E
S315080126D8002BD9D17B681B6814337B677B6F53E85A
S315080126E8003F3B673B6F23F00103C7F8B4307B68AB
S315080126F81B681433D7F8B420C7F88020FB67F96F2D
S31508012708D7F8802041E80023BB67BB6F002BE1D1CE
S315080127187B681B6814333B663B6E53E8003FFB65D1
S31508012728FB6D23F04003C7F8B0307B681B68143388
S31508012738D7F8B020FA66BB66B96EFA6E41E8002387
S315080127487B667B6E002BE3D17B68202283F84220C7
S315080127587B6800221A637B681B680C33FB64FB6C75
S3150801276853E8003FBB64BB6C23F01003C7F8AC30D1
S315080127787B681B680C33D7F8AC20BA657B65796D1D
S31508012788BA6D41E800233B653B6D002BE3D17B68B5
S31508012798DB6B1846FCF71BFF7B6802225A637B68CA
S315080127A89A8D7B68DB8D9BB2D31A9BB219467868DA
S315080127B8F9F7E0FF9CE000BF5D2B01087B689A8D5D
S315080127C87B68DB8D9BB2D31AA7F8CE307B68DB8D85
S315080127D89BB2002B00F08E80B7F8CE30002B00F0A4
S315080127E889807B681B680C33BB63BB6B53E8003F66
S315080127F87B637B6B23F49073C7F8C8307B681B68C7
S315080128080C33D7F8C8207A643B64396C7A6C41E88A
S315080128180023FB63FB6B002BE3D17B681B6814332E
S315080128287B627B6A53E8003F3B623B6A23F00103FC
S31508012838C7F8C4307B681B681433D7F8C4203A63D1
S31508012848FB62F96A3A6B41E80023BB62BB6A002B53
S31508012858E3D17B68202283F842207B6800221A6329
S315080128687B681B680C333B613B6953E8003FFB6097
S31508012878FB6823F01003C7F8C0307B681B680C3364
S31508012888D7F8C020FA61BB61B969FA6941E800233A
S315080128987B617B69002BE3D17B6802225A63B7F80F
S315080128A8CE3019467868F9F765FF23E0D7F8E4309A
S315080128B803F08003002B09D0D7F8E03003F0800332
S315080128C8002B03D0786800F0B9F914E0D7F8E4309A
S315080128D803F04003002B0ED0D7F8E03003F040038D
S315080128E8002B08D0786800F0F8F904E000BF02E088
S315080128F800BF00E000BFE837BD4680BD80B483B09D
S3150801290800AF786000BF0C37BD4680BC704780B4FD
S3150801291883B000AF786000BF0C37BD4680BC7047EE
S3150801292880B483B000AF786000BF0C37BD4680BC61
S31508012938704780B485B000AF78600023FB60002338
S31508012948BB607B6893F84130DBB2FB607B6893F820
S315080129584230DBB2BB60FB68DAB2BB68DBB2134351
S31508012968DBB218461437BD4680BC704780B586B0B9
S3150801297800AFF860B9603B601346FB713BE03B6A00
S31508012988B3F1FF3F37D0FBF7EFF802463B68D31A96
S315080129983A6A9A4202D33B6A002B01D103233AE0E9
S315080129A8FB681B68DB6803F00403002B23D0BB68AC
S315080129B8802B20D0BB68402B1DD0FB681B681B6881
S315080129C803F00803082B16D100237B61FB681B68F3
S315080129D81B687B61FB681B685B687B617B69F868B8
S315080129E800F056F8FB6808225A64FB68002283F847
S315080129F8402001230FE0FB681B681A68BB6813406F
S31508012A08BA689A420CBF01230023DBB21A46FB793E
S31508012A189A42B4D0002318461837BD4680BD80B4FB
S31508012A2885B000AFF860B9601346FB80FB68BA68E1
S31508012A389A62FB68FA889A85FB68FA88DA85FB68D8
S31508012A4800225A64FB68222283F84220FB681B6924
S31508012A58002B07D0FB681B68DA68FB681B6842F419
S31508012A688072DA60FB681B685A69FB681B6842F062
S31508012A7801025A61FB681B68DA68FB681B6842F041
S31508012A882002DA60002318461437BD4680BC704711
S31508012A9880B495B000AF78607B681B680C337B639C
S31508012AA87B6B53E8003F3B633B6B23F49073FB64F2
S31508012AB87B681B680C33FA6C3A64FB63F96B3A6CEE
S31508012AC841E80023BB63BB6B002BE5D17B681B6818
S31508012AD814333B623B6A53E8003FFB61FB6923F009
S31508012AE80103BB647B681B681433BA6CFA62BB6260
S31508012AF8B96AFA6A41E800237B627B6A002BE5D149
S31508012B087B681B6B012B19D17B681B680C33FB602F
S31508012B18FB6853E8003FBB60BB6823F010037B647E
S31508012B287B681B680C337A6CBA617B617969BA6907
S31508012B3841E800233B613B69002BE5D17B682022EC
S31508012B4883F842207B6800221A6300BF5437BD46C2
S31508012B5880BC704780B584B000AF78607B685B6AD3
S31508012B68FB60FB680022DA85FB680022DA84F868CC
S31508012B78FFF7CDFE00BF1037BD4680BD80B584B0CE
S31508012B8800AF78607B685B6AFB60FB689B6B002219
S31508012B985A63FB68DB6B002B04D0FB68DB6B5B6B4A
S31508012BA8002B17D1FB680022DA84FB680022DA8534
S31508012BB8FB6800225A64FB68202283F84120FB68D7
S31508012BC8202283F84220FB6800221A63F868FFF777
S31508012BD8A7FE00E000BF1037BD4680BD80B584B0AA
S31508012BE800AF78607B685B6AFB60FB68DB6B002279
S31508012BF85A63FB689B6B002B04D0FB689B6B5B6B6A
S31508012C08002B17D1FB680022DA84FB680022DA85D3
S31508012C18FB6800225A64FB68202283F84120FB6876
S31508012C28202283F84220FB6800221A63F868FFF716
S31508012C3877FE00E000BF1037BD4680BD80B485B079
S31508012C4800AF78607B6893F84130DBB2212B3ED11F
S31508012C587B689B68B3F5805F14D17B681B69002B79
S31508012C6810D17B681B6AFB60FB681B881A467B6860
S31508012C781B68C2F308025A607B681B6A9A1C7B6840
S31508012C881A6208E07B681B6A591C7A6811621A7805
S31508012C987B681B685A607B68DB8C9BB2013B9BB2DD
S31508012CA87A681946D184002B0FD17B681B68DA68C4
S31508012CB87B681B6822F08002DA607B681B68DA6821
S31508012CC87B681B6842F04002DA60002300E00223B1
S31508012CD818461437BD4680BC704780B582B000AF28
S31508012CE878607B681B68DA687B681B6822F0400293
S31508012CF8DA607B68202283F841207868F9F79AFD1B
S31508012D08002318460837BD4680BD80B58CB000AF8C
S31508012D1878607B6893F84230DBB2222B40F0AE80AC
S31508012D287B689B68B3F5805F17D17B681B69002BA5
S31508012D3813D10023FB627B689B6ABB627B681B68AD
S31508012D485B689BB2C3F308039AB2BB6A1A807B68AD
S31508012D589B6A9A1C7B689A6226E07B689B6AFB6277
S31508012D680023BB627B689B68B3F5805F07D07B68E5
S31508012D789B68002B0AD17B681B69002B06D17B68E7
S31508012D881B685B68DAB2FB6A1A7008E07B681B681D
S31508012D985B68DBB203F07F03DAB2FB6A1A707B68F9
S31508012DA89B6A5A1C7B689A627B68DB8D9BB2013BDE
S31508012DB89BB27A681946D185002B5DD17B681B6859
S31508012DC8DA687B681B6822F02002DA607B681B6870
S31508012DD8DA687B681B6822F48072DA607B681B688C
S31508012DE85A697B681B6822F001025A617B682022AE
S31508012DF883F842207B6800225A637B681B6B012B88
S31508012E0835D17B6800221A637B681B680C337B61A2
S31508012E187B6953E8003F3B613B6923F010037B62FA
S31508012E287B681B680C337A6A3A62FB61F9693A6A04
S31508012E3841E80023BB61BB69002BE5D17B681B68A8
S31508012E481B6803F01003102B0AD10023FB607B686B
S31508012E581B681B68FB607B681B685B68FB60FB6813
S31508012E687B689B8D19467868F9F784FC02E07868CF
S31508012E78FFF744FD002302E0002300E00223184679
S31508012E883037BD4680BD000080B584B000AF786094
S31508012E987B681B681B6923F440517B68DA687B6881
S31508012EA81B680A431A617B689A687B681B691A4317
S31508012EB87B685B691343BB607B681B68DB6823F423
S31508012EC8B05323F00C037A681268B9680B43D360C8
S31508012ED87B681B685B6923F440717B689A697B6820
S31508012EE81B680A435A617B681B682C4A934203D1BB
S31508012EF8FDF71AFCF86002E0FDF702FCF860FA68CB
S31508012F0813469B0013449A001A447B685B689B0026
S31508012F18B2FBF3F3224AA2FB03235B091901FA68F8
S31508012F2813469B0013449A001A447B685B689B0006
S31508012F38B2FBF3F21A4BA3FB02035B09642000FBFD
S31508012F4803F3D31A1B013233154AA2FB03235B0980
S31508012F5803F0F0031944FA6813469B0013449A00D0
S31508012F681A447B685B689B00B2FBF3F20C4BA3FB24
S31508012F7802035B09642000FB03F3D31A1B013233EE
S31508012F88074AA2FB03235B0903F00F027B681B6848
S31508012F980A449A6000BF1037BD4680BD0038014013
S31508012FA81F85EB51002B2DE9F0471D46BBBF03F1E1
S31508012FB800431D4600232D2388B01446B8BF14467E
S31508012FC8129A109E1370149BDDF84CA023F0200862
S31508012FD8B8F1460F05D0B8F1450F00D101360223DD
S31508012FE800E0032307AA049206AACDE902A2CDE9BD
S31508012FF8003622462B4600F03BFEB8F1470F074636
S3150801300819D1119BDB070ED500EB0609002200230F
S3150801301820462946F5F730FD08B1CDF81C9030222F
S31508013028079B4B451ED33846079B159ADB1B13602E
S3150801303808B0BDE8F087B8F1460F00EB0609E5D1F7
S315080130480378302B0AD10022002320462946F5F7B2
S3150801305813FD18B9C6F10106CAF80060DAF8003096
S315080130689944D3E7591C07911A70D9E7F7B5002986
S31508013078B6BF2D232B23494209290270437029DD3E
S315080130880DF107031D460A27B1FBF7F61A4607FB92
S315080130981614303402F8014C0C46632C314603F1F8
S315080130A8FF33F1DC3031941E03F8011C2346411C19
S315080130B8AB420AD30DF109039B1AAC4288BF002318
S315080130C802330344181A03B0F0BD13F8016B01F86B
S315080130D8016FEDE7302330318370C170031DF1E7C5
S315080130E82DE9F04F91B00C46DDF8688016461F4663
S315080130F8054600F0F7FC036818460893F5F790F8B3
S3150801310800230E93D8F800300990073323F00703F4
S3150801311803F1080294F818A0D4F800B0C8F80020FA
S31508013128D3E9008929F000430B93CDF828804FF09D
S31508013138FF32DDE90A01C4E912899C4BF5F7CEFC91
S3150801314870BBDDE90A014FF0FF32984BF5F7A8FC89
S3150801315830BB0022002340464946F5F797FC10B1D3
S315080131682D2384F84330924A924BBAF1470F8CBF04
S315080131789046984603234FF0000923612BF0040370
S31508013188236033462146284600970FAA00F0D4F94A
S31508013198013040F090804FF0FF3011B0BDE8F08F54
S315080131A842464B4640464946F5F798FC48B14B46D0
S315080131B8002BB8BF2D23804AB8BF84F843307F4B0C
S315080131C8D3E763680AF0DF015A1C3FD10623636017
S315080131D800224BF48063236006920EAACDE904A265
S315080131E80DAA03920DF13302CDE90132636842460D
S315080131F8009328464B460A91FFF7D4FE0A9980465A
S3150801320847290D9928D1C81C02DB6368994240DD14
S31508013218AAF1020A5FFA8AFA5246013904F15000FC
S315080132280D91FFF723FF0E9A81461318012A236188
S3150801323802DC2268D20701D5013323619DF83330B0
S31508013248002B9ED02D2384F843309AE74729BFD10E
S31508013258002BBDD10123BAE7BAF1650FDCD9BAF15A
S31508013268660F18D1002963680BDD216113B9226835
S31508013278D00702D501330B4423614FF00009A16534
S31508013288DCE713B92268D20701D50233F4E701232B
S31508013298F2E74FF0670A0E9B994205DB236821611D
S315080132A8D807EAD54B1CE7E70029CCBF0122C1F1AB
S315080132B802021344E0E723685A0507D423694246FC
S315080132C831462846B84701302BD164E7BAF1650F6C
S315080132D840F2DC80D4E9120100220023F5F7CCFB81
S315080132E8002833D0012331462846354AB8470130E4
S315080132F83FF451AFDDE90D38434502DB2368D807AA
S315080133080FD5DDE9082331462846B84701303FF489
S3150801331842AF4FF0000908F1FF3804F11A0AC84507
S3150801332809DC23689B0700F10281E0680F9B984234
S31508013338B8BF184631E70123524631462846B847E9
S3150801334801303FF428AF09F10109E8E70D9B002B85
S3150801335838DC012331462846194AB84701303FF473
S315080133681AAFDDE90D3959EA030302D12368D907EA
S31508013378D7D5DDE9082331462846B84701303FF451
S315080133880AAF4FF0000A04F11A0B0D9B5B4253452D
S3150801339801DC4B4693E701235A4631462846B84786
S315080133A801303FF4F8AE0AF1010AEEE7FFFFEF7FB5
S315080133B84C61010848610108546101085061010816
S315080133C858610108A36DDDF838A05345A8BF5346CF
S315080133D8002B994636DC4FF0000B29EAE97904F106
S315080133E81A02A36D0A93A3EB09035B4531DC0D9B0E
S315080133F89A453ADC2368DA0737D40D9BAAEB030901
S315080134080A9BAAEB03039945A8BF9946B9F1000F88
S3150801341833DC4FF0000829EAE97904F11A0B0D9B08
S31508013428AAEB0303A3EB090343457FF77AAF012305
S315080134385A4631462846B84701303FF4ACAE08F13A
S315080134480108ECE7424631462846B8470130C2D159
S31508013458A1E60123314628460A92B84701303FF4C6
S315080134689AAE0A9A0BF1010BBBE73146DDE9082347
S315080134782846B8470130C0D18DE60A9A4B463146E7
S3150801348828464244B8470130C3D184E6DDF838A056
S31508013498BAF1010F01DCDB0736D50123424631466D
S315080134A82846B84701303FF476AEDDE908233146A8
S315080134B82846B84701303FF46EAED4E91201002216
S315080134C800230AF1FF3AF5F7D7FAC0B9534608F1C6
S315080134D8010231462846B84701300CD15BE601237B
S315080134E85A4631462846B84701303FF454AE08F1E2
S315080134F80108D045F3DB4B4604F15002E0E64FF0EC
S31508013508000804F11A0BF4E701234246E1E701230F
S315080135184A4631462846B84701303FF43CAE08F1D9
S315080135280108E3680F995B1A4345F0DCFDE64FF09D
S31508013538000804F11909F4E72DE9F04716469846F3
S315080135488A680B6907469342B8BF1346336091F8F0
S3150801355843200C46DDF820900AB10133336023680D
S31508013568990642BF336802333360256815F00605A4
S3150801357806D104F1190AE36832689B1AAB422BDCB7
S3150801358894F843302268003B18BF0123920630D4C9
S315080135984146384604F14302C847013023D0236817
S315080135A8226903F00603042B14BF002533684FF07C
S315080135B8000608BFE56804F11A0408BFED1A54F8AD
S315080135C8123C08BF25EAE5759342C4BF9B1AED1854
S315080135D8B5421AD1002008E0012352464146384629
S315080135E8C847013003D14FF0FF30BDE8F0870135F0
S315080135F8C1E73020E11881F843005A1C94F84510B0
S315080136082244023382F84310C2E70123224641467F
S315080136183846C8470130E6D00136D9E72DE9FF47CC
S315080136280F7E9146782F80460C469A460C9E01F1E4
S31508013638430207D8622F0AD8002F00F0D180582FE5
S3150801364800F0B88004F1420684F842703AE0A7F11E
S315080136586303152BF6D801A151F823F0BD360108E5
S31508013668D13601084D3601084D3601084D3601088F
S315080136784D360108D13601084D3601084D3601087F
S315080136884D3601084D360108CF370108FB360108C2
S31508013698893701084D3601084D360108F137010801
S315080136A84D360108FB3601084D3601084D36010825
S315080136B89137010833681A1D1B68326004F14206FE
S315080136C884F8423001239CE033682068191D31606B
S315080136D8060601D51D6803E04506FBD5B3F9005072
S315080136E8002D03DA2D236D4284F843300A235848FE
S315080136F811E021683368080653F8045B02D44906C1
S3150801370848BFADB26F2F336014BF0A230823504848
S31508013718002184F843106668002EA66005DB216837
S315080137282E4321F0040121604BD01646B5FBF3F16F
S3150801373803FB1157C75D06F8017D2F46BB420D46A7
S31508013748F4D9082B0BD12368DF0708D523696168E3
S315080137589942DEBF302306F8013C06F1FF36921B73
S3150801376822614B4621464046CDF800A003AAFFF739
S31508013778E3FE01304AD14FF0FF3004B0BDE8F087C7
S31508013788236843F0200323607827324884F8457074
S31508013798236831681F0651F8045B02D45F0648BFDF
S315080137A8ADB23160D90744BF43F0200323601DB188
S315080137B81023ADE72648E9E7236823F020032360A9
S315080137C8F6E71646BDE733682568181D616930604E
S315080137D82E061B6801D5196002E06806FBD5198013
S315080137E8002316462361BCE7336800211A1D326097
S315080137F81E686268304600F079F908B1801B606076
S3150801380863682361002384F84330AAE732464946A8
S3150801381840462369D0470130ADD023689B0713D4A6
S31508013828E068039B9842B8BF1846A6E701233246C3
S3150801383849464046D04701309DD00135E36803998A
S315080138485B1AAB42F2DCEBE7002504F11906F5E74A
S315080138585A6101086B610108002310B50446C0E9DD
S315080138680033C0E90433836081814366C281836179
S31508013878194608225C3000F0FFF80D4B2462636292
S315080138880C4BA3620C4BE3620C4B23630C4B9C4217
S3150801389806D003F16802944202D0D0339C4205D17E
S315080138A804F15800BDE8104000F018B910BD00BF72
S315080138B801570108235701085B5701087F57010873
S315080138C8E0110020024A0349034800F0A5B800BFE1
S315080138D878000020A54F01088800002041680C4B94
S315080138E810B59942044601D001F058FBA168094B65
S315080138F8994202D0204601F051FBE168064B9942EC
S3150801390804D02046BDE8104001F048BB10BD00BFF1
S31508013918E011002048120020B012002010B50B4B08
S315080139280B4C0C4A20461A6004210022FFF794FF23
S3150801393804F1680001220921FFF78EFF04F1D0007E
S315080139480222BDE810401221FFF786BF181300208E
S31508013958E0110020CD380108014800F0C0B800BFC1
S315080139681D130020014800F0BBB800BF1D13002035
S3150801397810B50446FFF7F0FF236A1BB1BDE81040EE
S31508013988FFF7F0BF044B2362044B1B68002BF5D1E4
S31508013998FFF7C4FFF2E700BFE5380108181300204E
S315080139A830B51446002C05461A469BB005DA8B2312
S315080139B803604FF0FF301BB030BD4FF40273ADF80A
S315080139C80C304FF0000319930CBF234604F1FF335B
S315080139D8029305934FF6FF7300910491ADF80E30E3
S315080139E869461E9B00F074FF431CBCBF8B232B60E2
S315080139F8002CE0D00022009B1A70DCE707B500937B
S31508013A0813460A46014603480068FFF7C9FF03B08B
S31508013A185DF804FB840000202DE9F843074688462B
S31508013A2814460026D4E90195B9F1010905D5246892
S31508013A38002CF7D13046BDE8F883AB89012B07D9A5
S31508013A48B5F90E30013303D029463846C04706432F
S31508013A586835E9E70FB407B5064904AB086853F8AA
S31508013A68042B8168019301F057F803B05DF804EB5C
S31508013A7804B070478400002003460244934200D1EB
S31508013A88704703F8011BF9E7014B1868704700BF2F
S31508013A988400002070B500260C4D0D4C641BA4103B
S31508013AA8A64209D102F004F900260A4D0A4C641BFC
S31508013AB8A410A64205D170BD55F8043B98470136AE
S31508013AC8EEE755F8043B98470136F2E7C46401085E
S31508013AD8C4640108C4640108C864010870477047CA
S31508013AE87047000000487047C4010020034610B516
S31508013AF8C9B202449342184601D1002003E004786A
S31508013B0801338C42F6D110BD0A44914200F1FF33C4
S31508013B1800D1704710B511F8014B914203F8014FCE
S31508013B28F9D110BD1FB514461A46094B05461B6837
S31508013B38D8684CB1074BCDE9013400912B460649A3
S31508013B4801F01EFE01F0E4FF044B1C46F3E700BF33
S31508013B58840000207C61010889610108B7610108B0
S31508013B682DE9F74F03690C690746A3427EDB013C39
S31508013B78A30000F1140501F11408009305EB840369
S31508013B88019358F8243055F8242001339A42B2FB98
S31508013B98F3F608EB84092ED34FF0000AC446AE465D
S31508013BA8D3465CF8043B98B206FB00A01B0C020C32
S31508013BB806FB0323DEF8002080B292B2121A5A4491
S31508013BC8DEF800004FEA134A9BB2C3EB224303EB24
S31508013BD8104392B242EA0342E1454FEA234B4EF8B3
S31508013BE8042BDED2009BEB582BB9019B043B9D4263
S31508013BF81A462FD33C61384601F076FC002825DBA6
S31508013C082946002058F8042BD1F800C01FFA82FE6D
S31508013C181FFA8CF3A3EB0E030344120CC2EB2342DF
S31508013C2802EB1C429BB243EA0243C1454FEA2240D2
S31508013C3841F8043BE6D255F8242005EB840322B95A
S31508013C48043B9D421A460BD33C610136304603B004
S31508013C58BDE8F08F1268043B002ACBD1013CC6E7C0
S31508013C681268043B002AEFD1013CEAE70020EEE797
S31508013C782DE9F04F14461D46C76997B08146CDE927
S31508013C880645239E7FB9102001F05EF80246C9F859
S31508013C981C0020B9EF21AC4BAC48FFF743FFC0E93C
S31508013CA801770760C760D9F81C30196859B15A688D
S31508013CB8012393404A608B60484601F0E3F90022E4
S31508013CC8D9F81C301A602B1EAFBF0023012223F036
S31508013CD800430793A8BF3360DDF81C809C4BB8BF27
S31508013CE8326033EA080312D142F20F73229A13603B
S31508013CF8C8F31303234300F05E85249BDFF854A217
S31508013D08002B00F060850AF1030300F05ABDDDE9CE
S31508013D180623CDE90C23DDE90C0100220023F4F77B
S31508013D28ABFE074658B10123229A1360249B13B1A7
S31508013D38894B249A1360DFF824A200F044BD14AB1A
S31508013D48019315AB00934846DDE90C2301F07CFC89
S31508013D58C8F30A560390002E78D0DDE90C010D9BAD
S31508013D68A6F2FF36C3F3130343F07F5343F4401314
S31508013D781297194600227A4BF4F75EFA6CA3D3E92F
S31508013D880023F4F711FC6CA3D3E90023F4F756FAD8
S31508013D98044630460D46F4F79DFB69A3D3E900238B
S31508013DA8F4F702FC02460B4620462946F4F746FA7A
S31508013DB804460D46F4F7A8FE0022074600232046C6
S31508013DC82946F4F763FE40B13846F4F783FB2246E1
S31508013DD82B46F4F751FE00B9013F162F54D8DDE9F1
S31508013DE80C01604B03EBC703D3E90023F4F74EFE36
S31508013DF800284BD00023013F0F93149B9B1B5A1E87
S31508013E0849BFC3F10103002304930023099254BF50
S31508013E1804930993002F3BDB099B0E973B440993AF
S31508013E2800230A93209B092B65D8052BC4BF043B9D
S31508013E382093209BC8BF0024A3F10203D8BF0124FD
S31508013E48032B64D8DFE803F05355382CDDE91463EE
S31508013E581E4406F23243202BC1BFC3F1400308FAB8
S31508013E6803F806F2124324FA03F3D6BFC3F1200373
S31508013E7848EA030004FA03F0F4F71CFB0122A1F14E
S31508013E88F873013E129274E70123B5E70F90B4E778
S31508013E98049BDB1B04937B420A9300230E93C1E719
S31508013EA801230B93219B07EB030B0BF10103012B51
S31508013EB80893B8BF012306E001230B93219B002B26
S31508013EC828DD9B46089300210422D9F81C0002F133
S31508013ED814059D4226D94160484601F093F8824661
S31508013EE8002843D1024640F2AF111F4BD4E60023FE
S31508013EF8E3E70023D5E7012400230B9420934FF029
S31508013F08FF3B00221223CDF820B02192DBE70123DB
S31508013F180B93F4E74FF0010B5B46CDF820B0CDF8CB
S31508013F2884B0D0E701315200D1E700BFAFF3008072
S31508013F3861436F63A787D23FB3C8608B288AC63F98
S31508013F48FB799F501344D33FC5610108DC61010819
S31508013F580000F07FC161010859610108586101082B
S31508013F680000F83FF062010834620108D9F81C30EC
S31508013F781860089B0E2B00F2A180002C00F09E8089
S31508013F88002F33DD9C4B07F00F0203EBC203F8053C
S31508013F98D3E90034CDE910344FEA271416D5DDE9FB
S31508013FA80C01964B0326D3E90823F4F727FCCDE938
S31508013FB8060104F00F04914D54B9DDE91023DDE932
S31508013FC80601F4F71BFCCDE9060128E00226F2E70B
S31508013FD8E10708D5DDE91001D5E90023F4F7E4FA84
S31508013FE8CDE91001013664100835E5E700F0AF8020
S31508013FF8DDE90C017C42804B04F00F0203EBC20396
S31508014008D3E90023F4F7D0FA02260023CDE90601FD
S315080140187A4D2411002C40F08F80002BD3D1DDE98D
S3150801402806450F9B002B00F094800022204629465E
S31508014038734BF4F72BFD002800F08B80089B002BA7
S3150801404800F08780BBF1000F34DD2046002229469F
S315080140586C4BF4F7A9FA5C46CDE9060107F1FF3876
S3150801406801363046F4F736FADDE90623F4F79CFA01
S315080140780022654BF4F7E2F80546A1F15076002CC3
S315080140886AD1DDE906010022604BF4F7D5F8024644
S315080140980B46CDE906232A463346F4F715FD0028CB
S315080140A840F09882DDE906012A4606F10043F4F74D
S315080140B8EDFC38BBDDE90C34CDE90634159B002B3C
S315080140C8C0F257810E2F00F354814B4B03EBC703FC
S315080140D8D3E90034CDE90434219B002B80F2E5802D
S315080140E8089B002B00F3E1800CD1DDE904010022CD
S315080140F8464BF4F759FADDE90623F4F7DBFC002801
S3150801410800F0668200242546219B56466FEA030875
S3150801411800272146484600F0B5FF002D00F0BD806E
S315080141282FB1AF4203D03946484600F0ABFF2946BE
S31508014138484600F0A7FFB0E0E20705D5D5E9002310
S31508014148F4F732FA012301366410083562E70226C4
S3150801415865E7B846089C84E7274B0B9903EBC40324
S3150801416853E902235444002954D000202849F4F776
S3150801417845FB33462A46F4F75FF85646CDE910015A
S31508014188DDE90601F4F7C0FC0546F4F7A3F902468A
S315080141980B46DDE90601F4F74FF802460B463035BA
S315080141A8CDE90623DDE9102306F8015BF4F76EFC71
S315080141B8002872D1DDE9062300201149F4F73CF8F5
S315080141C8DDE91023F4F762FC002840F0B480A64222
S315080141D83FF470AFDDE9100100220A4BF4F7E4F960
S315080141E80022CDE91001DDE90601064BF4F7DCF9F1
S315080141F8CDE90601C4E700BFF0620108C8620108F3
S315080142080000F03F0000244000001C400000144054
S315080142180000E03F31462846F4F7C6F95646CDE987
S3150801422810011394DDE90601F4F76EFC0546F4F767
S3150801423851F902460B46DDE90601F3F7FDFF024689
S315080142480B46303506F8015BA642CDE906234FF041
S31508014258000224D1DDE91001AE4BF3F7EFFF024660
S315080142680B46DDE90601F4F72FFC002863D1DDE9E1
S3150801427810230020A749F3F7DFFF02460B46DDE9BD
S315080142880601F4F703FC00283FF414AF139E731EC6
S31508014298139316F8013C302BF8D047463BE09E4B62
S315080142A8F4F782F9CDE90601BCE75646DDE9064584
S315080142B8DDE9042320462946F4F7A0FAF4F724FC95
S315080142C88046F4F707F9DDE90423F4F76DF90246A0
S315080142D80B4620462946F3F7AFFF08F13004089D37
S315080142E806F8014BA6EB0A04A54202460B4633D14A
S315080142F8F3F7A4FFDDE9042304460D46F4F7E4FBC6
S31508014308C0B9DDE9042320462946F4F7B5FB10B1FF
S3150801431818F0010F0ED14846039900F0B3FE0023A1
S315080143283370229B01371F60249B002B00F04B82B8
S315080143381E6048E2B84633461E4613F8012D392A47
S3150801434806D19A45F8D1302208F101088AF80020E1
S315080143581A7801321A70A0E700226F4BF4F724F98C
S315080143680022002304460D46F4F786FB00289FD051
S31508014378D1E70B9A002A00F0EA80209A012A00F36D
S31508014388CD80129A002A00F0C18003F233430A9CB1
S31508014398049E049A01211A440492099A48461A4421
S315080143A8099200F023FF054666B1099B002B09DD32
S315080143B8B342A8BF3346049AF61AD21A0492099A3E
S315080143C8D31A09930A9B0BB30B9B002B00F0C680E3
S315080143D8002C00F0C08029462246484600F0BEFF58
S315080143E8039A01460546484600F016FF0399804692
S315080143F8484600F047FE0A9B1B1B0A9300F0B1804A
S3150801440841460A9A484600F0A9FF03900121484601
S3150801441800F0ECFE0E9B0446002B00F0D8811A46E4
S315080144280146484600F09AFF209B0446012B00F3F3
S315080144389F80069B002B40F09780079BC3F31303C5
S31508014448002B40F09380079B23F000431B0D1B05A7
S3150801445833B1049B01330493099B0133099301235F
S315080144680A930E9B002B00F0B881236904EB83039A
S31508014478186900F06FFEC0F12000099B184410F076
S315080144881F0000F08280C0F12003042B73DD049B12
S31508014498C0F11C0003440493099B06440344099389
S315080144A8049B002B05DD1A464846039900F0B0FF20
S315080144B80390099B002B05DD21461A46484600F05C
S315080144C8A7FF04460F9B002B61D02146039801F0EC
S315080144D80BF800285BDA00230A224846039900F0FC
S315080144E8F3FD0B9B07F1FF380390002B00F077814A
S315080144F8294600230A22484600F0E6FDBBF1000FCB
S3150801450805466FDC209B022B49DC6BE0149BC3F143
S3150801451836033CE70000E03F00002440089B5C1E88
S315080145280A9BA34209DB1C1B089B002BBFF630AF6D
S31508014538049B089A9E1A00232BE70A9B0E9AE31AEC
S315080145481A440A94049E0024089B0E9221E70A9CA1
S31508014558049E0B9D28E7DDF80C8051E70A9A039912
S3150801456850E7CDF80C8051E7002379E7069B77E7F2
S3150801457800230A9379E793D0049A1C331A440492C0
S31508014588099A1E441A4409928AE70346F4E7089BDE
S31508014598B846002B20DC9B46209B022B1EDDBBF16F
S315080145A8000F7FF4B1AD21465B460522484600F067
S315080145B88BFD01460446039800F096FF00287FF70D
S315080145C8A3AD5646312308F1010806F8013B9FE5D4
S315080145D8B846089C2546F4E7DDF820B00B9B002B66
S315080145E800F00181002E05DD29463246484600F0CD
S315080145F80FFF05460A9B002B5CD04846696800F000
S3150801460801FD064628B9024640F2EF21804BFFF71D
S3150801461843BB2A6905F10C01023292000C30FFF7F7
S3150801462873FA01223146484600F0F2FE2F4605463E
S315080146380AF1010304930AEB0B030A93069B03F099
S3150801464801030993049B2146039803F1FF3BFFF7EE
S3150801465887FA034639463033069003980B9300F0D8
S3150801466843FF2A4608902146484600F059FFC26882
S3150801467806460B9B02BB0146039800F035FF024626
S315080146880B9B31464846CDE90B3200F0FBFC209BD3
S315080146980C9A049E42EA0301099B19430B9B0DD107
S315080146A8392B27D0089A002A01DD069B31338BF866
S315080146B800302EE52846B9E70122E2E708990029DC
S315080146C804DB209801430998014320D1002AEEDD2D
S315080146D8012203994846049300F09AFE214603905D
S315080146E800F002FF0028049B02DCE0D1DA07DED5D8
S315080146F8392BDAD139238BF8003033461E4616F89A
S31508014708012C013B392A4ED001321A7001E5002ADB
S3150801471803DD392BEED00133C9E7049A0A9902F861
S31508014728013C8A4228D000230A220399484600F008
S31508014738CBFCAF4203904FF000034FF00A0239460B
S31508014748484607D100F0C0FC07460546049B0133D5
S31508014758049377E700F0B8FC2946074600230A229E
S31508014768484600F0B1FC0546F0E7BBF1000FCCBF9F
S315080147785E460126002756440122039948460493B2
S3150801478800F046FE2146039000F0AEFE0028B4DC90
S3150801479802D1049BDB07B0D433461E4613F8012D14
S315080147A8302AFAD0B5E49A45A8D1312308F1010887
S315080147B88AF80030ADE4249BDFF858A01BB10AF14A
S315080147C80803249A1360504617B0BDE8F08F209B5A
S315080147D8012B7FF72EAE0E9B0A9301204DE6BBF1FE
S315080147E8000F7FF7D9AE564621460398FFF7B8F961
S315080147F800F1300306F8013BA6EB0A029345B4DD3E
S3150801480800230A224846039900F05EFC0390EBE769
S3150801481834620108B86101082DE9F0471F468E6818
S315080148288246BE420C4690460B682DD8B1F90C2033
S3150801483812F4906F26D06569096905EB4505A3EB5E
S31508014848010905EBD5757B1C4B446D109D4238BF94
S315080148581D46530527D5294600F0A0FA064660B332
S315080148684A462169FFF750F9A38923F4906343F06F
S315080148788003A38126614E4426603E466561A5EB01
S315080148880905A560BE4200D93E463246414620681A
S3150801489801F0ABF80020A3689B1BA3602368334487
S315080148A82360BDE8F0872A4600F07CFF0646002803
S315080148B8E0D15046216901F047F90C23CAF80030BE
S315080148C8A3894FF0FF3043F04003A381E9E70000CD
S315080148D82DE9F04F98468B8907461B060D4614465F
S315080148E89DB010D50B6973B9402100F057FA2860B5
S315080148F8286130B90C233B604FF0FF301DB0BDE885
S31508014908F08F40236B610023099320238DF8293002
S3150801491830234FF00109CDF80C80DFF898818DF81E
S315080149282A3023469A4613F8012B0AB1252AF9D1C2
S31508014938BAEB040B0BD05B46224629463846FFF7E5
S315080149486BFF013000F0A780099A5A4409929AF830
S315080149580030002B00F09F8000234FF0FF32CDE98D
S3150801496805230AF1010A049307938DF853301A931C
S315080149785446052214F8011B4E48FFF7B7F8049A5E
S31508014988D8B9D00644BF20238DF85330110744BF40
S315080149982B238DF853309AF800302A2B15D0544614
S315080149A800204FF00A0C079A214611F8013B303BC3
S315080149B8092B4BD9B0B1079214E0A0EB080309FA01
S315080149C803F31343A2460493D2E7039B191D1B68F5
S315080149D80391002BBBBF5B4242F002020793079380
S315080149E8B8BF049223782E2B0AD163782A2B32D1A1
S315080149F8039B02341A1D1B68039243EAE373059362
S31508014A08DFF8B4A0032250462178FFF76FF838B1CA
S31508014A184022049BA0EB0A00824013430134049305
S31508014A2814F8011B062225488DF82810FFF75EF8A9
S31508014A38002836D0224B1BBB039B073323F00703F9
S31508014A4808330393099B334409936AE70C46012003
S31508014A580CFB0232A8E700234FF00A0C1946013469
S31508014A680593204610F8012B303A092A03D9002B59
S31508014A78C6D00591C4E7044601230CFB0121F0E7DA
S31508014A8803AB00932A4638460E4B04A9FEF728FBC2
S31508014A98421C0646D6D1AB895B063FF52DAF099868
S31508014AA82CE703AB00932A463846064B04A9FEF7BA
S31508014AB8B5FDEDE7456201084B6201084F62010839
S31508014AC8E930010821480108936810B4013B002B15
S31508014AD8936007DA9469A34201DB0A2902D110BC5B
S31508014AE800F08EBE1368581C10601970084610BC71
S31508014AF87047F8B506460F461446D518AC4201D193
S31508014B08002007E03A46304614F8011BFFF7DCFF98
S31508014B18431CF3D1F8BD00002DE9F04F0D461446A4
S31508014B28984606469DB018B1036A0BB9FEF720FFE9
S31508014B386B6ED90705D4AB899A0502D4A86DFEF719
S31508014B48CEFFAB891B0701D52B699BB92946304688
S31508014B5800F094FE70B16B6EDC0704D54FF0FF3098
S31508014B681DB0BDE8F08FAB899805F7D4A86DFEF797
S31508014B78B7FFF3E70023099320238DF8293030235B
S31508014B884FF00109CDF80C80DFF8A8818DF82A3095
S31508014B9823469A4613F8012B0AB1252AF9D1BAEB05
S31508014BA8040B0BD05B46224629463046FFF7A1FF80
S31508014BB8013000F0A780099A5A4409929AF80030F8
S31508014BC8002B00F09F8000234FF0FF32CDE9052323
S31508014BD80AF1010A049307938DF853301A93544638
S31508014BE8052214F8011B5348FEF780FF049AD8B921
S31508014BF8D10644BF20238DF85330130744BF2B230E
S31508014C088DF853309AF800302A2B15D054460020CF
S31508014C184FF00A0C079A214611F8013B303B092B3C
S31508014C284BD9B0B1079214E0A0EB080309FA03F3CC
S31508014C381343A2460493D2E7039B191D1B680391E4
S31508014C48002BBBBF5B4242F0020207930793B8BF2A
S31508014C58049223782E2B0AD163782A2B32D1039B07
S31508014C6802341A1D1B68039243EAE3730593DFF8B6
S31508014C78C8A0032250462178FEF738FF38B14022EA
S31508014C88049BA0EB0A00824013430134049314F8E9
S31508014C98011B062229488DF82810FEF727FF002848
S31508014CA83FD0274B1BBB039B073323F00703083366
S31508014CB80393099B3B4409936AE70C4601200CFBBD
S31508014CC80232A8E700234FF00A0C19460134059366
S31508014CD8204610F8012B303A092A03D9002BC6D0E9
S31508014CE80591C4E7044601230CFB0121F0E703AB50
S31508014CF800932A463046134B04A9FEF7F1F90746ED
S31508014D08781CD6D16B6ED90705D4AB899A0502D416
S31508014D18A86DFEF7E5FEAB895B063FF51FAF099857
S31508014D281EE703AB00932A463046064B04A9FEF74D
S31508014D3875FCE4E7456201084B6201084F62010800
S31508014D48E9300108FB4A0108024B0146186800F0D8
S31508014D5825B800BF8400002070B50F4E0C4631688F
S31508014D68054611B900F090FE30602146284600F044
S31508014D788BFE431C03D14FF0FF34204670BDC41C7B
S31508014D8824F00304A042F8D0211A284600F07CFE34
S31508014D980130F2D1EFE700BF201300202DE9F843CF
S31508014DA8CD1C25F0030508350C2D38BF0C25002D1B
S31508014DB8064601DBA94204D90C2333600020BDE865
S31508014DC8F883DFF8D48000F011F9D8F800301C46CA
S31508014DD844BB29463046FFF7BFFF431C044658D152
S31508014DE8D8F800402746002F43D1002C4BD023681A
S31508014DF83946304604EB030900F046FE814542D19F
S31508014E08216830466D1A2946FFF7A6FF01303AD0C0
S31508014E1823682B442360D8F800305A6862BBC8F85F
S31508014E2800700FE02268521B20D40B2A17D9611982
S31508014E38A342256018BF5960636808BFC8F80010FF
S31508014E4862514B60304600F0D7F804F10B00231D78
S31508014E5820F00700C21A1CBF1B1AA350AFE76268E5
S31508014E68A3420CBFC8F800205A60EBE723466468DA
S31508014E78AEE73C467F68B6E71A465B68A342FBD1AC
S31508014E8800235360DEE70C233046336000F0B4F89C
S31508014E9894E70560D6E700BF24130020B1F90C2072
S31508014EA8F8B5160705460C4654D44B68002B02DCA0
S31508014EB80B6C002B48DDE66A002E45D0002312F458
S31508014EC880522F68216A2B6030D0626DA3895907F1
S31508014ED805D56368D21A636B0BB1236CD21A002302
S31508014EE82846E66A216AB047431CA38906D1296878
S31508014EF81D292BD8284ACA40D60727D50022626019
S31508014F082269D904226004D5421C01D12B6803B948
S31508014F186065616B2F60B9B104F14403994202D007
S31508014F28284600F011FE002363630DE00123284695
S31508014F38B0470246501CC9D12B68002BC6D01D2B79
S31508014F4801D0162B1DD12F60002021E043F0400324
S31508014F581BB21AE00F69002FF6D0930718BF002372
S31508014F680E6808BF4B69F61B0F608B60002EEBDDD8
S31508014F7833463A462846216AD4F828C0E047002825
S31508014F8807DCB4F90C3043F040034FF0FF30A38136
S31508014F98F8BD0744361AE9E70100402038B50B6918
S31508014FA805460C4613B90025284638BD18B1036AC3
S31508014FB80BB9FEF7DDFCB4F90C30002BF3D0626EA1
S31508014FC8D00704D4990502D4A06DFEF788FD2846B2
S31508014FD82146FFF763FF636E0546DA07E4D4A3891A
S31508014FE89B05E1D4A06DFEF77BFDDDE70148FEF7D9
S31508014FF876BD00BF1C1300200148FEF771BD00BF2E
S315080150081C13002070B5C66904460D4676B91020EA
S31508015018FFF79AFE0246E06120B96B21174B18483B
S31508015028FEF780FDC0E901660660C660E669F368B1
S3150801503883B1E369DB6853F82500B8B9012101FA98
S3150801504805F6721D2046920000F069FD60B1C0E9B7
S3150801505801560EE021220421204600F060FDE3698D
S31508015068F060DB68002BE4D1002070BD026843F8C4
S3150801507825200023C0E90333F7E700BFC561010806
S315080150885662010870B5C66905460C4676B91020F8
S31508015098FFF75AFE0246E86120B98F21084B0948ED
S315080150A8FEF740FDC0E901660660C6603CB1EB69DA
S315080150B86268DB6853F82210216043F8224070BD04
S315080150C8C5610108566201082DE9F04107460C46F3
S315080150D81E4600200D6901F1140CDCF80030013078
S315080150E899B202FB01611E0C0B0C02FB063389B24D
S315080150F801EB034185424FEA13464CF8041BECDCE5
S315080151080EB3A368AB4219DC616838460131FFF76B
S3150801511879FF804628B90246BA210C4B0C48FEF796
S3150801512801FD226904F10C01023292000C30FEF7E6
S31508015138EBFC21463846FFF7A5FF444604EB8503F1
S3150801514801355E6125612046BDE8F08134620108B2
S31508015158566201080346B0F5803F3ABF030410209A
S315080151680020B3F1807F3CBF1B020830B3F1805F92
S315080151783CBF1B010430B3F1804F3CBF9B00023092
S31508015188002B05DB13F0804F00F1010008BF202032
S3150801519870470368024613F007000BD0D90721D4D4
S315080151A8980749BF5B089B08012013605CBF02206A
S315080151B81360704799B209B910201B0CD9B209B9FD
S315080151C808301B0A190704BF1B090430990704BFCD
S315080151D89B080230D90703D45B0800F1010003D004
S315080151E813607047002070472020704710B50C4699
S315080151F80121FFF707FF024628B940F24511044B7A
S315080152080448FEF78FFC01234461036110BD00BF02
S3150801521834620108566201082DE9F04F17460A69F2
S315080152283B6989469A42A2BF3B460F4699463D695C
S31508015238D9F810A0BB68796805EB0A06B34285B0A8
S31508015248B8BF0131FFF7DEFE30B902464FF4B17136
S31508015258404B4148FEF766FC00F114042346002238
S3150801526804EB860E734520D307F1140809F11401D6
S3150801527808EB850501EB8A030293EB1B153B23F023
S31508015288030304331537BD4238BF04230193029B30
S3150801529803918B420CD8002E03DD5EF8043D002BE2
S315080152A855D0066105B0BDE8F08F43F8042BD9E758
S315080152B8B1F800A0BAF1000F1FD0C446A1460027CD
S315080152C85CF8042BD9F800301FFA82FB9BB20AFB5B
S315080152D80B333B44D9F80070120C3F0C0AFB0272D7
S315080152E802EB13429BB243EA024365454FEA12476A
S315080152F849F8043BE4D8019BE750039B0431B3F80A
S315080153080290B9F1000F20D04746A4464FF0000A8B
S315080153182368B7F800B0BCF802209BB209FB0B2238
S31508015328524443EA02434CF8043B57F8043B4FEA14
S31508015338134ABCF80030BD4209FB0A3303EB124392
S315080153484FEA134AE5D8019AA35004349FE7013E68
S31508015358A1E700BF34620108566201082DE9F8433E
S31508015368154612F0030207460E4607D0254C013AA0
S31508015378002354F82220FFF7A7FE0646AD103DD0B4
S31508015388FC697CB91020FFF7DFFC0246F86128B9E9
S3150801539840F2B3111C4B1D48FEF7C4FBC0E9014492
S315080153A80460C460D7F81C80D8F808404CB940F2A4
S315080153B871213846FFF71AFF00230446C8F8080082
S315080153C803604FF00009EB070AD5314622463846ED
S315080153D8FFF722FF804631463846FFF753FE464611
S315080153E86D100BD0206838B9224621463846FFF792
S315080153F813FF2060C0F800900446E4E73046BDE88C
S31508015408F88300BFBC620108C56101085662010834
S315080154182DE9F0470C46074691462369496803EB87
S315080154286218A3684FEA621A08F10106B3420BDB50
S315080154383846FFF7E7FD054648B902464FF4EF71C6
S31508015448274B2848FEF76EFB01315B00EEE7002380
S3150801545800F1140100F110021846534533DB20699F
S315080154682AEAEA7A04F1140319F01F0901EB8A01F9
S3150801547803EB800C2BD08A460022C9F1200E186846
S3150801548800FA09F010434AF8040B53F8042B9C4513
S3150801549822FA0EF2F3D8ACEB0403153B23F0030307
S315080154A8043304F11500604588BF0423CA500AB1BC
S315080154B808F10206013E384621462E61FFF7E2FD4C
S315080154C82846BDE8F08742F8040F0133C5E70439D1
S315080154D853F8042B9C4541F8042FF9D8EAE700BF8D
S315080154E8346201085662010803460A69006930B53B
S315080154F8801A0ED11433143103EB820401EB8201AD
S3150801550854F8045D51F8042D954203D005D24FF09D
S31508015518FF3030BDA342F3D3FBE70120F9E70000CA
S315080155282DE9F74F89460646114648461446FFF7B8
S31508015538DBFF051E12D129463046FFF763FD0246F1
S3150801554828B940F237213E4B3E48FEF7EBFA0123CC
S31508015558C0E90435104603B0BDE8F08FBCBF4B4619
S31508015568A1463046D9F80410BABF1C4601250025BC
S31508015578FFF748FD024618B940F24521304BE3E7E3
S3150801558800F1140BD9F8107009F11003C5604FF032
S31508015598000C09F11405D946266904F1140E05EB20
S315080155A887080EEB86060193019B5EF8040B53F8F0
S315080155B804AF81B201931FFA8AF35B1A000C63449C
S315080155C8C0EB1A4000EB23409BB243EA00437645F9
S315080155D84FEA204C49F8043BE6D8331B153B23F020
S315080155E8030315340433A64238BF04231D445B4418
S315080155F81E462C4644450ED308F10301491B21F0E2
S315080156080301033DA84538BF00210B4453F8041D7F
S3150801561899B117619EE7E64654F8041B1FFA81FCFF
S31508015628F444080C714400EB2C4089B241EA004164
S315080156384FEA204C46F8041BDCE7013FE6E700BFC2
S3150801564834620108566201082DE97343012190461F
S315080156589946089EFFF7D6FC044630B9024640F239
S315080156680F31234B2348FEF75DFAC9F30A55C9F3E7
S3150801567813030DB143F480130193B8F1000324D041
S3150801568868460093FFF785FDDDE90012D8B1C0F138
S31508015698200302FA03F30B43C24063610192019B9B
S315080156A8002B0CBF01220222A3612261ADB1A5F22A
S315080156B8334505443560C0F13500099B1860204615
S315080156C802B0BDE870836161E9E701A8FFF761FDEA
S315080156D8019B012263612030E7E7A0F2324004EB1F
S315080156E8820330601869FFF735FDC0EB4210E4E71D
S315080156F8346201085662010810B50C46B1F90E1054
S3150801570800F0B0F90028ABBF636DA3891B1823F411
S315080157188053ACBF6365A38110BD2DE9F0411F46CF
S315080157288B890546DB050C46164605D50223002254
S31508015738B1F90E1000F084F9A389324623F480538F
S31508015748A38128463B46B4F90E10BDE8F04100F09E
S31508015758ABB910B50C46B1F90E1000F071F9431C36
S31508015768A38915BF606523F4805343F48053A38145
S3150801577818BFA38110BDB1F90E1000F0A7B9000032
S315080157880EB403B5014603AB054853F8042B006864
S315080157980193FFF7C1F902B05DF804EB03B070474E
S315080157A8840000202DE9F041074614460D4621B923
S315080157B81146BDE8F041FFF7F1BA2AB900F0C4F974
S315080157C825462846BDE8F08100F018FA84420646BF
S315080157D802D8B4EB500FF4D821463846FFF7DEFA5B
S315080157E8804608B94546ECE7B4422246294628BF09
S315080157F83246FEF789F92946384600F0A5F9F1E750
S31508015808F8B50E461446054618B1036A0BB9FEF7EC
S31508015818AFF8A369A360A3891A0701D5236943B910
S315080158282146284600F02AF818B14FF0FF373846BE
S31508015838F8BD23682269F6B2981A6369374683421E
S3150801584805DC21462846FFF7A9FB0028EDD1A36800
S31508015858013BA36023685A1C22601E706269431CB7
S315080158689A4204D0A389DB07E1D50A2EDFD121465E
S315080158782846FFF793FB0028D9D0D6E738B5294B30
S31508015888054618680C4618B1036A0BB9FEF770F88D
S31508015898B4F90C30190722D4DA0607D409222A6082
S315080158A843F040034FF0FF30A38133E0580712D580
S315080158B8616B41B104F14403994202D0284600F0CC
S315080158C843F900236363A38923F02403A3810023EF
S315080158D8636023692360A38943F00803A3812369C5
S315080158E84BB9A38903F42073B3F5007F03D0214686
S315080158F8284600F03EF8B4F90C3013F001020AD034
S315080159080022A26062695242A261226942B913F071
S315080159188000C5D138BD990758BF6269A260F4E706
S315080159280020F7E78400002070B50C46B1F90E107F
S31508015938154600291E4696B00CDAA389002113F0EC
S31508015948800F14BF40234FF48063002031602B6019
S3150801595816B070BD6A4600F0C9F80028EDDB019952
S3150801596801F47041A1F50053594259414FF4806336
S31508015978EBE78B89F7B59D0706460C4607D504F16B
S315080159884703236023610123636103B0F0BD6A46B7
S3150801599801ABFFF7C9FF009F054639463046FFF7B1
S315080159A8FDF948B9B4F90C309A05EED423F0030386
S315080159B843F00203A381E2E7A389C4E9040743F094
S315080159C88003A381019B20605BB13046B4F90E10B0
S315080159D800F026F828B1A38923F0030343F001034D
S315080159E8A381A3891D43A581CFE7884210B501EB99
S315080159F8020402D98442234607D8431EA14208D085
S31508015A0811F8012B03F8012FF8E7014602448A42E7
S31508015A1800D110BD13F8014D02F8014DF7E7000052
S31508015A2838B50023054D044608462B60F7F737FCB9
S31508015A38431C02D12B6803B1236038BD2813002003
S31508015A4838B50446084611460022054D2A601A4605
S31508015A58F7F72FFC431C02D12B6803B1236038BD25
S31508015A682813002038B50446084611460022054D74
S31508015A782A601A46F7F7DCFB431C02D12B6803B1E7
S31508015A88236038BD2813002038B50023054D044680
S31508015A9808462B60F7F71AFC431C02D12B6803B199
S31508015AA8236038BD2813002038B504460846114630
S31508015AB80022054D2A601A46F4F7C6FC431C02D192
S31508015AC82B6803B1236038BD2813002038B5002395
S31508015AD8054D044608462B60F7F7C7FB431C02D158
S31508015AE82B6803B1236038BD2813002038B5002375
S31508015AF8064D0446084611462B60F7F7C1FB431CB9
S31508015B0802D12B6803B1236038BD00BF28130020D2
S31508015B18062008B500F0B0F80120F7F77EFB70B546
S31508015B28A1FB025434B92946FFF738F9064628B9BC
S31508015B38304670BD0C2200260260F9E72A4621463E
S31508015B48FDF79AFFF4E7000038B50546002940D065
S31508015B5851F8043C0C1F002BB8BFE418FFF746FAA6
S31508015B681C4A136833B9636014602846BDE838408F
S31508015B78FFF742BAA34208D9206821188B4201BF08
S31508015B8819685B6809182160EDE71A465B680BB165
S31508015B98A342FAD911685018A0420BD120680144CA
S31508015BA8501883421160E0D118685B680844106090
S31508015BB85360DAE702D90C232B60D6E72068211847
S31508015BC88B4201BF19685B680918216063605460D4
S31508015BD8CBE738BD2413002082B001B901A942B127
S31508015BE84BB113780B601278101E18BF012002B04A
S31508015BF870471046FBE76FF00100F8E751F8043CD7
S31508015C08181F002BBCBF0B58C01870470346084617
S31508015C1841B1FF2A04D98A224FF0FF301A6070472A
S31508015C2801200A7070471F2938B505460C4604D95C
S31508015C38162303604FF0FF3038BDC26B12B152F814
S31508015C4821304BB9284600F031F822460146284644
S31508015C58BDE8384000F018B8012B0AD0591C03D101
S31508015C68162303600120E7E70021204642F824109D
S31508015C7898470020E0E70000024B01461868FFF73D
S31508015C88D2BF00BF8400002038B50023064D04465C
S31508015C98084611462B60F7F7B0FA431C02D12B6860
S31508015CA803B1236038BD00BF28130020F7F79EBA51
S31508015CB8F8B500BFF8BC08BC9E467047F8B500BFE2
S30D08015CC8F8BC08BC9E467047B2
S31508015CD0434F4E4E2564204572726F723A202564F1
S31508015CE00A000000436F6E6E6563746F723A205541
S31508015CF06E6B6E6F776E0A00436F6E6E6563746FB7
S31508015D00723A20556E706C75676765640A00000003
S31508015D10436F6E6E6563746F723A2044697361628C
S31508015D206C65640A00000000436F6E6E6563746FEC
S31508015D30723A20507265706172696E670A000000D6
S31508015D40436F6E6E6563746F723A2041757468525B
S31508015D50657175697265640A00000000436F6E6EAD
S31508015D606563746F723A2057616974696E67466F25
S31508015D7072456E657267790A00000000436F6E6EA0
S31508015D806563746F723A204368617267696E67501A
S31508015D90617573656445560A00000000436F6E6EAF
S31508015DA06563746F723A204368617267696E6750FA
S31508015DB06175736564455653450A0000436F6E6EF7
S31508015DC06563746F723A204368617267696E670A20
S31508015DD000000000436F6E6E6563746F723A20416E
S31508015DE075746854696D656F75740A00436F6E6ED4
S31508015DF06563746F723A2046696E69736865640AE9
S31508015E0000000000436F6E6E6563746F723A204638
S31508015E10696E6973686564455653450A0000000052
S31508015E20436F6E6E6563746F723A2046696E697365
S31508015E3068656445560A0000436F6E6E6563746F44
S31508015E40723A205265706C756767696E670A000059
S31508015E50434F4E4E2564204368617267696E672019
S31508015E6046696E69736865643A0A00004368617237
S31508015E7067696E6720456E657267793A2025640AF7
S31508015E8000000000434353206D6F64756C652073F1
S31508015E90746172740A00000053657269616C206E40
S31508015EA0756D6265723A2025640A0000426F617257
S31508015EB064207265766973696F6E3A2025640A00F3
S31508015EC046572076657273696F6E3A2025642E25CA
S31508015ED0642E25640A000000505355206F6E207405
S31508015EE0696D656F75740A00436F6E746163746FCB
S31508015EF072206572726F722C2073746F7070696E7E
S31508015F00672E2E2E0A000000505355206F66662014
S31508015F1074696D656F75740A000000004553544F26
S31508015F2050207472696767657265640A000000002B
S31508015F3053746F7070696E67206368617267696E02
S31508015F40672E2E2E0A00000046696E69736865641D
S31508015F5045562C2073746F7070696E672E2E2E0A43
S31508015F60000000004368617267696E672065727296
S31508015F706F722025642C207374617465202D3E2070
S31508015F8064697361626C65640A0000004368617242
S31508015F9067696E67207065726D69747465642C2013
S31508015FA07374617274206368617267696E670A0047
S31508015FB043617220756E706C75676765640A0000C7
S31508015FC05265706C756767696E672E2E2E0A00001A
S31508015FD05265706C756767696E672066696E697365
S31508015FE06865642C206275742063617220756E7011
S31508015FF06C75676765640A005265706C75676769D1
S315080160006E672066696E69736865642C20636172C0
S3150801601020706C75676765642C20737461746520DC
S315080160202D3E2061757468207265717569726564A3
S315080160300A000000457665726573742074696D659A
S315080160406F75740A0000000043435320696E697432
S315080160500A0000004576657265737420726573657A
S315080160607420636F6D6D616E640A00005061636B25
S31508016070657420435243206572726F720A000000EC
S31508016080556E6B6E6F776E20636D642030782530A0
S3150801609032780A005061636B6574206C656E206DF9
S315080160A069736D6174636820636D643D307825306A
S315080160B032780A0053657420436F6E6669673A2021
S315080160C025732025640A0000506F776572206C6974
S315080160D06D69743A2025640A0000000043686172FC
S315080160E06765207065726D69743A2025640A000037
S315080160F00000000000000000010203040607080969
S31508016100000000000102030400000405060708094F
S3150801611000000000000D000001020304050607083F
S31508016120090A0B0C0D0E0F100000040506070809D5
S3150801613000000000000D000001020304050607081F
S31508016140090A0B0C0D0E0F10494E4600696E6600C2
S315080161504E414E006E616E003000303132333435B7
S3150801616036373839414243444546003031323334B3
S315080161703536373839616263646566002C20667581
S315080161806E6374696F6E3A20006173736572746920
S315080161906F6E2022257322206661696C65643A2038
S315080161A066696C6520222573222C206C696E652030
S315080161B02564257325730A00496E66696E697479C3
S315080161C0004E614E005245454E54206D616C6C6F10
S315080161D06320737563636565646564002F62756919
S315080161E06C642F676E752D746F6F6C732D666F7285
S315080161F02D73746D33325F31332E332E72656C31E4
S315080162002E32303234303932362D313731352F731B
S3150801621072632F6E65776C69622F6E65776C69623A
S315080162202F6C6962632F7374646C69622F64746F6F
S31508016230612E630042616C6C6F63207375636365DD
S315080162406564656400232D302B2000686C4C00655D
S315080162506667454647002F6275696C642F676E75D8
S315080162602D746F6F6C732D666F722D73746D333267
S315080162705F31332E332E72656C312E323032343023
S315080162803932362D313731352F7372632F6E657773
S315080162906C69622F6E65776C69622F6C6962632F10
S315080162A07374646C69622F6D707265632E63004343
S315080162B000504F534958002E000000000500000009
S315080162C0190000007D0000000080E03779C34143D2
S315080162D0176E05B5B5B89346F5F93FE9034F384D3D
S315080162E0321D30F94877825A3CBF737FDD4F1575E9
S315080162F0000000000000F03F0000000000002440FC
S3150801630000000000000059400000000000408F40D6
S31508016310000000000088C34000000000006AF84041
S315080163200000000080842E4100000000D012634165
S315080163300000000084D797410000000065CDCD41DB
S31508016340000000205FA00242000000E876483742BC
S31508016350000000A2941A6D42000040E59C30A2425A
S315080163600000901EC4BCD64200003426F56B0C43CF
S315080163700080E03779C3414300A0D8855734764376
S3150801638000C84E676DC1AB43003D9160E458E143D7
S31508016390408CB5781DAF154450EFE2D6E41A4B444C
S315080163A092D54D06CFF08044F64AE1C7022DB54491
S315080163B0B49DD9794378EA44002020202020202062
S315080163C02020282828282820202020202020202096
S315080163D020202020202020202088101010101010A6
S315080163E010101010101010101004040404040404F2
S315080163F0040404101010101010104141414141418C
S31508016400010101010101010101010101010101016D
S31508016410010101011010101010104242424242427D
S31508016420020202020202020202020202020202023D
S3150801643002020202101010102000000000000000E5
S31508016440000000000000000000000000000000003D
S31508016450000000000000000000000000000000002D
S31508016460000000000000000000000000000000001D
S31508016470000000000000000000000000000000000D
S3150801648000000000000000000000000000000000FD
S3150801649000000000000000000000000000000000ED
S315080164A000000000000000000000000000000000DD
S311080164B0000000000000000000000000D1
S30D080164BC6C1DFF7F01000000C1
S309080164C40D8200082E
S309080164C8E98100084F
S315080164CCE401000006060600400000320A320040CC
S315080164DC00000000008000320A3200008000000033
S315080164EC0000FA320A32000000FA000000FF0032FE
S315080164FC0A32000020000000FFFFFF320A3200FFBB
S3150801650CFFFF0000FF0000320A320020000064067B
S3150801651C0100000000FFFF00000000000000000061
S3150801652C52555301000000FE529E66000024F400E9
S3150801653C100000000100000000000000030000002C
S3150801654CE01100208800002000000000E011002066
S3150801655C48120020B01200200000000000000000C4
S3150801656C0000000000000000000000000000000010
S3150801657C0000000000000000000000000000000000
S3150801658C00000000000000000000000000000000F0
S3150801659C000000004300000000000000000000009D
S315080165AC00000000000000000000000000000000D0
S315080165BC000000004300000000000000000000007D
S315080165CC00000000000000000000000000000000B0
S315080165DC000000004300000000000000000000005D
S315080165EC0000000000000000000000000000000090
S315080165FC000000004300000000000000000000003D
S3150801660C000000000000000000000000000000006F
S3150801661C000000004300000000000000000000001C
S3150801662C000000000000000000000000000000004F
S3150801663C00000000430000000000000000000000FC
S3150801664C000000000000000000000000000000002F
S3150801665C00000000430000000000000000000000DC
S3150801666C000000000000000000000000000000000F
S3150801667C00000000155C0108E15B01080000000040
S3150801668CB8630108B7620108B7610108B761010867
S3150801669CB7610108B7610108B7610108B76101085B
S315080166ACB7610108B7610108B7610108FFFFFFFF70
S315080166BCFFFFFFFFFFFFFFFFFFFF00000100415334
S315080166CC43494900000000000000000000000000DA
S315080166DC000000000000000000000000000041530B
S315080166EC43494900000000000000000000000000BA
S315080166FC000000000000000000000000000000007F
S7050800DA75A3
